:020000040800F2
:1000000000060020E1020008E3020008E302000805
:10001000E3020008E3020008E3020008E30200082C
:10002000E3020008E3020008E3020008E92A0008EE
:10003000E3020008E3020008E3020008E30200080C
:10004000E3020008E3020008E3020008E3020008FC
:10005000E3020008E3020008E3020008E3020008EC
:10006000E3020008E3020008E302000805110008AB
:100070002D1100085911000885110008B111000860
:10008000D911000805120008E3020008E302000885
:10009000E3020008E3020008E3020008E3020008AC
:1000A000E3020008E3020008E3020008E30200089C
:1000B000E3020008E3020008E3020008E30200088C
:1000C000E3020008E3020008E3020008E30200087C
:1000D000E3020008E3020008E3020008E30200086C
:1000E000E3020008E3020008E3020008E30200085C
:1000F000E3020008E3020008E302000831120008EE
:10010000E3020008E3020008CD420008E302000811
:10011000E3020008E3020008E3020008E30200082B
:100120005D12000885120008B1120008DD120008F7
:1001300009130008E3020008E3020008E3020008D4
:10014000E3020008E3020008E3020008E3020008FB
:10015000311300085D13000889130008E30200084A
:10016000E3020008E3020008E3020008E3020008DB
:10017000E3020008D5360008E3020008E3020008A5
:10018000E3020008E3020008E3020008E3020008BB
:10019000E3020008E3020008E3020008E3020008AB
:1001A000E3020008E3020008E3020008E30200089B
:1001B000E3020008E3020008E3020008E30200088B
:1001C000E3020008E3020008E3020008E30200087B
:1001D000E3020008C1360008E3020008E302000859
:1001E000E3020008E3020008E3020008E30200085B
:1001F000E3020008E3020008E3020008E30200084B
:10020000E3020008E3020008E3020008E30200083A
:10021000E3020008E3020008E3020008E30200082A
:10022000E3020008E3020008E3020008E30200081A
:10023000E3020008E3020008E3020008E30200080A
:10024000E3020008E3020008E3020008E3020008FA
:10025000E3020008E3020008E3020008E3020008EA
:10026000E3020008E3020008E3020008E3020008DA
:10027000E3020008E3020008E3020008E3020008CA
:10028000E3020008E3020008E3020008E3020008BA
:10029000E3020008E3020008E3020008E3020008AA
:1002A000E3020008E3020008E3020008E30200089A
:1002B000E3020008E3020008E3020008E30200088A
:1002C000E3020008E3020008E3020008E30200087A
:1002D000E3020008E3020008E3020008E30200086A
:1002E00002E000F000F8FEE772B6374880F30888B5
:1002F000364880F3098836483649086040F20000E5
:10030000CCF200004EF63471CEF200010860BFF36B
:100310004F8FBFF36F8F40F20000C0F2F0004EF637
:100320008851CEF200010860BFF34F8FBFF36F8F8B
:100330004FF00000E1EE100A4EF63C71CEF20001E3
:100340000860062080F31488BFF36F8F02F02EFC44
:1003500003F076FD4FF055301F491B4A91423CBFD8
:1003600041F8040BFAE71D49184A91423CBF41F895
:10037000040BFAE71A491B4A1B4B9A423EBF51F83D
:10038000040B42F8040BF8E700201849184A914280
:100390003CBF41F8040BFAE702F046FC03F0D4FD41
:1003A000144C154DAC4203DA54F8041B8847F9E7A6
:1003B00000F042F8114C124DAC4203DA54F8041B21
:1003C0008847F9E702F02EBC00060020002200203A
:1003D0000000000808ED00E00000002000060020FA
:1003E000C0470008002200205C220020602200207C
:1003F00004440020E0020008E0020008E0020008D7
:10040000E00200082DE9F04F2DED108AC1F80CD064
:10041000D0F80CD0BDEC108ABDE8F08F002383F338
:1004200011882846A047002001F012FEFEE701F0E7
:100430009DFD00DFFEE7000038B500F037FC00F05E
:10044000B3FD02F011FB054602F044FB0446C0B9BF
:100450000E4B9D4217D001339D4241F2883512BFA9
:10046000044600250124002002F008FB0CB100F036
:1004700073F800F06DFD284600F01CF900F06CF8F0
:10048000F9E70025EFE70546EDE700BF010007B0FB
:1004900008B500F0DDFBA0F120035842584108BD2B
:1004A00007B5042101900DEB010000F0EFFB03B054
:1004B0005DF804FB38B5302383F3118817480368CF
:1004C0000BB101F091FE0023154A4FF47A711348E5
:1004D00001F080FE002383F31188124C236813B1CE
:1004E0002368013B2360636813B16368013B636069
:1004F0000D4D2B7833B963687BB9022000F092FC74
:10050000322363602B78032B07D163682BB9022059
:1005100000F088FC4FF47A73636038BD60220020DD
:10052000B50400088023002078220020084B1870B2
:1005300003280CD8DFE800F008050208022000F0CC
:1005400067BC022000F05ABC024B00225A60704780
:100550007822002080230020F8B5504B504A1C46DA
:100560001968013100F0998004339342F8D1626830
:100570004C4B9A4240F291804B4B9B6803F10063D5
:1005800003F5C0239A4280F08880002000F0A8FB89
:100590000220FFF7CBFF454B0021D3F8E820C3F83A
:1005A000E810D3F81021C3F81011D3F81021D3F8B4
:1005B000EC20C3F8EC10D3F81421C3F81411D3F8CD
:1005C0001421D3F8F020C3F8F010D3F81821C3F8A1
:1005D0001811D3F81821D3F8802042F00062C3F834
:1005E0008020D3F8802022F00062C3F88020D3F866
:1005F0008020D3F8802042F00072C3F88020D3F826
:10060000802022F00072C3F88020D3F8803072B6C8
:100610004FF0E023C3F8084DD4E90004BFF34F8F37
:10062000BFF36F8F224AC2F88410BFF34F8F536914
:1006300023F480335361BFF34F8FD2F8803043F6F9
:10064000E076C3F3C905C3F34E335B0103EA060C3E
:1006500029464CEA81770139C2F87472F9D2203BFD
:1006600013F1200FF2D1BFF34F8FBFF36F8FBFF3A2
:100670004F8FBFF36F8F536923F40033536100230F
:10068000C2F85032BFF34F8FBFF36F8F302383F325
:100690001188854680F308882047F8BD00000608C9
:1006A00020000608FFFF0508002200200044025831
:1006B00000ED00E02DE9F04F95B0DFF8D892202250
:1006C000FF21029004A8D9F8085000F0EBFBA84ADB
:1006D0001378A3B90121A74811700360302383F375
:1006E000118803680BB101F07FFD0023A24A4FF48B
:1006F0007A71A04801F06EFD002383F31188029BFC
:1007000013B19E4B029A1A609D4A1378032B03D0B3
:1007100000231370994A53604FF0000B029C5E4611
:10072000DA46CDF804B0012000F072FB24B1934BFF
:100730001B68002B00F02882002000F089FAB0F13D
:100740000008F3DB012000F059FBA8F121031F2B67
:10075000E9D801A252F823F0D9070008F5070008EC
:100760008308000827070008270700082707000854
:100770000D090008FF0A0008F10900084D0A0008E9
:10078000730A0008990A000827070008AB0A000846
:10079000CF0A0008470B0008610800082707000877
:1007A0008F0B0008E507000861080008270700080C
:1007B0004D0A000827070008270700082707000838
:1007C0002707000827070008270700082707000851
:1007D00027070008830800080220FFF759FE0028B9
:1007E00040F0FF81029B02216648BBF1000F08BF69
:1007F0001C4640E04FF47A7000F02AFA071EF1DB45
:100800000220FFF745FE0028ECD0013F052F00F243
:10081000EA81DFE807F003070A0D10330520FFF730
:100820003FFE14E0D9F80000F9E7D9F80400F6E734
:10083000D9F80800F3E74FF01C08404608F1040817
:1008400000F050FAFFF72CFEB8F12C0FF5D1012083
:10085000019B4FF0000A00FA07F71F43FBB2019318
:1008600000F06CFB2EB1019B03F00B030B2B08BFB8
:1008700000240221444800F009FA54E7D9F80C009A
:10088000CDE7002EAED0019B03F00B030B2BA9D1BB
:100890000220FFF7FDFD07460028A3D00120002617
:1008A00000F01EFA0220FFF741FE1FFA86FB5846B1
:1008B00000F026FA044688B1A8F1400258460136F5
:1008C0005142514100F02CFA0028EED1BB460446BB
:1008D00002212E483E4600F0D9F924E725460120A2
:1008E000FFF724FED9F80830AB4207D9284600F0BC
:1008F000F9F9013040F07A810435F3E70025204B07
:10090000BB463E461D701D4B5D60A9E7002E3FF4BF
:1009100069AF019B03F00B030B2B7FF463AF022045
:10092000FFF704FE322000F093F9B0F10008FFF663
:1009300059AF18F003077FF455AF08EB0503D9F85A
:10094000082093423FF64EAFB8F5807F3FF74AAF9D
:100950000F4BB84503931FDD4FF47A7000F078F920
:100960000028FFF63FAF039B013703F8010BF0E7C8
:100970007C23002060220020B50400088023002092
:1009800078220020644300085C43000860430008AC
:100990007C22002000220020C820FFF779FD0746B6
:1009A00000283FF41FAF1F2D11D8C5F1200204AB62
:1009B00025F003008F494245184428BF4246039260
:1009C00000F04AFA039AFF218A4800F06BFA4FEAD6
:1009D000A803C8F3870287492846039300F06AFA00
:1009E000064600283FF474AF039B05EB830537E709
:1009F0000220FFF74DFD00283FF4F4AE00F0AEF901
:100A000000283FF4EFAE0027B846D9F80830BB42C3
:100A100018D91F2F11D8049B01330ED027F00303E0
:100A200014AA134453F8403C0C93404604220CA9EA
:100A3000043700F051FB8046E7E7384600F052F9F2
:100A40000C90F2E74046FFF72BFD09E700236421F5
:100A50000CA80C9300F010F900287FF4C3AE02201C
:100A6000FFF716FD00283FF4BDAE0C9800F06CF9BE
:100A7000E9E7002364210CA80C9300F0FDF800289E
:100A80007FF4B0AE0220FFF703FD00283FF4AAAECA
:100A90000C9800F05BF9D6E70220FFF7F9FC00287C
:100AA0003FF4A0AE00F06AF9CDE70220FFF7F0FCBA
:100AB00000283FF497AE0CA9142000F065F90390CC
:100AC000FFF7EEFC03990CA800F0E0F8C8E602205E
:100AD000FFF7DEFC00283FF485AE474B0CAF03F177
:100AE000100C1868083353F8041C3A46634503C2D7
:100AF0001746F6D11020FFF7D3FC1021E3E7322090
:100B000000F0A6F8071EFFF66DAEBB077FF46AAED5
:100B100007EB0A03D9F8082093423FF663AE0220A0
:100B2000FFF7B6FC00283FF45DAE27F003075744FB
:100B3000BA453FF495AE50460AF1040A00F0D2F8E7
:100B4000FFF7AEFCF4E74FF47A70FFF7A1FC002842
:100B50003FF448AE00F002F9002849D0049B01336D
:100B60000BD0082204A9002000F0A4F900283FD0EF
:100B70002022FF2104A800F095F92048022100F06E
:100B800085F81F4801F06AFA15B0BDE8F08F002E15
:100B90003FF428AE019B03F00B030B2B7FF422AE36
:100BA000002364210CA80C9300F066F80746002887
:100BB0007FF418AE0220FFF76BFC804600283FF45C
:100BC00011AE02210D4800F061F841F2883001F0C9
:100BD00045FA0C9800F0E6F946463C4600F0AEF9BE
:100BE000A1E506463CE64FF0000AFBE5BB466FE692
:100BF00037466DE67C220020484300085C4300082D
:100C0000A08601000F4B70B51B780C460133DBB298
:100C1000012B11D80C4D4FF47A732968A2FB0332D3
:100C200022460E6A01462846B047844204D1074B4B
:100C3000002201201A7070BD4FF4FA7001F00EFA14
:100C40000020F8E710220020B0260020B423002066
:100C5000002307B5024601210DF107008DF807308A
:100C6000FFF7D0FF20B19DF8070003B05DF804FB4B
:100C70004FF0FF30F9E700000A46042108B5FFF7FE
:100C8000C1FF80F00100C0B2404208BD30B4054C45
:100C90000A46014623682046DD69034BAC4630BC5A
:100CA000604700BFB0260020A086010070B50A4E44
:100CB00000240A4D01F0F0FC30802868338883421C
:100CC00008D901F0E5FC2B6804440133B4F5C02FCA
:100CD0002B60F2D370BD00BFB62300208823002014
:100CE00001F0B4BD00F1006000F5C020006870475D
:100CF00000F10060920000F5C02001F029BD000065
:100D0000054B1A68054B1B889B1A834202D9104475
:100D100001F0BEBC0020704788230020B6230020CD
:100D200038B50446074D29B128682044BDE838404D
:100D300001F0C6BC2868204401F0B0FC0028F3D0C4
:100D400038BD00BF882300200020704700F1FF500D
:100D500000F58F10D0F8000870470000064991F8A0
:100D6000243033B100230822086A81F82430FFF7C9
:100D7000BFBF0120704700BF8C230020014B1868C3
:100D8000704700BF0010005C194B01380322084473
:100D900070B51D68174BC5F30B042D0C1E88A642B9
:100DA0000BD15C680A46013C824213460FD214F90B
:100DB000016F4EB102F8016BF6E7013A03F1080347
:100DC000ECD181420B4602D22C2203F8012B0424E1
:100DD000094A1688AE4204D1984284BF967803F837
:100DE000016B013C02F10402F3D1581A70BD00BF3F
:100DF0000010005C1422002094430008022803D154
:100E0000024B4FF000629A61704700BF000C02581D
:100E1000022803D1024B4FF400629A61704700BF71
:100E2000000C0258022804D1024A536983F400637B
:100E300053617047000C025870B504464FF47A763F
:100E40004CB1412C254628BF412506FB05F0641B0B
:100E500001F004F9F4E770BD002310B5934203D00C
:100E6000CC5CC4540133F9E710BD0000013810B563
:100E700010F9013F3BB191F900409C4203D11AB1F6
:100E80000131013AF4E71AB191F90020981A10BD26
:100E90001046FCE703460246D01A12F9011B00294E
:100EA000FAD1704702440346934202D003F8011B73
:100EB000FAE770472DE9F8431F4D14460746884668
:100EC00095F8242052BBDFF870909CB395F824303D
:100ED0002BB92022FF2148462F62FFF7E3FF95F848
:100EE00024004146C0F1080205EB8000A24228BF61
:100EF0002246D6B29200FFF7AFFF95F82430A41B2C
:100F000017441E449044E4B2F6B2082E85F82460DB
:100F1000DBD1FFF723FF0028D7D108E02B6A03EBD2
:100F200082038342CFD0FFF719FF0028CBD10020E6
:100F3000BDE8F8830120FBE78C230020024B1A78E0
:100F4000024B1A70704700BFB4230020102200200B
:100F500010B5114C114800F0B1FB21460F4800F0CC
:100F6000D9FB24684FF47A70D4F89020D2F8043872
:100F700043F00203C2F80438FFF75EFF0849204639
:100F800000F0D6FCD4F89020D2F8043823F0020305
:100F9000C2F8043810BD00BF50450008B02600203C
:100FA00058450008704700002DE9F04771B6464BE0
:100FB00001201D68454BB3F8008000231A461946EE
:100FC00000F08AFA0446802001F0DEFC0746002883
:100FD00062D0002C60D03E4EADB24FF0800A7369F3
:100FE000284643F0C0637361D6F8143143F0C06300
:100FF000C6F8143101F04CFB05EB080200FB05F3C9
:101000004FF4D06C50434FF03D0E984233D93269C3
:10101000520144D4D6F81021510140D4216803F183
:1010200000628A602268D7602268C2F804A0226841
:10103000C2F800C0D4F80090D9F8002042F00102B4
:10104000C9F80020D4F80090D9F8002022F01E0240
:10105000C9F80020D4F80090D9F80020D207FBD4BA
:1010600094F80C90803361680EFA09F20A60CCE7BC
:10107000002001F0EBFB204600F06EFA384601F04C
:10108000B9FC134B5A6942F0C0625A61D3F814217B
:1010900042F0C062C3F8142161B6BDE8F0870D4B81
:1010A0009A6A42F400729A629A6A42F400429A6220
:1010B00061B60026012001F0C9FBB045D8D9A819B6
:1010C000013601F0FDFAF8E788230020B62300205E
:1010D0000020005200ED00E030B50A44084D914276
:1010E0000DD011F8013B5840082340F30004013BA8
:1010F0002C4013F0FF0384EA5000F6D1EFE730BD37
:101100002083B8ED08B5074B074A196801F03D0187
:10111000996053680BB190689847BDE8084001F0AA
:101120001BBD00BF00000240B823002008B5084BDB
:101130001968890901F03D018A019A60054AD3685E
:101140000BB110699847BDE8084001F005BD00BF2C
:1011500000000240B823002008B5084B1968090CAC
:1011600001F03D010A049A60054A53690BB1906988
:101170009847BDE8084001F0EFBC00BF0000024006
:10118000B823002008B5084B1968890D01F03D010E
:101190008A059A60054AD3690BB1106A9847BDE881
:1011A000084001F0D9BC00BF00000240B823002075
:1011B00008B5074B074A596801F03D01D960536AE9
:1011C0000BB1906A9847BDE8084001F0C5BC00BF6C
:1011D00000000240B823002008B5084B596889096F
:1011E00001F03D018A01DA60054AD36A0BB1106B48
:1011F0009847BDE8084001F0AFBC00BF00000240C6
:10120000B823002008B5084B5968090C01F03D01CE
:101210000A04DA60054A536B0BB1906B9847BDE83E
:10122000084001F099BC00BF00000240B823002034
:1012300008B5084B5968890D01F03D018A05DA604F
:10124000054AD36B0BB1106C9847BDE8084001F01C
:1012500083BC00BF00000240B823002008B5074B44
:10126000074A196801F03D019960536C0BB1906C0D
:101270009847BDE8084001F06FBC00BF0004024081
:10128000B823002008B5084B1968890901F03D0111
:101290008A019A60054AD36C0BB1106D9847BDE87E
:1012A000084001F059BC00BF00040240B8230020F0
:1012B00008B5084B1968090C01F03D010A049A6051
:1012C000054A536D0BB1906D9847BDE8084001F099
:1012D00043BC00BF00040240B823002008B5084BFF
:1012E0001968890D01F03D018A059A60054AD36DA0
:1012F0000BB1106E9847BDE8084001F02DBC00BF4F
:1013000000040240B823002008B5074B074A59687B
:1013100001F03D01D960536E0BB1906E9847BDE866
:10132000084001F019BC00BF00040240B8230020AF
:1013300008B5084B5968890901F03D018A01DA6056
:10134000054AD36E0BB1106F9847BDE8084001F015
:1013500003BC00BF00040240B823002008B5084BBE
:101360005968090C01F03D010A04DA60054A536F1F
:101370000BB1906F9847BDE8084001F0EDBB00BF8E
:1013800000040240B823002008B5084B5968890DB5
:1013900001F03D018A05DA60054AD36F13B1D2F836
:1013A00080009847BDE8084001F0D6BB0004024029
:1013B000B823002000230C4910B51A460B4C0B60D3
:1013C00054F82300026001EB430004334260402BD9
:1013D000F6D1074A4FF0FF339360D360C2F8083468
:1013E000C2F80C3410BD00BFB8230020A44300088D
:1013F000000002400F28F8B510D9102810D011288D
:1014000011D0122808D10F240720DFF8C8E00126E8
:10141000DEF80050A04208D9002653E00446F4E765
:101420000F240020F1E70724FBE706FA00F73D420E
:101430004AD1264C4FEA001C3D4304EB00160EEB4C
:10144000C000CEF80050C0E90123FBB273B12048C0
:10145000D0F8D83043F00103C0F8D830D0F80031CC
:1014600043F00103C0F80031D0F8003117F47F4F8A
:101470000ED01748D0F8D83043F00203C0F8D83067
:10148000D0F8003143F00203C0F80031D0F8003149
:1014900054F80C00036823F01F030360056815F07F
:1014A0000105FBD104EB0C033D2493F80CC05F68ED
:1014B00004FA0CF43C6021240560446112B1987B6D
:1014C00000F054F83046F8BD0130A3E7A44300080B
:1014D00000440258B823002010B5302484F311884A
:1014E000FFF788FF002383F3118810BD10B5044671
:1014F000807B00F051F801231549627B03FA02F268
:101500000B6823EA0203DAB20B6072B9114AD2F80F
:10151000D81021F00101C2F8D810D2F8001121F042
:101520000101C2F80011D2F8002113F47F4F0ED14F
:10153000084BD3F8D82022F00202C3F8D820D3F801
:10154000002122F00202C3F80021D3F8003110BDBF
:10155000B82300200044025808B5302383F31188D3
:10156000FFF7C4FF002383F3118808BD090100F1D0
:101570006043012203F56143C9B283F8001300F010
:101580001F039A4043099B0003F1604303F5614345
:10159000C3F880211A60704700F01F0301229A40AF
:1015A000430900F160409B0000F5614003F1604396
:1015B00003F56143C3F88020C3F88021002380F83D
:1015C00000337047026843681143016003B1184754
:1015D0007047000013B5406B00F58054D4F8A43870
:1015E0001A681178042914D1017C022911D11979C2
:1015F000012312898B4013420BD101A94C3002F018
:101600009BF9D4F8A4480246019B2179206800F098
:10161000DFF902B010BD0000143002F01DB9000067
:101620004FF0FF33143002F017B900004C3002F0D5
:10163000EFB900004FF0FF334C3002F0E9B9000081
:10164000143002F0EBB800004FF0FF31143002F01C
:10165000E5B800004C3002F0BBB900004FF0FF329B
:101660004C3002F0B5B900000020704710B500F50D
:101670008054D4F8A4381A681178042917D1017C51
:10168000022914D15979012352898B4013420ED17A
:10169000143002F07DF8024648B1D4F8A4484FF463
:1016A000407361792068BDE8104000F07FB910BD3B
:1016B000406BFFF7DBBF0000704700007FB5124BA7
:1016C00001250426044603600023057400F184020A
:1016D00043602946C0E902330C4B02901430019359
:1016E0004FF44073009602F02FF8094B04F6944231
:1016F000294604F14C000294CDE900634FF4407395
:1017000002F0F6F804B070BDA4440008B116000859
:10171000D51500080A68302383F311880B790B3341
:1017200042F823004B79133342F823008B7913B12D
:101730000B3342F8230000F58053C3F8A4180223AA
:101740000374002080F311887047000038B5037FD0
:10175000044613B190F85430ABB90125201D022185
:10176000FFF730FF04F114006FF00101257700F05E
:101770009DFC04F14C0084F854506FF00101BDE869
:10178000384000F093BC38BD10B501210446043048
:10179000FFF718FF0023237784F8543010BD0000B2
:1017A00038B504460025143001F0E6FF04F14C0082
:1017B000257702F0B5F8201D84F854500121FFF779
:1017C00001FF2046BDE83840FFF750BF90F8803059
:1017D00003F06003202B06D190F881200023212AFA
:1017E00003D81F2A06D800207047222AFBD1C0E95F
:1017F0001D3303E0034A426707228267C367012063
:10180000704700BF2C22002037B500F58055D5F871
:10181000A4381A68117804291AD1017C022917D139
:101820001979012312898B40134211D100F14C0424
:10183000204602F035F958B101A9204602F07CF8A3
:10184000D5F8A4480246019B2179206800F0C0F831
:1018500003B030BD01F10B03F0B550F8236085B043
:1018600004460D46FEB1302383F3118804EB85074F
:10187000301D0821FFF7A6FEFB6806F14C005B69EE
:101880001B681BB1019002F065F8019803A902F0F2
:1018900053F8024648B1039B2946204600F098F8C9
:1018A000002383F3118805B0F0BDFB685A69126804
:1018B000002AF5D01B8A013B1340F1D104F18002CC
:1018C000EAE70000133138B550F82140ECB130237D
:1018D00083F3118804F58053D3F8A4281368527950
:1018E00003EB8203DB689B695D6845B104216018E6
:1018F000FFF768FE294604F1140001F053FF20466B
:10190000FFF7B4FE002383F3118838BD7047000051
:1019100001F020BA01234022002110B5044600F84E
:10192000303BFFF7BFFA0023C4E9013310BD0000CC
:1019300010B53023044683F311882422416000212E
:101940000C30FFF7AFFA204601F026FA0223002000
:10195000237080F3118810BD70B500EB810305463C
:1019600050690E461446DA6018B110220021FFF7C4
:1019700099FAA06918B110220021FFF793FA3146B5
:101980002846BDE8704001F00DBB000083682022AE
:10199000002103F0011310B5044683601030FFF7F7
:1019A00081FA2046BDE8104001F088BBF0B4012563
:1019B00000EB810447898D40E4683D43A46945817B
:1019C00023600023A2606360F0BC01F0A5BB0000AF
:1019D000F0B4012500EB810407898D40E4683D43A4
:1019E0006469058123600023A2606360F0BC01F09C
:1019F0001BBC000070B5022300250446242203709E
:101A00002946C0F888500C3040F8045CFFF74AFAC9
:101A1000204684F8705001F059FA63681B6823B1BE
:101A200029462046BDE87040184770BD0378052B55
:101A300010B504460AD080F88C3005230370436843
:101A40001B680BB1042198470023A36010BD000060
:101A50000178052906D190F88C20436802701B6834
:101A600003B118477047000070B590F87030044615
:101A700013B1002380F8703004F18002204601F099
:101A800041FB63689B68B3B994F8803013F060053C
:101A900035D00021204601F033FE0021204601F020
:101AA00023FE63681B6813B106212046984706236E
:101AB00084F8703070BD204698470028E4D0B4F810
:101AC0008630A26F9A4288BFA36794F98030A56FD1
:101AD000002B4FF0300380F20381002D00F0F280E4
:101AE000092284F8702083F3118800212046D4E96C
:101AF0001D23FFF76DFF002383F31188DAE794F8C5
:101B0000812003F07F0343EA022340F20232934232
:101B100000F0C58021D8B3F5807F48D00DD8012BC7
:101B20003FD0022B00F09380002BB2D104F1880249
:101B300062670222A267E367C1E7B3F5817F00F025
:101B40009B80B3F5407FA4D194F88230012BA0D1C3
:101B5000B4F8883043F0020332E0B3F5006F4DD0A3
:101B600017D8B3F5A06F31D0A3F5C063012B90D87F
:101B70006368204694F882205E6894F88310B4F875
:101B80008430B047002884D0436863670368A36744
:101B90001AE0B3F5106F36D040F6024293427FF45C
:101BA00078AF5C4B63670223A3670023C3E794F815
:101BB0008230012B7FF46DAFB4F8883023F002033C
:101BC000A4F88830C4E91D55E56778E7B4F880309B
:101BD000B3F5A06F0ED194F88230204684F88A3095
:101BE00001F0D2F963681B6813B1012120469847C0
:101BF000032323700023C4E91D339CE704F18B0306
:101C000063670123C3E72378042B10D1302383F3C8
:101C100011882046FFF7BAFE85F311880321636817
:101C200084F88B5021701B680BB12046984794F8BC
:101C30008230002BDED084F88B300423237063685D
:101C40001B68002BD6D0022120469847D2E794F893
:101C5000843020461D0603F00F010AD501F044FA36
:101C6000012804D002287FF414AF2B4B9AE72B4BAA
:101C700098E701F02BFAF3E794F88230002B7FF419
:101C800008AF94F8843013F00F01B3D01A06204641
:101C900002D501F04DFDADE701F03EFDAAE794F855
:101CA0008230002B7FF4F5AE94F8843013F00F01EE
:101CB000A0D01B06204602D501F022FD9AE701F0D4
:101CC00013FD97E7142284F8702083F311882B46C4
:101CD0002A4629462046FFF769FE85F31188E9E682
:101CE0005DB1152284F8702083F31188002120460D
:101CF000D4E91D23FFF75AFEFDE60B2284F870207D
:101D000083F311882B462A4629462046FFF760FEBA
:101D1000E3E700BFD4440008CC440008D0440008E6
:101D200038B590F870300446002B3ED0063BDAB24E
:101D30000F2A34D80F2B32D8DFE803F037313108BF
:101D4000223231313131313131313737856FB0F8AD
:101D500086309D4214D2C3681B8AB5FBF3F203FBA5
:101D600012556DB9302383F311882B462A46294634
:101D7000FFF72EFE85F311880A2384F870300EE0F9
:101D8000142384F87030302383F311880023204615
:101D90001A461946FFF70AFE002383F3118838BD5F
:101DA000C36F03B198470023E7E70021204601F005
:101DB000A7FC0021204601F097FC63681B6813B163
:101DC0000621204698470623D7E7000010B590F873
:101DD00070300446142B29D017D8062B05D001D813
:101DE0001BB110BD093B022BFBD80021204601F09E
:101DF00087FC0021204601F077FC63681B6813B163
:101E0000062120469847062319E0152BE9D10B231C
:101E100080F87030302383F3118800231A46194666
:101E2000FFF7D6FD002383F31188DAE7C3689B69C7
:101E30005B68002BD5D1C36F03B19847002384F8AA
:101E40007030CEE700238268037503691B689968C8
:101E50009142FBD25A68036042601060586070473C
:101E600000238268037503691B6899689142FBD857
:101E70005A680360426010605860704708B50846B1
:101E8000302383F311880A7D0023052A06D8DFE872
:101E900002F00B050503120E826913604FF0FF3349
:101EA0008361FFF7CFFF002383F3118808BD8269A8
:101EB000936801339360D0E9003213605A60EDE714
:101EC000FFF7C0BF054BD9680875186802685360F2
:101ED0001A600122D8600275FEF794BA40240020EF
:101EE0000C4B30B5DD684B1C87B004460FD02B4639
:101EF000094A684600F06EF92046FFF7E3FF009BB1
:101F000013B1684600F070F9A86907B030BDFFF75B
:101F1000D9FFF9E7402400207D1E000838B50C4D9C
:101F200004468161EB6881689A68914203D8BDE8F4
:101F30003840FFF787BF1846FFF792FF012301469D
:101F4000EC6020462375BDE83840FEF75BBA00BF61
:101F500040240020044B1A68DB6890689B68984214
:101F600094BF00200120704740240020084B10B58A
:101F70001C68D868226853601A600122DC602275F0
:101F8000FFF76EFF01462046BDE81040FEF73ABA63
:101F90004024002038B50123084C002523706560DB
:101FA00001F0BAFD01F0E0FD0549064801F0B4FE7C
:101FB0000223237085F3118838BD00BFA8260020B6
:101FC000DC4400084024002000F044B9034A516872
:101FD00053685B1A9842FBD8704700BF001000E0BE
:101FE0008B600223086108468B8270478368A3F1E7
:101FF000840243F8142C026943F8442C426943F8E4
:10200000402C094A43F8242CC268A3F1200043F86D
:10201000182C022203F80C2C002203F80B2C034A84
:1020200043F8102C704700BF1D0400084024002016
:1020300008B5FFF7DBFFBDE80840FFF741BF000030
:10204000024BDB6898610F20FFF73CBF4024002063
:10205000302383F31188FFF7F3BF000008B5014672
:10206000302383F311880820FFF73AFF002383F31E
:10207000118808BD064BDB6839B1426818605A60A8
:10208000136043600420FFF72BBF4FF0FF30704711
:10209000402400200368984206D01A68026050600D
:1020A00018469961FFF70CBF7047000038B5044629
:1020B0000D462068844200D138BD036823605C600F
:1020C0008561FFF7FDFEF4E7036810B59C68A24246
:1020D0000CD85C688A600B604C602160596099681C
:1020E0008A1A9A604FF0FF33836010BD121B1B6881
:1020F000ECE700000A2938BF0A2170B504460D46F6
:102100000A26601901F002FD01F0EAFC041BA54259
:1021100003D8751C04462E46F3E70A2E04D9012085
:10212000BDE8704001F038BE70BD0000F8B5144B3A
:102130000D460A2A4FF00A07D96103F110018260A7
:1021400038BF0A224160196914460160486018616D
:10215000A81801F0CBFC01F0C3FC431B0646A342C8
:1021600006D37C1C28192746354601F0CFFCF2E740
:102170000A2F04D90120BDE8F84001F00DBEF8BDDA
:1021800040240020F8B506460D4601F0A9FC0F4A90
:10219000134653F8107F9F4206D12A460146304627
:1021A000BDE8F840FFF7C2BFD169BB68441A2C19DB
:1021B00028BF2C46A34202D92946FFF79BFF22469F
:1021C00031460348BDE8F840FFF77EBF40240020B9
:1021D00050240020C0E90323002310B45DF8044B11
:1021E0004361FFF7CFBF000010B5194C2369984237
:1021F0000DD08168D0E9003213605A609A680A44B1
:102200009A60002303604FF0FF33A36110BD0268A2
:10221000234643F8102F53600022026022699A423D
:1022200003D1BDE8104001F06BBC936881680B449A
:10223000936001F055FC2269E1699268441AA24258
:10224000E4D91144BDE81040091AFFF753BF00BF9D
:10225000402400202DE9F047DFF8BC8008F110078A
:102260002C4ED8F8105001F03BFCD8F81C40AA685E
:10227000031B9A423ED814444FF00009D5E90032BE
:10228000C8F81C4013605A60C5F80090D8F81030A8
:10229000B34201D101F034FC89F31188D5E903314F
:1022A00028469847302383F311886B69002BD8D0D8
:1022B00001F016FC6A69A0EB040982464A450DD27A
:1022C000022001F069FD0022D8F81030B34208D195
:1022D00051462846BDE8F047FFF728BF121A2244AE
:1022E000F2E712EB09092946384638BF4A46FFF79C
:1022F000EBFEB5E7D8F81030B34208D01444C8F864
:102300001C00211AA960BDE8F047FFF7F3BEBDE845
:10231000F08700BF50240020402400200020704798
:10232000FEE70000704700004FF0FF3070470000EC
:1023300002290CD0032904D00129074818BF002026
:102340007047032A05D8054800EBC20070470448CF
:1023500070470020704700BFB44500083C220020B1
:102360006845000870B59AB005460846144601A9AC
:1023700000F0C2F801A8FEF78DFD431C0022C6B292
:102380005B001046C5E9003423700323023404F8CF
:10239000013C01ABD1B202348E4201D81AB070BDFB
:1023A00013F8011B013204F8010C04F8021CF1E7D8
:1023B00008B5302383F311880348FFF725FA00237B
:1023C00083F3118808BD00BFB026002090F880304C
:1023D00003F01F02012A07D190F881200B2A03D1B4
:1023E0000023C0E91D3315E003F06003202B08D162
:1023F000B0F884302BB990F88120212A03D81F2A05
:1024000004D8FFF7E3B9222AEBD0FAE7034A426780
:1024100007228267C3670120704700BF3322002074
:1024200007B5052917D8DFE801F019160319192097
:10243000302383F31188104A01210190FFF78CFAB1
:10244000019802210D4AFFF787FA0D48FFF7A8F916
:10245000002383F3118803B05DF804FB302383F37A
:1024600011880748FFF772F9F2E7302383F31188E8
:102470000348FFF789F9EBE7084500082C450008F9
:10248000B026002038B50C4D0C4C2A460C4904F1FE
:102490000800FFF767FF05F1CA0204F110000949BF
:1024A000FFF760FF05F5CA7204F118000649BDE8A0
:1024B0003840FFF757BF00BF883F00203C22002074
:1024C000E8440008F2440008FD44000870B50446E2
:1024D00008460D46FEF7DEFCC6B2204601340378FE
:1024E0000BB9184670BD32462946FEF7BFFC0028DE
:1024F000F3D10120F6E700002DE9F84F05460C4620
:10250000FEF7C8FC2C49C6B22846FFF7DFFF08B12A
:102510000536F6B229492846FFF7D8FF08B110362C
:10252000F6B2632E0DD8DFF89080DFF89090244F3C
:10253000DFF894A0DFF894B02E7846B92670BDE895
:10254000F88F29462046BDE8F84F01F0F5BE252E4C
:102550002ED1072241462846FEF788FC70B9DBF8E9
:10256000003007350C3444F80C3CDBF8043044F8F8
:10257000083CDBF8083044F8043CDDE70822494613
:102580002846FEF773FC98B9A21C0E4B197802324C
:102590000909C95D02F8041C13F8011B01F00F01C1
:1025A0005345C95D02F8031CF0D118340835C3E760
:1025B000013504F8016BBFE7D4450008FD4400086D
:1025C000E945000800E8F11F0CE8F11FDC450008B0
:1025D000BFF34F8F044B1A695107FCD1D3F8102178
:1025E0005207F8D1704700BF0020005208B50D4BCC
:1025F0001B78ABB9FFF7ECFF0B4BDA68D10704D5BA
:102600000A4A5A6002F188325A60D3F80C21D20784
:1026100006D5064AC3F8042102F18832C3F8042122
:1026200008BD00BFE641002000200052230167459D
:1026300008B5114B1B78F3B9104B1A69510703D534
:10264000DA6842F04002DA60D3F81021520705D56B
:10265000D3F80C2142F04002C3F80C21FFF7B8FF79
:10266000064BDA6842F00102DA60D3F80C2142F03E
:102670000102C3F80C2108BDE641002000200052F1
:102680000F289ABF00F580604004002070470000CA
:102690004FF4003070470000102070470F2808B535
:1026A0000BD8FFF7EDFF00F500330268013204D1CB
:1026B00004308342F9D1012008BD0020FCE700006E
:1026C0000F2838B505463FD8FFF782FF1F4CFFF7AC
:1026D0008DFF4FF0FF3307286361C4F814311DD814
:1026E0002361FFF775FF030243F02403E360E3680F
:1026F00043F08003E36023695A07FCD42846FFF7C0
:1027000067FFFFF7BDFF4FF4003100F0C5F9284621
:10271000FFF78EFFBDE83840FFF7C0BFC4F81031A7
:10272000FFF756FFA0F108031B0243F02403C4F88F
:102730000C31D4F80C3143F08003C4F80C31D4F8D8
:1027400010315B07FBD4D9E7002038BD00200052D0
:102750002DE9F84F04460D46104644EA0203DE0612
:1027600002D00020BDE8F88F20F01F00DFF8D4B0C1
:10277000DFF8D4A0FFF73AFF05EB0008454503D189
:102780000120FFF755FFEDE720222946204601F002
:10279000C3FD10B920342035F0E7234604F12002B0
:1027A0001F68791CDDD104339342F9D104F17843D9
:1027B0002048214EB3F5801F204B38BF184603F147
:1027C000F80332BFD946D1461E46FFF701FF076026
:1027D000A4EB050C336805F11C0143F002033360E0
:1027E0002B1FD9F8007017F00507FAD153F8042F02
:1027F0008B424CF80320F4D1BFF34F8FFFF7E8FE74
:102800004FF0FF330360336823F002033360BFF3FC
:102810004F8F0B4BC3F85C42BFF34F8FBFF36F8FEB
:1028200020222946204601F077FD0028B2D0384604
:10283000A7E700BF142100520C20005214200052C0
:1028400000ED00E0102000521021005210B5084C9D
:10285000237828B11BB9FFF7C9FE0123237010BDEF
:10286000002BFCD02070BDE81040FFF7E1BE00BF98
:10287000E64100202DE9F04F0D4685B0814658B164
:1028800011F00D0614BF2022082211F00803019355
:1028900004D0431E03426AD0002435E0002E37D016
:1028A00009F11F0121F01F094FF00108324F05F017
:1028B0000403DFF8D0A005EA080BBBF1000F32D00B
:1028C0007869C0072FD408F101080C37B8F1060F5A
:1028D000F3D19EB9294D4946A819019201F066F934
:1028E000044600283AD11836019A782EF3D1494689
:1028F00001F05CF90446002830D1019A494620488D
:1029000001F054F9044668BB204605B0BDE8F08FDD
:102910000029C9D101462846029201F047F9044630
:10292000E0B9029AC0E713B178694107CBD5AC078B
:1029300002D578698007C6D5019911B17869010778
:10294000C1D51820494600FB08A0CDE9022301F0BB
:102950002DF90446DDE902230028B4D04A460021BF
:10296000204601E04A460021FEF79CFACCE70246E9
:10297000002E95D198E700BFFC45000818420020C2
:10298000E8410020004200200121FFF773BF000052
:10299000F8B500231A461A600433B3F5806FFAD1F4
:1029A000114D01241827114E07FB046001342A69D8
:1029B00055F80C1F01F0E6F8062CF5D137254FF439
:1029C000C0542046FFF7E0FF014628B122460848E0
:1029D000BDE8F84001F0D6B8C4EBC404013D4FEAAD
:1029E000D404EED1F8BD00BFFC4500080042002031
:1029F000E841002008B101F04BB970470244074B91
:102A0000D2B210B5904200D110BD441C00B253F8B0
:102A1000200041F8040BE0B2F4E700BF504000583A
:102A20000E4B30B51C6F240405D41C6F1C671C6F43
:102A300044F400441C670A4C02442368D2B243F4B5
:102A400080732360074B904200D130BD441C51F885
:102A5000045B00B243F82050E0B2F4E700440258AF
:102A6000004802585040005807B5012201A9002033
:102A7000FFF7C4FF019803B05DF804FB13B50446EB
:102A8000FFF7F2FFA04205D0012201A90020019426
:102A9000FFF7C6FF02B010BD0144BFF34F8F064BD6
:102AA000884204D3BFF34F8FBFF36F8F7047C3F8D3
:102AB0005C022030F4E700BF00ED00E0034B1A6831
:102AC0001AB9034AD2F8D0241A6070479042002005
:102AD0000040025808B5FFF7F1FF024B1868C0F339
:102AE000806008BD90420020EFF3098305496833F8
:102AF0004A6B22F001024A6383F30988002383F3BF
:102B00001188704700EF00E0302080F3118862B632
:102B10000D4B0E4AD96821F4E0610904090C0A43FF
:102B20000B49DA60D3F8FC2042F08072C3F8FC2035
:102B3000084AC2F8B01F116841F00101116020225B
:102B4000DA7783F82200704700ED00E00003FA0511
:102B500055CEACC5001000E0302310B583F31188CA
:102B60000E4B5B6813F4006314D0F1EE103AEFF3F0
:102B700009844FF08073683CE361094BDB6B23668B
:102B800084F30988FFF7E6F910B1064BA36110BD85
:102B9000054BFBE783F31188F9E700BF00ED00E088
:102BA00000EF00E02F0400083204000870B5BFF306
:102BB0004F8FBFF36F8F1A4A0021C2F85012BFF334
:102BC0004F8FBFF36F8F536943F400335361BFF3EB
:102BD0004F8FBFF36F8FC2F88410BFF34F8FD2F8BF
:102BE000803043F6E074C3F3C900C3F34E335B0196
:102BF00003EA0406014646EA81750139C2F86052CB
:102C0000F9D2203B13F1200FF2D1BFF34F8F53695C
:102C100043F480335361BFF34F8FBFF36F8F70BDA9
:102C200000ED00E0FEE70000214B2248224A70B58B
:102C3000904237D3214BC11EDA1C121A22F0030234
:102C40008B4238BF00220021FEF72CF91C4A0023DA
:102C5000C2F88430BFF34F8FD2F8803043F6E0746F
:102C6000C3F3C900C3F34E335B0103EA0406014614
:102C700046EA81750139C2F86C52F9D2203B13F152
:102C8000200FF2D1BFF34F8FBFF36F8FBFF34F8F82
:102C9000BFF36F8F0023C2F85032BFF34F8FBFF3E3
:102CA0006F8F70BD53F8041B40F8041BC0E700BFD2
:102CB0001C48000804440020044400200444002070
:102CC00000ED00E0074BD3F8D81021EA0001C3F86B
:102CD000D810D3F8002122EA0002C3F80021D3F86B
:102CE000003170470044025870B5D0E924430022F7
:102CF0004FF0FF359E6804EB42135101D3F80009F1
:102D0000002805DAD3F8000940F08040C3F8000934
:102D1000D3F8000B002805DAD3F8000B40F0804010
:102D2000C3F8000B013263189642C3F80859C3F880
:102D3000085BE0D24FF00113C4F81C3870BD0000EE
:102D4000890141F02001016103699B06FCD4122036
:102D5000FFF73CB910B50A4C2046FEF7DBFD094BE6
:102D6000C4F89030084BC4F89430084C2046FEF765
:102D7000D1FD074BC4F89030064BC4F8943010BD19
:102D800094420020000008406846000830430020BC
:102D9000000004407446000870B503780546012B16
:102DA0005CD1434BD0F89040984258D1414B0E2112
:102DB0006520D3F8D82042F00062C3F8D820D3F8B9
:102DC000002142F00062C3F80021D3F80021D3F8BB
:102DD000802042F00062C3F88020D3F8802022F0E7
:102DE0000062C3F88020D3F88030FEF7BFFB324B7F
:102DF000E360324BC4F800380023D5F89060C4F883
:102E0000003EC02323604FF40413A3633369002BF7
:102E1000FCDA01230C203361FFF7D8F83369DB07B4
:102E2000FCD41220FFF7D2F83369002BFCDA00261D
:102E30002846A660FFF758FF6B68C4F81068DB6887
:102E4000C4F81468C4F81C6883BB1D4BA3614FF021
:102E5000FF336361A36843F00103A36070BD194BA6
:102E60009842C9D1134B4FF08060D3F8D82042F07C
:102E70000072C3F8D820D3F8002142F00072C3F8E2
:102E80000021D3F80021D3F8802042F00072C3F86B
:102E90008020D3F8802022F00072C3F88020D3F87D
:102EA0008030FFF70FFF0E214D209EE7064BCDE748
:102EB00094420020004402584014004003002002C5
:102EC000003C30C030430020083C30C0F8B5D0F89A
:102ED0009040054600214FF000662046FFF730FF86
:102EE000D5F8941000234FF001128F684FF0FF3097
:102EF000C4F83438C4F81C2804EB431201339F4251
:102F0000C2F80069C2F8006BC2F80809C2F8080BE1
:102F1000F2D20B68D5F89020C5F898306362102380
:102F20001361166916F01006FBD11220FFF74EF858
:102F3000D4F8003823F4FE63C4F80038A36943F4DE
:102F4000402343F01003A3610923C4F81038C4F8E8
:102F500014380B4BEB604FF0C043C4F8103B094BE7
:102F6000C4F8003BC4F81069C4F80039D5F89830AB
:102F700003F1100243F48013C5F89820A362F8BD52
:102F80004446000840800010D0F8902090F88A1045
:102F9000D2F8003823F4FE6343EA0113C2F8003884
:102FA000704700002DE9F84300EB8103D0F8905002
:102FB0000C468046DA680FFA81F94801166806F077
:102FC0000306731E022B05EB41134FF0000194BF63
:102FD000B604384EC3F8101B4FF0010104F1100382
:102FE00098BF06F1805601FA03F3916998BF06F580
:102FF000004600293AD0578A04F158013743490165
:103000006F50D5F81C180B430021C5F81C382B183D
:103010000127C3F81019A7405369611E9BB3138A97
:10302000928B9B08012A88BF5343D8F898209818A0
:1030300042EA034301F140022146C8F898002846BD
:1030400005EB82025360FFF77BFE08EB8900C36843
:103050001B8A43EA845348341E4364012E51D5F839
:103060001C381F43C5F81C78BDE8F88305EB4917E9
:10307000D7F8001B21F40041C7F8001BD5F81C1835
:1030800021EA0303C0E704F13F030B4A2846214627
:1030900005EB83035A60FFF753FE05EB4910D0F8A8
:1030A000003923F40043C0F80039D5F81C3823EA6E
:1030B0000707D7E70080001000040002D0F8942032
:1030C0001268C0F89820FFF70FBE00005831D0F802
:1030D000903049015B5813F4004004D013F4001FF2
:1030E0000CBF0220012070474831D0F890304901D0
:1030F0005B5813F4004004D013F4001F0CBF0220EF
:103100000120704700EB8101CB68196A0B681360DE
:103110004B6853607047000000EB810330B5DD68F9
:10312000AA691368D36019B9402B84BF4023136088
:103130006B8A1468D0F890201C4402EB4110013CCB
:1031400009B2B4FBF3F46343033323F0030343EA0C
:10315000C44343F0C043C0F8103B2B6803F00303A3
:10316000012B0ED1D2F8083802EB411013F4807F06
:10317000D0F8003B14BF43F0805343F00053C0F835
:10318000003B02EB4112D2F8003B43F00443C2F88B
:10319000003B30BD2DE9F041D0F8906005460C466B
:1031A00006EB4113D3F8087B3A07C3F8087B08D530
:1031B000D6F814381B0704D500EB8103DB685B6885
:1031C0009847FA071FD5D6F81438DB071BD505EB4F
:1031D0008403D968CCB98B69488A5A68B2FBF0F687
:1031E00000FB16228AB91868DA6890420DD2121ACA
:1031F000C3E90024302383F3118821462846FFF7D2
:103200008BFF84F31188BDE8F081012303FA04F2F7
:103210006B8923EA02036B81CB68002BF3D0214634
:103220002846BDE8F041184700EB81034A0170B51C
:10323000DD68D0F890306C692668E66056BB1A44A9
:103240004FF40020C2F810092A6802F00302012A94
:103250000AB20ED1D3F8080803EB421410F4807FB1
:10326000D4F8000914BF40F0805040F00050C4F87A
:10327000000903EB4212D2F8000940F00440C2F802
:1032800000090122D3F8340802FA01F10143C3F81E
:10329000341870BD19B9402E84BF402020602068CA
:1032A0001A442E8A8419013CB4FBF6F440EAC44067
:1032B00040F00050C6E700002DE9F843D0F89060D8
:1032C00005460C464F0106EB4113D3F8088918F068
:1032D000010FC3F808891CD0D6F81038DB0718D5C1
:1032E00000EB8103D3F80CC0DCF81430D3F800E015
:1032F000DA68964530D2A2EB0E024FF000091A6050
:10330000C3F80490302383F31188FFF78DFF89F30E
:10331000118818F0800F1DD0D6F834380126A64049
:10332000334217D005EB84030134D5F89050D3F81D
:103330000CC0E4B22F44DCF8142005EB0434D2F8BE
:1033400000E05168714514D3D5F8343823EA0606F5
:10335000C5F83468BDE8F883012303FA01F2038954
:1033600023EA02030381DCF80830002BD1D0984710
:10337000CFE7AEEB0103BCF81000834228BF034641
:10338000D7F8180980B2B3EB800FE3D89068A0F1AA
:10339000040959F8048FC4F80080A0EB0908984488
:1033A000B8F1040FF5D818440B4490605360C8E797
:1033B0002DE9F84FD0F8905004466E69AB691E4075
:1033C00016F480586E6103D0BDE8F84FFEF712BBCB
:1033D000002E12DAD5F8003E9B0705D0D5F8003E46
:1033E00023F00303C5F8003ED5F80438204623F047
:1033F0000103C5F80438FEF72BFB370505D5204639
:10340000FFF772FC2046FEF711FBB0040CD5D5F88F
:10341000083813F0060FEB6823F470530CBF43F425
:10342000105343F4A053EB6031071BD56368DB688E
:103430001BB9AB6923F00803AB612378052B0CD1D2
:10344000D5F8003E9A0705D0D5F8003E23F00303D7
:10345000C5F8003E2046FEF7FBFA6368DB680BB157
:1034600020469847F30200F1BA80B70226D5D4F877
:10347000909000274FF0010A09EB4712D2F8003B69
:1034800003F44023B3F5802F11D1D2F8003B002B79
:103490000DDA62890AFA07F322EA0303638104EB77
:1034A0008703DB68DB6813B139462046984701374C
:1034B000D4F89430FFB29B689F42DDD9F00619D54D
:1034C000D4F89000026AC2F30A1702F00F0302F464
:1034D000F012B2F5802F00F0CA80B2F5402F09D16A
:1034E00004EB8303002200F58050DB681B6A9742DF
:1034F00040F0B0803003D5F8185835D5E90303D52E
:1035000000212046FFF746FEAA0303D501212046ED
:10351000FFF740FE6B0303D502212046FFF73AFE7A
:103520002F0303D503212046FFF734FEE80203D51D
:1035300004212046FFF72EFEA90203D505212046CF
:10354000FFF728FE6A0203D506212046FFF722FE78
:103550002B0203D507212046FFF71CFEEF0103D500
:1035600008212046FFF716FE700340F1A780E90707
:1035700003D500212046FFF79FFEAA0703D50121AE
:103580002046FFF799FE6B0703D502212046FFF77F
:1035900093FE2F0703D503212046FFF78DFEEE068D
:1035A00003D504212046FFF787FEA80603D5052191
:1035B0002046FFF781FE690603D506212046FFF766
:1035C0007BFE2A0603D507212046FFF775FEEB0593
:1035D00074D520460821BDE8F84FFFF76DBED4F83A
:1035E00090904FF0000B4FF0010AD4F894305FFA3E
:1035F0008BF79B689F423FF638AF09EB4713D3F830
:10360000002902F44022B2F5802F20D1D3F80029FE
:10361000002A1CDAD3F8002942F09042C3F80029AE
:10362000D3F80029002AFBDB3946D4F89000FFF7D5
:1036300087FB22890AFA07F322EA0303238104EBBA
:103640008703DB689B6813B13946204698470BF126
:10365000010BCAE7910701D1D0F80080072A02F1D7
:1036600001029CBF03F8018B4FEA18283FE704EBE7
:10367000830300F58050DA68D2F818C0DCF808201F
:10368000DCE9001CA1EB0C0C00218F4208D1DB68A7
:103690009B699A683A449A605A683A445A6029E7A2
:1036A00011F0030F01D1D0F800808C4501F1010128
:1036B00084BF02F8018B4FEA1828E6E7BDE8F88FCF
:1036C00008B50348FFF774FEBDE80840FFF744BAA9
:1036D0009442002008B50348FFF76AFEBDE80840A1
:1036E000FFF73ABA30430020D0F8903003EB411195
:1036F000D1F8003B43F40013C1F8003B70470000D1
:10370000D0F8903003EB4111D1F8003943F40013A5
:10371000C1F8003970470000D0F8903003EB411138
:10372000D1F8003B23F40013C1F8003B70470000C0
:10373000D0F8903003EB4111D1F8003923F4001395
:10374000C1F800397047000030B50433039C0172A2
:10375000002104FB0325C160C0E90653049B0363F9
:10376000059BC0E90000C0E90422C0E90842C0E9A5
:103770000A11436330BD00000022416AC260C0E903
:103780000411C0E90A226FF00101FEF78FBC0000AE
:10379000D0E90432934201D1C2680AB9181D7047BA
:1037A00000207047036919600021C2680132C260BD
:1037B000C269134482699342036124BF436A03616F
:1037C000FEF768BC38B504460D46E3683BB1626954
:1037D0000020131D1268A3621344E36207E0237AFA
:1037E00033B929462046FEF745FC0028EDDA38BDFE
:1037F0006FF00100FBE70000C368C269013BC360D2
:103800004369134482699342436124BF436A43611D
:1038100000238362036B03B11847704770B53023F0
:10382000044683F31188866A3EB9FFF7CBFF05464D
:1038300018B186F31188284670BDA36AE26A13F8AE
:10384000015B9342A36202D32046FFF7D5FF00231A
:1038500083F31188EFE700002DE9F84F04460E4688
:10386000174698464FF0300989F311880025AA467B
:10387000D4F828B0BBF1000F09D141462046FFF72C
:10388000A1FF20B18BF311882846BDE8F88FD4E959
:103890000A12A7EB050B521A934528BF9346BBF1BA
:1038A000400F1BD9334601F1400251F8040B9142FD
:1038B00043F8040BF9D1A36A403640354033A36284
:1038C000D4E90A239A4202D32046FFF795FF8AF3F0
:1038D0001188BD42D8D289F31188C9E730465A46CB
:1038E000FDF7BAFAA36A5E445D445B44A362E7E76E
:1038F00010B5029C0433017203FB0421C460C0E9CB
:1039000006130023C0E90A33039B0363049BC0E949
:103910000000C0E90422C0E90842436310BD000072
:10392000026A6FF00101C260426AC0E9042200220B
:10393000C0E90A22FEF7BABBD0E904239A4201D1BA
:10394000C26822B9184650F8043B0B607047002348
:103950001846FAE7C3680021C2690133C3604369AE
:10396000134482699342436124BF436A4361FEF773
:1039700091BB000038B504460D46E3683BB12369AE
:1039800000201A1DA262E2691344E36207E0237A71
:1039900033B929462046FEF76DFB0028EDDA38BD25
:1039A0006FF00100FBE7000003691960C268013A8B
:1039B000C260C269134482699342036124BF436AAF
:1039C000036100238362036B03B118477047000053
:1039D00070B530230D460446114683F31188866A7C
:1039E0002EB9FFF7C7FF10B186F3118870BDA36A27
:1039F0001D70A36AE26A01339342A36204D3E169B2
:103A000020460439FFF7D0FF002080F31188EDE74E
:103A10002DE9F84F04460D46904699464FF0300A7E
:103A20008AF311880026B346A76A4FB94946204653
:103A3000FFF7A0FF20B187F311883046BDE8F88F6B
:103A4000D4E90A073A1AA8EB0607974228BF174697
:103A5000402F1BD905F1400355F8042B9D4240F837
:103A6000042BF9D1A36A40364033A362D4E90A2378
:103A70009A4204D3E16920460439FFF795FF8BF39E
:103A800011884645D9D28AF31188CDE729463A46AE
:103A9000FDF7E2F9A36A3D443E443B44A362E5E7F7
:103AA000D0E904239A4217D1C3689BB1836A8BB1D2
:103AB000043B9B1A0ED01360C368013BC360C3690B
:103AC0001A4483699A42026124BF436A0361002356
:103AD00083620123184670470023FBE700F060BAB9
:103AE000014B586A704700BF000C0040034B002296
:103AF00058631A610222DA60704700BF000C004070
:103B0000014B0022DA607047000C0040014B586303
:103B1000704700BF000C0040024B034A1A60034A82
:103B20005A607047E443002008440020000002204F
:103B3000074B494210B55C68201A08401968821A80
:103B40008A4203D3A24201D85A6010BD0020FCE78C
:103B5000E443002008B5302383F31188FFF7E8FF22
:103B6000002383F3118808BD04480121044B03603E
:103B70000023C0E901330C3000F016B9EC430020FB
:103B8000553B0008CB1D083A23F00703591A521A77
:103B9000012110B4D2080024C0E9004384600C3035
:103BA0001C605A605DF8044B00F0FEB82DE9F84F38
:103BB000364ECD1D0F46002818BF0646082A4FEA8C
:103BC000D50538BF082206F10C08341D9146404641
:103BD00000F006F909F10701C9F1000E2246246838
:103BE0006CB9404600F006F93368CBB30822494669
:103BF000E8009847044698B340E9026730E004EBD8
:103C0000010CD4F804A00CEA0E0C0AF10100ACF18E
:103C1000080304EBC0009842E0D9A0EB0C0CB5EB14
:103C2000EC0F4FEAEC0BD9D89C421CD204F10802ED
:103C3000AB45A3EB02024FEAE202626009D9691CBC
:103C4000ED43206803EBC1025D44556043F8310049
:103C500022601C465F60404644F8086B00F0CAF8DA
:103C60002046BDE8F88FAA45216802D1116023469D
:103C7000EFE7013504EBC50344F8351003F1080103
:103C8000401AC01058601360F1E700BFEC430020F9
:103C9000F8B550F8043C044650F8085CA0F108065A
:103CA00007332F1D0C35DB0840F8043C284600F094
:103CB00097F83B469F421A6801D0B34228D20AB116
:103CC000964225D244F8082C54F8042C1E60013288
:103CD00054F8081C06EBC200814206D14868024431
:103CE00044F8042C0A6844F8082C5868411C03EB7B
:103CF000C1018E4207D154F8042C013202445A60AB
:103D000054F8082C1A602846BDE8F84000F072B854
:103D10001346CFE7FEE7000070B51B4B00250446B5
:103D200086B058600E4685620163FEF7EDFE04F131
:103D30001003A560E562C4E904334FF0FF33C4E922
:103D40000044C4E90635FFF7CBFE2B46024604F1DA
:103D500034012046C4E9082380230C4A2565FEF778
:103D60003FF901230A4AE0600092037568467268D1
:103D70000192B268CDE90223064BCDE90435FEF786
:103D800057F906B070BD00BFA82600208046000885
:103D900085460008153D0008024AD36A1843D062E0
:103DA000704700BF40240020C0E9000081607047D8
:103DB0008368013B002B10B583600CDA074BDC688D
:103DC0004368A061206063601C6044600520FEF7CA
:103DD00079F8A06910BD0020FCE700BF4024002056
:103DE00008B5302383F31188FFF7E2FF002383F344
:103DF000118808BD08B5302383F311888368013327
:103E0000002B836007DC036800211A6802605060A1
:103E10001846FEF783F8002383F3118808BD0000DD
:103E20004B6843608B688360CB68C3600B694361F8
:103E30004B6903628B6943620B6803607047000043
:103E400008B53C4B40F2FF713B48D3F888200A4349
:103E5000C3F88820D3F8882022F4FF6222F00702FA
:103E6000C3F88820D3F88820D3F8E0200A43C3F8A9
:103E7000E020D3F808210A43C3F808212F4AD3F8D9
:103E800008311146FFF7CCFF00F5806002F11C01FC
:103E9000FFF7C6FF00F5806002F13801FFF7C0FFB1
:103EA00000F5806002F15401FFF7BAFF00F5806071
:103EB00002F17001FFF7B4FF00F5806002F18C01A0
:103EC000FFF7AEFF00F5806002F1A801FFF7A8FF41
:103ED00000F5806002F1C401FFF7A2FF00F58060E9
:103EE00002F1E001FFF79CFF00F5806002F1FC01A8
:103EF000FFF796FF02F58C7100F58060FFF790FFE9
:103F000000F01AF90E4BD3F8902242F00102C3F8E8
:103F10009022D3F8942242F00102C3F894220522A1
:103F2000C3F898204FF06052C3F89C20054AC3F8AC
:103F3000A02008BD00440258000002588C4600082A
:103F400000ED00E01F00080308B500F0D3F9FEF70C
:103F500021F8104BD3F8DC2042F04002C3F8DC20FB
:103F6000D3F8042122F04002C3F80421D3F804312D
:103F7000094B1A6842F008021A601A6842F00402FB
:103F80001A60FEF79BFDFEF703FDBDE80840FEF753
:103F900079BA00BF00440258001802487047000078
:103FA000114BD3F8E82042F00802C3F8E820D3F818
:103FB000102142F00802C3F810210C4AD3F8103146
:103FC000D36B43F00803D363C722094B9A624FF0C7
:103FD000FF32DA6200229A615A63DA605A60012283
:103FE0005A611A60704700BF004402580010005C1C
:103FF000000C0040094A08B51169D3680B40D9B2DA
:104000009B076FEA0101116107D5302383F3118803
:10401000FDF7DAFF002383F3118808BD000C004090
:10402000064BD3F8DC200243C3F8DC20D3F804218C
:104030001043C3F80401D3F8043170470044025818
:1040400008B53C4B4FF0FF31D3F8802062F00042BE
:10405000C3F88020D3F8802002F00042C3F880200B
:10406000D3F88020D3F88420C3F88410D3F88420B8
:104070000022C3F88420D3F88400D86F40F0FF40BA
:1040800040F4FF0040F4DF4040F07F00D867D86F75
:1040900020F0FF4020F4FF0020F4DF4020F07F00FC
:1040A000D867D86FD3F888006FEA40506FEA505055
:1040B000C3F88800D3F88800C0F30A00C3F888006A
:1040C000D3F88800D3F89000C3F89010D3F890008C
:1040D000C3F89020D3F89000D3F89400C3F894105C
:1040E000D3F89400C3F89420D3F89400D3F8980040
:1040F000C3F89810D3F89800C3F89820D3F8980024
:10410000D3F88C00C3F88C10D3F88C00C3F88C2043
:10411000D3F88C00D3F89C00C3F89C10D3F89C1003
:10412000C3F89C20D3F89C30FDF744F9BDE8084063
:1041300000F0D4B80044025808B50122534BC3F82C
:104140000821534BD3F8F42042F00202C3F8F420C4
:10415000D3F81C2142F00202C3F81C210222D3F83A
:104160001C314C4BDA605A689104FCD54A4A1A60FB
:1041700001229A60494ADA6000221A614FF44042F3
:104180009A61444B9A699204FCD51A6842F4807291
:104190001A603F4B1A6F12F4407F04D04FF4803204
:1041A0001A6700221A671A6842F001021A60384B37
:1041B0001A685007FCD500221A611A6912F03802F9
:1041C000FBD1012119604FF0804159605A67344A90
:1041D000DA62344A1A611A6842F480321A602C4B4F
:1041E0001A689103FCD51A6842F480521A601A6862
:1041F0009204FCD52C4A2D499A6200225A63196315
:1042000001F57C01DA6301F2E71199635A64284AE7
:104210001A64284ADA621A6842F0A8521A601C4BE3
:104220001A6802F02852B2F1285FF9D148229A6147
:104230004FF48862DA6140221A621F4ADA641F4A28
:104240001A651F4A5A651F4A9A6532231E4A13602F
:10425000136803F00F03022BFAD10D4A136943F0E0
:1042600003031361136903F03803182BFAD14FF0DD
:104270000050FFF7D5FE4FF08040FFF7D1FE4FF022
:104280000040BDE80840FFF7CBBE00BF00800051F2
:10429000004402580048025800C000F0020000012B
:1042A0000000FF010088900812102000630209013D
:1042B000470E0508DD0BBF012000002000000110A3
:1042C0000910E000000101100020005208B5FFF7BE
:1042D00091FEBDE80840FEF73FBC000009217A20AE
:1042E00008B5FDF743F907213220BDE80840FDF786
:1042F0003DB9000008B5FFF7A3FE00F00BF8FDF78D
:1043000007FBFDF7D9F9FFF749FEBDE80840FFF7C5
:10431000E5BB00007047000010B50139024490422F
:1043200001D1002005E0037811F8014FA34201D02C
:10433000181B10BD0130F2E7034611F8012B03F8FA
:10434000012B002AF9D17047346162383434656436
:10435000343636633131383100000000121000006D
:10436000121100001213000053544D333248373FEE
:104370003F3F0053544D3332483733782F3732782C
:104380000053544D3332483734332F3735332F37BA
:104390003530000001105A00031059000120580068
:1043A00003205600100002400800024000080240AE
:1043B00000000B00280002400800024004080240F0
:1043C00006010C00400002400800024008080240BC
:1043D00010020D0058000240080002400C08024084
:1043E00016030E00700002400C000240100802404C
:1043F00000040F00880002400C0002401408024034
:1044000006051000A00002400C00024018080240FF
:1044100010061100B80002400C0002401C080240C7
:1044200016072F0010040240080402402008024032
:104430000008380028040240080402402408024012
:1044400006093900400402400804024028080240DE
:10445000100A3A0058040240080402402C080240A6
:10446000160B3B00700402400C040240300802406E
:10447000000C3C00880402400C0402403408024056
:10448000060D4400A00402400C040240380802401B
:10449000100E4500B80402400C0402403C080240E3
:1044A000160F46000000000035160008211600080F
:1044B0005D16000849160008551600084116000848
:1044C0002D160008191600086916000800000000E3
:1044D000010000000000000063300000D844000824
:1044E00098240020A82600204172647550696C6FE2
:1044F000740025424F415244252D424C002553451E
:104500005249414C2500000002000000000000005C
:1045100055180008C518000840004000583F00200A
:10452000683F0020020000000000000003000000BF
:10453000000000000D19000800000000100000003D
:10454000783F002000000000010000000000000093
:1045500094420020010102002124000831230008B8
:10456000CD230008B1230008430000007045000877
:1045700009024300020100C03209040000010202E6
:104580000100052400100105240100010424020299
:104590000524060001070582030800FF0904010045
:1045A000020A000000070501024000000705810221
:1045B0004000000012000000BC450008120110017C
:1045C00002000040091241570002010203010000ED
:1045D0000403090425424F415244250041495242F7
:1045E0005241494E48373433003031323334353656
:1045F000373839414243444546000000000000205E
:104600000000020002000000000000300000040072
:104610000800000000000024000008000400000062
:104620000004000000FC0000020000000000043054
:1046300000800000080000000000003800000100B9
:104640000100000000000000691A0008211D000898
:10465000CD1D000840004000CC430020CC4300208A
:1046600001000000DC430020800000004001000049
:104670000800000000010000001000000800000019
:104680006D61696E0069646C650000004000802AFD
:1046900000000000AAAAAAAA40000024FFFF000010
:1046A0000000000000A00A00000000000000000060
:1046B000AAAAAAAA00000000FFFF00000000000054
:1046C000000000000000000000000000AAAAAAAA42
:1046D00000000000FFFF00000000000000000000DC
:1046E0000001400000000000AAAAAAAA00010000E0
:1046F000FFF70000000000000000000000000000C4
:1047000000000000AAAAAAAA00000000FFFF000003
:104710000000000000000000000000000000000099
:10472000AAAAAAAA00000000FFFF000000000000E3
:10473000000000000000000000000000AAAAAAAAD1
:1047400000000000FFFF000000000000000000006B
:104750000000000000000000AAAAAAAA00000000B1
:10476000FFFF00000000000000000000000000004B
:1047700000000000AAAAAAAA00000000FFFF000093
:104780000000000000000000000000000000000029
:10479000AAAAAAAA00000000FFFF00000000000073
:1047A000000000000000000000000000AAAAAAAA61
:1047B00000000000FFFF00000000000000000000FB
:1047C000B70400000000000000001A000000000014
:1047D000FF000000000000006843000883040000A0
:1047E0007343000850040000814300080096000055
:1047F000000008009600000000080000040000000F
:10480000D04500080000000000000000000000008B
:10481000000000000000000000000000FFFFFFFF9C
:10482000FFFFFFFFFFFFFFFFFFFFFFFFFFFFFFFF98
:10483000FFFFFFFFFFFFFFFFFFFFFFFFFFFFFFFF88
:10484000FFFFFFFFFFFFFFFFFFFFFFFFFFFFFFFF78
:10485000FFFFFFFFFFFFFFFFFFFFFFFFFFFFFFFF68
:020000040805ED
:020000040806EC
:10000000000600309D0D0608BDC412085103060805
:1000100045C412083DC4120841C412089F0D0608C9
:100020009F0D06089F0D06089F0D060829A31708B7
:100030009F0D06089F0D06089F0D06089F0D0608D8
:100040009F0D06089F0D06089F0D06089F0D0608C8
:100050009F0D06089F0D0608B9B21708E5B21708EC
:1000600011B317083DB3170869B31708155B1708D4
:100070003D5B1708695B1708955B1708C15B17089C
:10008000E95B1708155C1708395717089F0D060814
:100090009F0D06089F0D06089F0D060895B31708CB
:1000A0009F0D0608F9B417089F0D06080DB517082F
:1000B00011B5170825B517089F0D06080D6217081A
:1000C000356317089F0D06089F0D0608656617081B
:1000D0007D6617086DB4170881B4170895B4170822
:1000E000F9B317089F0D06089F0D06084DB51708B0
:1000F0009F0D06089F0D06089F0D0608415C170816
:100100009F0D06089F0D060839B517089F0D0608B4
:10011000A9B41708BDB417089F0D06089F0D06085F
:100120006D5C1708955C1708C15C1708ED5C170833
:10013000195D17089F0D06089F0D06089F0D0608FC
:100140009F0D06089F0D06089F0D06089F0D0608C7
:10015000415D17086D5D1708995D17089F0D06082A
:100160009F0D06089F0D06089F0D06089F0D0608A7
:100170009F0D060815AF17089F0D06089F0D06086E
:100180009F0D06089F0D0608D1B41708E5B417089F
:10019000956617089F0D06089F0D06089F0D060817
:1001A0009F0D06089F0D06089F0D06089F0D060867
:1001B0009F0D06089F0D06089F0D06089F0D060857
:1001C0009F0D06089F0D06089F0D06089F0D060847
:1001D0009F0D060801AF17089F0D06089F0D060822
:1001E0009F0D06089F0D06089F0D06089F0D060827
:1001F0009F0D06089F0D06089F0D06089F0D060817
:100200009F0D06089F0D06089F0D06089F0D060806
:100210009F0D06089F0D06089F0D06089F0D0608F6
:100220009F0D06089F0D06089F0D06089F0D0608E6
:100230009F0D06089F0D06089F0D060859571708C1
:100240009F0D0608E158170809591708355917086E
:10025000615917088D591708B9591708E559170832
:10026000115A17089F0D06089F0D06089F0D0608D6
:100270009F0D06089F0D06089F0D06089F0D060896
:100280009F0D06089F0D06089F0D06089F0D060886
:100290009F0D06089F0D06089F0D06089F0D060876
:1002A0009F0D06089F0D06089F0D06089F0D060866
:1002B0009F0D06089F0D06089F0D06089F0D060856
:1002C0009F0D06089F0D06089F0D06089F0D060846
:1002D0009F0D06089F0D06089F0D06089F0D060836
:1002E00055450608DD7C0608BDBE0608D929070865
:1002F000599A0708294D0808A5550A08F5AF0C08B2
:100300002DB60C0811460D08EDAB0D0845B50D08CE
:1003100095B80D08A13E0E0815450E0889670E0810
:1003200011CA0F08995F100879BD1208EDD612089E
:1003300031501608B1771608A58E1608BDC01608EC
:1003400081C6160800000000000000000000000048
:10035000EFF30383EFF30982EFF30881DFF814D0A2
:100360002DE9FE4F684600F0F1FFBDE8FE4F8D46D7
:1003700070470000AC320030F1EE101AA0EC200AF9
:1003800001607047A0EC108A704700BF81F0004107
:1003900002E000BF83F0004330B54FEA41044FEA6A
:1003A000430594EA050F08BF90EA020F1FBF54EA05
:1003B000000C55EA020C7FEA645C7FEA655C00F0A1
:1003C000E2804FEA5454D4EB5555B8BF6D420CDD72
:1003D0002C4480EA020281EA030382EA000083EAF5
:1003E000010180EA020281EA0303362D88BF30BD95
:1003F00011F0004F4FEA01314FF4801C4CEA1131EB
:1004000002D0404261EB410113F0004F4FEA033349
:100410004CEA133302D0524263EB430394EA050FD4
:1004200000F0A780A4F10104D5F1200E0DDB02FA43
:100430000EFC22FA05F2801841F1000103FA0EF2D7
:10044000801843FA05F359410EE0A5F120050EF19D
:10045000200E012A03FA0EFC28BF4CF0020C43FACE
:1004600005F3C01851EBE37101F0004507D54FF0DB
:10047000000EDCF1000C7EEB00006EEB0101B1F52B
:10048000801F1BD3B1F5001F0CD349085FEA300071
:100490004FEA3C0C04F101044FEA445212F5800F7C
:1004A00080F09A80BCF1004F08BF5FEA500C50F119
:1004B000000041EB045141EA050130BD5FEA4C0CFC
:1004C000404141EB0101013C28BFB1F5801FE9D259
:1004D00091F0000F04BF01460020B1FA81F308BF7C
:1004E0002033A3F10B03B3F120020CDA0C3208DD48
:1004F00002F1140CC2F10C0201FA0CF021FA02F123
:100500000CE002F11402D8BFC2F1200C01FA02F192
:1005100020FA0CFCDCBF41EA0C019040E41AA2BFB7
:1005200001EB0451294330BD6FEA04041F3C1CDA7F
:100530000C340EDC04F11404C4F1200220FA04F09F
:1005400001FA02F340EA030021FA04F345EA030149
:1005500030BDC4F10C04C4F1200220FA02F001FA0B
:1005600004F340EA0300294630BD21FA04F029468D
:1005700030BD94F0000F83F4801306BF81F4801126
:100580000134013D4EE77FEA645C18BF7FEA655C99
:1005900029D094EA050F08BF90EA020F05D054EA6B
:1005A000000C04BF1946104630BD91EA030F1EBF70
:1005B0000021002030BD5FEA545C05D14000494174
:1005C00028BF41F0004130BD14F580043CBF01F567
:1005D000801130BD01F0004545F0FE4141F470014D
:1005E0004FF0000030BD7FEA645C1ABF1946104628
:1005F0007FEA655C1CBF0B46024650EA013406BF29
:1006000052EA033591EA030F41F4002130BD00BFE7
:1006100090F0000F04BF0021704730B54FF48064A4
:1006200004F132044FF000054FF0000150E700BF25
:1006300090F0000F04BF0021704730B54FF4806484
:1006400004F1320410F0004548BF40424FF0000171
:100650003EE700BF42004FEAE2014FEA31014FEAB4
:1006600002701FBF12F07F4393F07F4F81F0605103
:10067000704732F07F4208BF704793F07F4F04BF4E
:1006800041F40021704730B54FF4607401F000452B
:1006900021F000411CE700BF50EA010208BF70478B
:1006A00030B54FF000050AE050EA010208BF70477C
:1006B00030B511F0004502D5404261EB41014FF4E5
:1006C000806404F132045FEA915C3FF4D8AE4FF0ED
:1006D00003025FEADC0C18BF03325FEADC0C18BFD0
:1006E000033202EBDC02C2F1200300FA03FC20FA21
:1006F00002F001FA03FE40EA0E0021FA02F114446E
:10070000BDE600BF80F0004002E000BF81F0004184
:1007100042001FBF5FEA410392EA030F7FEA226CA7
:100720007FEA236C6AD04FEA1262D2EB1363C1BF37
:10073000D218414048404140B8BF5B42192B88BFA6
:10074000704710F0004F40F4000020F07F4018BFC9
:10075000404211F0004F41F4000121F07F4118BFE9
:10076000494292EA030F3FD0A2F1010241FA03FC91
:1007700010EB0C00C3F1200301FA03F100F0004379
:1007800002D5494260EB4000B0F5000F13D3B0F141
:10079000807F06D340084FEA310102F10102FE2AB0
:1007A00051D2B1F1004F40EBC25008BF20F0010020
:1007B00040EA03007047490040EB0000013A28BFBF
:1007C000B0F5000FEDD2B0FA80FCACF1080CB2EB42
:1007D0000C0200FA0CF0AABF00EBC25052421843C0
:1007E000BCBFD0401843704792F0000F81F4000165
:1007F00006BF80F400000132013BB5E74FEA410338
:100800007FEA226C18BF7FEA236C21D092EA030FA3
:1008100004D092F0000F08BF0846704790EA010F1D
:100820001CBF0020704712F07F4F04D1400028BF4A
:1008300040F00040704712F100723CBF00F500002C
:10084000704700F0004343F0FE4040F40000704762
:100850007FEA226216BF08467FEA2363014642020E
:1008600006BF5FEA412390EA010F40F48000704721
:100870004FF0000304E000BF10F0004348BF4042C7
:100880005FEA000C08BF704743F0964301464FF003
:1008900000001CE050EA010208BF70474FF000035F
:1008A0000AE000BF50EA010208BF704711F00043A0
:1008B00002D5404261EB41015FEA010C02BF844670
:1008C0000146002043F0B64308BFA3F18053A3F5CF
:1008D0000003BCFA8CF2083AA3EBC25310DB01FA16
:1008E00002FC634400FA02FCC2F12002BCF1004F9A
:1008F00020FA02F243EB020008BF20F0010070472B
:1009000002F1200201FA02FCC2F1200250EA4C007E
:1009100021FA02F243EB020008BF20EADC707047C4
:100920007BB972B90029BEBF00204FF0004106E03C
:1009300008BF00281CBF6FF000414FF0FF3000F0EF
:100940002BBAADF1080C6DE904CE002909DB002BB0
:100950001ADB00F0B9F8DDF804E0DDE9022304B0A9
:100960007047404261EB4101002B1BDB00F0ACF80B
:10097000DDF804E0DDE9022304B0404261EB41010F
:10098000524263EB43037047524263EB430300F070
:100990009BF8DDF804E0DDE9022304B0404261EB9E
:1009A00041017047524263EB430300F08DF8DDF8DC
:1009B00004E0DDE9022304B0524263EB43037047D5
:1009C00053B94AB9002908BF00281CBF4FF0FF31B6
:1009D0004FF0FF3000F0E0B9ADF1080C6DE904CE46
:1009E00000F072F8DDF804E0DDE9022304B070479E
:1009F000430803F05533C01A830803F0333300F083
:100A00003330184400EB101000F00F3000EB0020E2
:100A100000EB0040000E704708B502460B4643EC61
:100A2000172BB5EEC07BF1EE10FA03D4BDE80840F9
:100A300000F02AB8B1EE477B51EC170B00F024F818
:100A4000404261EB410108BD9FED0B6B07EE900A40
:100A50009FED0B5BB7EEE77A27EE066BBCEEC66B3D
:100A6000B8EE464BA4EE457BFCEEC77B16EE101AA3
:100A700017EE900A704700BF000000000000F03D34
:100A8000000000000000F0419FED0B6B41EC170BE4
:100A90009FED0B5B27EE066BBCEEC66BB8EE464BCC
:100AA000A4EE457BFCEEC77B16EE101A17EE900AFB
:100AB000704700BFAFF30080000000000000F03D71
:100AC000000000000000F0412DE9F047089D0446B9
:100AD0008E46002B4DD18A42944669D9B2FA82F2F1
:100AE00052B101FA02F3C2F1200120FA01F10CFA2D
:100AF00002FC41EA030E94404FEA1C48210CBEFB65
:100B0000F8F61FFA8CF708FB16E341EA034306FBED
:100B100007F199420AD91CEB030306F1FF3080F07C
:100B20001F81994240F21C81023E63445B1AA4B2C9
:100B3000B3FBF8F008FB103344EA034400FB07F76B
:100B4000A7420AD91CEB040400F1FF3380F00A81AC
:100B5000A74240F207816444023840EA0640E41BA1
:100B600000261DB1D4400023C5E900433146BDE84D
:100B7000F0878B4209D9002D00F0EF800026C5E9EF
:100B8000000130463146BDE8F087B3FA83F6002E07
:100B90004AD18B4202D3824200F2F980841A61EB7F
:100BA000030301209E46002DE0D0C5E9004EDDE79D
:100BB00002B9FFDEB2FA82F2002A40F09280A1EB85
:100BC0000C014FEA1C471FFA8CFE0126200CB1FBDA
:100BD000F7F307FB131140EA01410EFB03F08842D3
:100BE00008D91CEB010103F1FF3802D2884200F260
:100BF000CB804346091AA4B2B1FBF7F007FB1011F2
:100C000044EA01440EFB00FEA64508D91CEB04048F
:100C100000F1FF3102D2A64500F2BB800846A4EBEA
:100C20000E0440EA03409CE7C6F12007B34022FAD5
:100C300007FC4CEA030C20FA07F401FA06F31C4304
:100C4000F9404FEA1C4900FA06F3B1FBF9F8200C11
:100C50001FFA8CFE09FB181140EA014108FB0EF057
:100C6000884202FA06F20BD91CEB010108F1FF3AA7
:100C700080F08880884240F28580A8F102086144B3
:100C8000091AA4B2B1FBF9F009FB101144EA0141C1
:100C900000FB0EFE8E4508D91CEB010100F1FF346C
:100CA0006CD28E456AD90238614440EA0840A0FB04
:100CB0000294A1EB0E01A142C846A64656D353D0DA
:100CC0005DB1B3EB080261EB0E0101FA07F722FAFE
:100CD00006F3F1401F43C5E9007100263146BDE827
:100CE000F087C2F12003D8400CFA02FC21FA03F38A
:100CF000914001434FEA1C471FFA8CFEB3FBF7F00B
:100D000007FB10360B0C43EA064300FB0EF69E422F
:100D100004FA02F408D91CEB030300F1FF382FD2C8
:100D20009E422DD9023863449B1B89B2B3FBF7F670
:100D300007FB163341EA034106FB0EF38B4208D949
:100D40001CEB010106F1FF3816D28B4214D9023E8A
:100D50006144C91A46EA004638E72E46284605E7A8
:100D60000646E3E61846F8E64B45A9D2B9EB020879
:100D700064EB0C0E0138A3E74646EAE7204694E709
:100D80004046D1E7D0467BE7023B614432E730463C
:100D900009E76444023842E7704700BF02E000F010
:100DA00000F8FEE772B6374880F30888364880F3CB
:100DB000098836483649086040F20000CCF200004D
:100DC0004EF63471CEF200010860BFF34F8FBFF3CF
:100DD0006F8F40F20000C0F2F0004EF68851CEF264
:100DE00000010860BFF34F8FBFF36F8F4FF000001B
:100DF000E1EE100A4EF63C71CEF2000108600620CA
:100E000080F31488BFF36F8F19F1F0FA1AF182FEA4
:100E10004FF055301F491B4A91423CBF41F8040B2B
:100E2000FAE71D49184A91423CBF41F8040BFAE722
:100E30001A491B4A1B4B9A423EBF51F8040B42F819
:100E4000040BF8E700201849184A91423CBF41F8CA
:100E5000040BFAE719F108FB1AF1E0FE144C154DEA
:100E6000AC4203DA54F8041B8847F9E703F0D2FADE
:100E7000114C124DAC4203DA54F8041B8847F9E7D1
:100E800019F1F0BA00060030002200300000060818
:100E900008ED00E00000003000060030208E1B0846
:100EA00000220030B4300030B830003024E9013086
:100EB000E002060844030608440306084403060843
:100EC0002DE9F04F2DED108AC1F80CD0D0F80CD0E0
:100ED000BDEC108ABDE8F08F002383F3118828460B
:100EE000A047002018F104F8FEE717F16DFE00DFBF
:100EF000FEE7000070B54FF0FF0C4CF4E06C1CEA0C
:100F000011541DBF1CEA135594EA0C0F95EA0C0FFF
:100F100000F0DEF82C4481EA030621EA4C5123EA72
:100F20004C5350EA013518BF52EA033541F48011A1
:100F300043F4801338D0A0FB02CE4FF00005E1FB54
:100F400002E506F00042E0FB03E54FF00006E1FB9E
:100F500003569CF0000F18BF4EF0010EA4F1FF04E1
:100F6000B6F5007F64F5407404D25FEA4E0E6D4121
:100F700046EB060642EAC62141EA55514FEAC52032
:100F800040EA5E504FEACE2EB4F1FD0C88BFBCF5AE
:100F9000E06F1ED8BEF1004F08BF5FEA500E50F15F
:100FA000000041EB045170BD06F0004646EA010125
:100FB00040EA020081EA0301B4EB5C04C2BFD4EB57
:100FC0000C0541EA045170BD41F480114FF0000E50
:100FD000013C00F3AB8014F1360FDEBF002001F0BE
:100FE000004170BDC4F10004203C35DA0C341BDC38
:100FF00004F11404C4F1200500FA05F320FA04F00A
:1010000001FA05F240EA020001F0004221F000413D
:1010100010EBD37021FA04F642EB06015EEA430EB0
:1010200008BF20EAD37070BDC4F10C04C4F12005E0
:1010300000FA04F320FA05F001FA04F240EA020093
:1010400001F0004110EBD37041F100015EEA430E64
:1010500008BF20EAD37070BDC4F1200500FA05F284
:101060004EEA020E20FA04F301FA05F243EA020303
:1010700021FA04F001F0004121FA04F220EA020012
:1010800000EBD3705EEA430E08BF20EAD37070BD58
:1010900094F0000F0FD101F00046400041EB010138
:1010A00011F4801F08BF013CF7D041EA060195F01A
:1010B000000F18BF704703F00046520043EB0303D4
:1010C00013F4801F08BF013DF7D043EA06037047C1
:1010D00094EA0C0F0CEA135518BF95EA0C0F0CD0CC
:1010E00050EA410618BF52EA4306D1D181EA030112
:1010F00001F000414FF0000070BD50EA410606BF0C
:101100001046194652EA430619D094EA0C0F02D150
:1011100050EA013613D195EA0C0F05D152EA033695
:101120001CBF104619460AD181EA030101F00041B3
:1011300041F0FE4141F470014FF0000070BD41F0FC
:10114000FE4141F4780170BD4FEA410212F50012F0
:1011500015D211D56FF47873B3EB625212D94FEAFE
:10116000C12343F0004343EA505311F0004F23FAE8
:1011700002F018BF404270474FF00000704750EA3D
:10118000013005D111F0004008BF6FF000407047FA
:101190004FF00000704700BF4FEA4102B2F1E04358
:1011A00024BFB3F5001CDCF1FE5C0DD901F0004C4E
:1011B0004FEAC0024CEA5070B2F1004F40EB83009E
:1011C00008BF20F00100704711F0804F21D113F1CA
:1011D0003872BCBF01F00040704741F480114FEA03
:1011E0005252C2F11802C2F1200C10FA0CF320FA8C
:1011F00002F018BF40F001004FEAC1234FEAD323A9
:1012000003FA0CFC40EA0C0023FA02F34FEA430312
:10121000CCE77FEA625307D150EA01331EBF4FF09B
:10122000FE4040F44000704701F0004040F0FE40B6
:1012300040F40000704700BF01F0FF01102A2BDBD3
:1012400010F0070F08D010F8013B013A8B422DD067
:1012500010F0070F42B3F6D1F0B441EA012141EAA0
:10126000014122F007047FF000070023F0E8025656
:10127000083C85EA010586EA010685FA47F5A3FAE6
:1012800087F586FA47F6A5FA87F68EB9EED1F0BC57
:1012900001F0FF0102F0070232B110F8013B013A00
:1012A00083EA010313B1F8D1002070470138704779
:1012B000002D06BF35460338073815F0010F07D15A
:1012C000013015F4807F02BF013015F4C03F0130BA
:1012D000F0BC0138704700BFEC46A0E8F05F4FF06B
:1012E00000007047B0E8F05FE546080008BF012045
:1012F000704700BF10F8012B11F8013B012A28BFED
:101300009A42F7D0D01A7047034613F8012B002AEF
:10131000FBD1181A0138704710B5044620461CB19D
:1013200054F80C3B013300D110BD0822012100F01C
:1013300071FB54F80C0C54F8082C14F8041C121A05
:10134000B2FBF1F200F066FBE8E70000C26AD0E908
:10135000003112F0040F2DE9F04118BF0B46A6B082
:101360000021594C042601270291CDE90003D00643
:101370004CBF03F1200203F168020392DA6903997A
:10138000D2099B6902F004021B880A4303F47F43DD
:1013900003924FF0E022A3F53E41D2F8882D02F4EB
:1013A000A002B2F5A00F04BF012202924B424B41B2
:1013B0000493464D03A82C6000F02AFA0422012170
:1013C000434800F027FB0422012102A800F022FB81
:1013D00010220121019800F01DFB0098202201211C
:1013E0000C3000F017FB019804220121103000F0AE
:1013F00011FB0422012103A800F00CFB01980C2230
:101400000121143000F006FB0C220121009800F0AD
:1014100001FB029BDA071FD5009BDB6ADB064ED47B
:1014200015A8FEF7AFFFDDF804C00DF1140E0CF1A6
:1014300020030CF160081868083353F8041C724646
:10144000434503C29646F6D1DCF8603025938422EA
:10145000012105A800F0DEFA00F0C0F8FFF75CFFFC
:101460004FF0E023D3F8003D03F47023B3F5402F91
:101470000ED0184B05A88DF81C60059314338DF819
:10148000287006934FF0FF33CDE90833FFF744FF90
:101490002B68A34206D0104B0422012105A8059316
:1014A00000F0B8FA00F02AFA002882D0049B1BB1A1
:1014B000019A93690233936126B0BDE8F08105A8D3
:1014C000FEF75AFFC3E700BFED55CEACB830003091
:1014D0005C48180828ED00E0ACCE55ED37B50E4D50
:1014E0002A78202A15D10D4C0D4823680D4918443F
:1014F000019218F137F923680021019A2033094835
:10150000297023601EF1FCFA03B0BDE8304018F1E9
:101510001FBE03B030BD00BFAC320030D43200304B
:10152000E09C1B08AE32003008B5262015F1D2FF32
:10153000144BD3F8902042F40032C3F89020D3F833
:10154000902022F40032C3F89020D3F89020D3F8F2
:10155000E82042F40032C3F8E820D3F8102142F426
:101560000032C3F810216D22D3F81031064BDA6037
:101570004FF0FF321A620D221A600122034B1A70DB
:1015800008BD00BF0044025800440040E43200306F
:10159000014B1868704700BFFCFF1F08014B024851
:1015A000C01A7047E09C1B080000200800487047E4
:1015B000E09C1B0807490022074B5B1A9A4201D3A3
:1015C0000120704751F8040B013001D10432F5E7D6
:1015D00000207047E09C1B08000020085E4B2DE9AE
:1015E000F74F1A6802255D4B02F56A58DFF89491AF
:1015F0001A7808F118085A4F5A4C9044DFF888A11D
:1016000017F1F8F9A9EB070B06460EB14E2D49D993
:10161000A9EB0702B2EB080700F192804E2D00F211
:101620008F80DFF868C16B1C4F4E0C21DBB2ACEB36
:1016300006006943B84273DD60184FF0010C665034
:1016400090463E4480F808C04660B2EB080213D4CE
:101650004F2B11D0454E19464548AB1C351ADBB20D
:1016600095424FF00C0505FB01F163DD651801267D
:10167000024460502E726A600C2201215343E2182A
:1016800011724FF0FF31E15051603A4B1B782BB192
:10169000394B1B682360394B1B686360314803B0CA
:1016A000BDE8F08F336AF06953450ABF344BF31A33
:1016B000A3EB0A0380B1019318F142FA019B58B1E0
:1016C0002A460C2101354A430121EDB2A0180172CE
:1016D000F169A1500D3141600C200121984400FBBB
:1016E00005FCD84504EB0C0244F80C6006F13C0CF8
:1016F0001172C2F804C005EB010205F10205D2B275
:10170000EDB200FB02F204EB02000172316AA1505B
:101710001944416014D2304617F17CF9064674E74B
:1017200067184FF0010E8044665087F808E0C7F84C
:1017300004C08AE7621801256050157256609BE765
:101740004F2D01D82B4697E7012384F8BC334FF087
:10175000FF33C4E9ED3398E7D4320030AC320030C7
:10176000E09C1B0804220030B83000300000043038
:1017700028E9013000220030D8320030D032003069
:1017800000220030000020080006003024E901306B
:101790000C4B1B7810B50BB9FFF7C6FE00230A49A6
:1017A0000A48CA699206FCD54A6A1C5CD2B29442C5
:1017B00005D10133DBB20E2BF3D1002010BD002385
:1017C000EFE700BFE43200300044004060481808F2
:1017D00038B5084B04461B780BB9FFF7A5FEE4B2F9
:1017E000054DAC62EB695B0600D538BD18F1B0FC65
:1017F000F8E700BFE43200300044004010B5441E5A
:1018000014F8010F00B910BDFFF7E2FFF8E7000080
:1018100070B502680446EFF30581D9205369C9B257
:10182000CAF012FE294B1B78A3B1294B94E80300A0
:1018300083E803002748FFF7E1FF6368B3B1264858
:10184000FFF7DCFF2548FFF7D9FFFFF7A1FF24488A
:10185000FFF7D4FF234D2B783BB124681CB1204601
:1018600018F16EF920B900232B7070BD1E48E7E710
:1018700020461E4E18F178F900F2145084421FD20F
:10188000204618F171F930602046194E18F180F9A0
:1018900004F5E053834217D9204618F179F93060F6
:1018A0000023144A1360144A1370FFF783FE0028C4
:1018B000D9D018F14DFC0120BDE8704017F1DABF16
:1018C000A4F214533360DFE73360E9E7AD32003050
:1018D000DC32003070481808754818088648180827
:1018E000606919080022003080481808D83200309A
:1018F000D0320030D4320030AC320030284B1A786D
:1019000070B542B12748FFF779FF274B5868003878
:1019100018BF012070BD254A107800283CD0244E05
:10192000244C33682448254D1A1D21782D1A0A4469
:10193000AA4205D3224A4FF0FF31D1612022227002
:101940002278D2B103F120018D4205D81F2A9FBF12
:101950001B4AD3612022227020221949184417F112
:1019600001FF32682378002115481344202221709A
:1019700033601EF1C5F818F1EBFB33689D4207D9BF
:101980000F4920220F48CB6117F1ECFE18F1E0FB64
:10199000002017F16FFFB8E701221A70BAE700BF05
:1019A000AD320030CC481808DC3200300022003064
:1019B000D4320030AC320030E09C1B08000020081C
:1019C000AE320030E0FF1F082DE9F84307460E460F
:1019D0000024DFF83890DFF83880B44201D1BDE848
:1019E000F88324B1230702D14846FFF707FF3D5D86
:1019F00001342B0905F00F0518F80300FFF7E8FE86
:101A000018F80500FFF7E4FEE7E700BF6069190872
:101A1000DC481808474B1B782DE9F74F07460E4660
:101A200090465BB1022925D0042938D0012902D182
:101A30001146FFF7C9FF4048FFF7E0FE3F4B1B7818
:101A4000002B4ED03E4A00253E4BA2EB030938E066
:101A500037F81430ADF8043024B1620702D12846BB
:101A6000FFF7CCFE0134022101A8FFF7ADFFA0452E
:101A7000EED1E0E70024304DF9E757F82430019328
:101A800024B1A30702D12846FFF7B8FE0421013490
:101A90000DEB0100FFF798FFA045EED1CBE7002446
:101AA000254DF9E7FFF71AFD022E1DD0042E2CD08C
:101AB000012E06D12378795D5A1C2270224AD15416
:101AC0000135A8450DD0214B214C1B6822780433E9
:101AD00013444B45E6D31C4B4FF0FF32DA61202311
:101AE000237003B0BDE8F08F2378DFF85CA05A1CA8
:101AF00022703A780AF80320FFF7F0FC23785A1C8A
:101B0000227000220AF80320DAE74FF0000ADFF81B
:101B100038B022783B78511C23FA0AF30AF1080AFC
:101B200021700BF80230FFF7D9FCBAF1200FF0D189
:101B3000C6E700BFAD3200306069190800220030EE
:101B400000002008E09C1B08AE320030D432003088
:101B5000AC320030036800221B6818477FB5039140
:101B600040210546B4F0C0FF039A18B9012420466D
:101B700004B070BD134E039296F9623E002BF5D06F
:101B800082F028FC437A039A53B982F023FC847ACA
:101B9000039A2CB90C4B40212846B4F0ADFFE6E780
:101BA0000A4BB6F9641ED3F8643BB3F90830994286
:101BB000DCDD074B4021284600240093054BB4F0A0
:101BC0009BFFD4E7E8620030F0481808E882003054
:101BD0000F491808FD481808F0B50D4620210446A5
:101BE0002DED028B9DB0B4F07FFF002800F0BA808D
:101BF0005D4E96F9623EBBB106F50052B6F9643E01
:101C0000D2F8642BB2F90C1003F10A02914203DD01
:101C100040F28D32934207DC544B2A462021204665
:101C2000B4F06AFF002099E096F9513E022B05D1ED
:101C30004F4B2A4620212046B4F05EFFB6F8283EDE
:101C400041F65832A3F57A739BB293420FD8494FAD
:101C500006F69862D7F83C3A92ED007AD3ED097A0D
:101C6000B4EEE77AF1EE10FA03DD434BD5E7434BD0
:101C7000D3E706F69C62D3ED0B7A92ED007AB4EED0
:101C8000E77AF1EE10FAF0DCB6F95E3E002B01DCEB
:101C90003B4BC2E7A7F5405393F898280D2A06D886
:101CA0000123934013F4215F01D0364BB5E736484A
:101CB00012F0E6F9012806D1D7F8480ABEF092FFE3
:101CC00048B1012810D0314B93F8211F11F01001B9
:101CD0002AD02F4BA1E72F4B00932F4B2A462021D0
:101CE0002046B4F009FF9DE7284B93F87C3BCBB12D
:101CF00019212A4869F056FFA0B106F63C63192164
:101D0000264893ED008A69F07DFFDFED257AB8EE75
:101D1000C88A20EE270AB4EEC08AF1EE10FAD2DDAE
:101D2000204BD9E7204BD7E7602204A803911DF18F
:101D3000E7FE642303AA1D49D7F8440ABCF07EFFDE
:101D400018B903AB00931A4BC8E7642303AA1949D7
:101D5000D7F83C0AB9F0E6FD0028F2D01DB0BDEC82
:101D6000028BF0BD0120F9E7E8620030184918083D
:101D70002B491808E8A2003063491808534918088D
:101D80007D49180892491808C4C20030E882003022
:101D9000234A1808D7491808B249180820430030C8
:101DA0000000C842F6491808E7491808384A1808D8
:101DB0003C4A18084E4A180870B59AB00E460021E1
:101DC0006022054602A801911DF19AFE642201A934
:101DD00009489BF083F8044640B99DF9043043B9A3
:101DE000064B074A31462846B5F090F820461AB00F
:101DF00070BD01ABF5E700BFAC8B0030544A18084A
:101E00005DDD1A0808B51AF03BF90121BDE808406C
:101E100019F074B92DE9F043DFF850910546ADB0E3
:101E20000E46D9F8080F03681B69984780461AF0D8
:101E300027F900210746602214A813911DF160FEC6
:101E4000642313AA4146384619F048FB044648B9B2
:101E500013AB3B4A31462846B5F058F820462DB022
:101E6000BDE8F083374899F0C1F9B8F1000F03D10C
:101E700095F91E30012B0AD1334816F033FF80B993
:101E8000324A31462846B5F041F80024E6E710F022
:101E9000060FE3D0A9F5A04016F024FF08B92C4A9C
:101EA000EFE703A9384619F01BF928B19DF80D306A
:101EB0005B0601D5274AE4E7DFF8B4800023D8EDBC
:101EC000007AF5EEC07AF1EE10FAC7DD0DF12009C7
:101ED0000893099305AA0A9307AB04A9384601930E
:101EE00006ABCDF8009019F019FD1B4B48460B933B
:101EF0001A4B0D931A4B0F931A4B11933FF0FEFDA3
:101F0000059B0422D8ED007A0E93049B8DED0C0AFC
:101F10001093069B12930BAB93ED017AB4EEE77A24
:101F2000F1EE10FA04D5013A03F10803F4D195E774
:101F30001B6831460C4A2846B4F0E8FFA5E700BF0D
:101F40006C4A1808CC6C0030E8320030754A18082A
:101F50008C4A1808B24A18084FA718080C8C1A089F
:101F600009B91A0852C21808C04A1808E882003095
:101F70006871003008B5064B93F8213F9B0704D5E4
:101F8000044AB4F0C3FF002008BD0120FCE700BFF5
:101F9000E8820030D04A180870B50C4C05460E4651
:101FA000D4F8080F03685B69984710B101242046F4
:101FB00070BDA4F5A04016F0A7FE04460028F5D198
:101FC000034A31462846B4F0A1FFF0E7E88200302A
:101FD000E04A18082DE9704D484D9BB082468B466B
:101FE000D5F82C3F93F8D56066B9454B1B68986AC5
:101FF00003685B6B9847044640B9424A59465046CD
:10200000B4F084FF30461BB0BDE8708D82F0E2F979
:10201000202183F0AFFC58B182F0DCF91F2183F05E
:10202000A9FC80B30024384A59465046B4F06EFFEC
:1020300095F8F63E43B195F8F83E2BB10024334AAB
:1020400059465046B4F062FF59465046B6F01AF869
:1020500000216022884202A8019108BF0C461DF1B0
:102060004FFDD5F82C0F01AA642103681B6898471F
:10207000054680B92C4601AB254A59465046B4F076
:1020800045FF2646BEE782F0A5F9A52183F072FC44
:102090000028C7D1CCE7002CF3D0DAF808303BB9E0
:1020A000DAF80030594650469B6B98470446E8E7FB
:1020B00059465046FFF790FD804659465046FFF777
:1020C0007BFE08EA00005946C4B25046FFF752FFB3
:1020D000594604405046FFF741FD594604405046DA
:1020E000FFF75AFF594604405046B5F05DF859468F
:1020F00004405046B5F0DEFF0440C2E7E8820030FD
:1021000088C70030F44A18080B4B1808254B1808EC
:102110003D4B180808B5FFF75DFF034A82F8E80E4B
:10212000024A907108BD00BFE88200309DC90030AE
:10213000F7B506460F46B4F013FD0446A0B30221DE
:102140003046B4F0D1FC054670B319F099FF4FF456
:102150008071044618F0D2FF48BB20464FF400714E
:1021600018F0CCFF04460023019319F089FF01A960
:1021700018F05CFDECB1DDED017A0F4BF1EE677A02
:1021800093ED007A77EEC77AB7EE007AF0EEE77A51
:10219000F4EEC77AF1EE10FA06DD0024074B3A465A
:1021A00002213046B4F0A8FC204603B0F0BD002464
:1021B000D9E72C46F8E700BFF0AC0030484B1808D0
:1021C000F8B504460F46B5F08BF8102105462046B9
:1021D000B4F08AFC58B12046FFF714FE064630B929
:1021E0003546044B3A4610212046B4F085FC28467B
:1021F000F8BD00BF5C4B180870B505460E46B4F03C
:10220000F5FB044678B180212846B4F06DFC50B14E
:10221000074B93F8ED3443B10024064B324680213E
:102220002846B4F069FC204670BD0446FBE700BFB9
:10223000E8920030704B180838B50D4D0446D5F8BB
:10224000480ABEF0CFFC012810D0D5F8480ABEF0ED
:10225000C9FC022804D02046BDE83840B4F0C8BB11
:10226000044811F00DFF0128F5D138BD0020FCE72E
:10227000E8A20030C4C20030F0B50F4D85B006466C
:102280000F46D5F85C3B6A460093D5F8603B019356
:10229000D5F8643B0293D5F8683B0393B5F080FE14
:1022A000044639463046B4F081FC2040C0B285F87F
:1022B000E70E05B0F0BD00BFE88200302DE9F8431D
:1022C000DFF8AC90064626480F4698F08FFF04468C
:1022D000D9F8080FDFF89C8003681B69984705460A
:1022E00030B914F0060F03D1D9F83C3F022B09D1C5
:1022F00039463046B4F02CFD054618B9002488F85C
:1023000007400AE039463046FFF784FD04460028BE
:10231000F4D02DB9012388F807302046BDE8F883B2
:1023200008213046B4F0E0FB0028F3D00D482BF034
:10233000A3F80028EED00C4BB02193F8142401FB35
:10234000023203F54053B2F81E22B3F9523E9A42CC
:10235000E0DD064B3A4608213046B4F0CDFBCDE730
:10236000CC6C003008340030E8320030844B180860
:10237000E88200309DC9003070B588B005460E4631
:10238000B4F0ECFD044688B320212846B4F0ACFB41
:1023900060B31B4B93F8802B42B393F85C3B9B07D5
:1023A00024D507AA06A9174894F026FDF0B19DEDA3
:1023B000077ADFED157AB4EEE77AF1EE10FA15D868
:1023C000B7EEC77A0024202128468DED027BDDED93
:1023D000067AFDEEE77A08A3D3E90023CDED007A73
:1023E000CDE90423094B3246B4F086FB204608B001
:1023F00070BD00BFAFF30080000000403333E33F07
:10240000E8A20030DC7100309A99193F944B18080B
:102410002DE9F3410F46054619F032FE804618F0CB
:1024200021FE044640B9594A01212846B4F06EFD08
:10243000204602B0BDE8F081404619F007FB48B9DC
:1024400023F0DAFA90F8461323F0C4F9044608B9E9
:102450004F4AE9E74F4E3946D6F8080F03689B69A3
:102460009847044658B9D6F8080F03689B6C9847FC
:10247000494A034601212846B4F048FDD8E7AB6835
:10248000002BD5D010212846B4F02EFB20B3D8ED78
:10249000967A98ED950A20EE270A1AF113FCDFEDE3
:1024A0003F7AA6F5005320EE270ADFED3D7AB3F917
:1024B000283E20EE270A07EE903AF8EEE77AB4EECF
:1024C000E70AF1EE10FA07DD364B0122102128460B
:1024D000B4F012FB0024ABE720212846B4F004FB43
:1024E00038B196F8213FDB0603D52F4B012220217E
:1024F000EDE740212846B4F0F7FAE8B1012F14D0F7
:10250000232F12D0042F10D0284800F0C3FBB5EEC3
:10251000C00AF1EE10FA1DDD254B012240212846AC
:102520000093244BB4F0E8FAD4E7D6F8080F036818
:102530005B6C98470028E7D01F4B1B68D86A03687C
:10254000DB6998470128014619D11C4A2846B4F096
:10255000DDFCBFE7D6F8080F03685B69984730B128
:10256000D6F8643BB3F90A30002BE5DDD4E7D6F8A2
:10257000080F03681B6898470B28DDD1F0E7394640
:10258000284602B0BDE8F041B5F098B9C04B180834
:10259000D14B1808E8820030E54B1808E02E654260
:1025A0000000C842F94B1808234A1808E8320030E6
:1025B0000F491808014C180888C700300D4C18083E
:1025C00070B505460E46FFF725FC084B044631461C
:1025D000D8712846FFF7E0FC00283146284608BF9E
:1025E0000024B5F08BFC204070BD00BF9DC90030B9
:1025F0002DE9F341554F3B78002B40F0A480544C1B
:102600000126D4F82C5F3E7095F8D55025B13B706B
:10261000284602B0BDE8F081B5F014FE054630B999
:102620004C4A3870137843F001031370F0E773F0ED
:10263000FBFF314673F01AF9A4F5A04007F090FEB5
:10264000454B1E710B26013E62F00EFA62F02AF92C
:1026500016F0FF06F7D1414801F0C4FA19F010FD59
:1026600004F65472D0F81812116090F88832DA0724
:1026700053D418F0A9FF73F0D7FF3C2173F010FF7B
:1026800004F6147300221A600021344801F054FB50
:10269000324816F027FB01463148C5F09BFC314B10
:1026A000314E01211B68D86A03681B68984796F869
:1026B000BC3BD4F82C0F6FF3410386F8BC3B036896
:1026C000DB6A98470121D4F82C0FC1F05BFD73F051
:1026D000ABFF8046D4F8080F03681B689847A6F53F
:1026E00080430146404693F8382C4FF0000873F0C1
:1026F00095FAA6F5E04007F025FE6FF0C1FC6EF0FC
:10270000EDFF87F80080C9F00BFF0123C6F8540ADB
:1027100084F8F93E84F8FD8E7AE79B07B4D43146FD
:102720000E4805F0B5FE0023019319F0A9FC01A99C
:1027300018F07CFADDED017A04F61473F1EE677A95
:10274000C3ED007AA0E7002562E700BFE532003064
:10275000E8820030BCC900309DC90030E83200304A
:10276000A089003088C70030E8A200302DE9F0438E
:102770003F4C87B007460D46D4F82C3F164693F8D9
:10278000D530002B71D05AB1012901D0232907D1AE
:1027900094F8EB3E23B90025284607B0BDE8F08346
:1027A000002D56D0294632463846B5F00BFE054678
:1027B0000028F0D019F064FC074623F01DF980468C
:1027C000384618F003F9D8B198F92830022B17D100
:1027D00000264FF00009F1B203AA3846CDF80C905C
:1027E0000191CDF81090CDF8149018F013FD0199D7
:1027F00018B103AA404622F0ABFD0136032EEAD100
:1028000001211C4808F01CF801211A4807F070FF4C
:102810000021D4F82C0FC1F0B5FC174841F0C2FDDF
:1028200073F002FF002173F021F8144B00211B68A4
:10283000D86A03681B689847D4F8081F002310481B
:1028400084F8F93E0B1A383059425941C5F004FE5C
:10285000A2E7D4F8080F03685B6998470028A1D164
:1028600094F8EB3E002B9DD195E7012594E700BF3E
:10287000E8820030E832003028BB003088C70030E2
:1028800038BE00300020704710B5064CD4F8080F51
:1028900003685B6A984718B1D4F82C3F93F8D500C9
:1028A00010BD00BFE882003030B52DED028B87B03F
:1028B000B0EE408A0C46FFF7E7FF0546E8B1B4EEFC
:1028C000488A2268636803A9D4ED027AF1EE10FA0F
:1028D0009FED0C0AF1EE677A039204934FF0000229
:1028E0004FF00103084850FE080ACDED057ACDE906
:1028F000002368BF13460FF077FB284607B0BDECF6
:10290000028B30BD0000000060C1003007B50191AE
:10291000FFF7BAFF30B10199044803B05DF804EB4A
:1029200000F0E6BB03B05DF804FB00BFE832003006
:10293000014898F017BE00BFCC6C003000F5A040F5
:1029400008B590F8E93E8B4209D080F8E91E31B114
:1029500073F06AFE0F21BDE8084073F0A1BD08BD09
:1029600070B500F5A04605460C46D6F83C3F8B42B4
:1029700012D0012911D0022916D059B973F054FE92
:102980001B2173F08DFD0D4A05F5BA40062110306C
:1029900079F0C4F9C6F83C4F70BD73F045FE1A21BA
:1029A00073F07EFD064AEFE7012101F0C5F973F0EF
:1029B0003BFE1D2173F074FD024AE5E7884C1808C0
:1029C0009D4C1808984C180800F5A04210B592F8D4
:1029D000213F0C4603F00101A14209D064F300033A
:1029E00082F8213FDB0704D407F086F8024B9C7283
:1029F00010BD07F077FAF9E79DC9003000F5A04057
:102A000090F8213F61F3410380F8213F014B197396
:102A1000704700BF9DC9003010B5044681F0DAFC54
:102A2000202182F0A7FF003804F5A04418BF012040
:102A300084F8F60E10BD000070B504466FF020FB60
:102A4000436F04F5E045D5F8442AC2F86832D5F85A
:102A50003C2A936604F5104292F89D244AB904F585
:102A6000A044D4F82C2FD360D5F83C0A03689B6DA2
:102A70009847D5F83C0A0368BDE87040DB6D1847FD
:102A8000F0B500F5A04504462DED028BD5F82C3F9E
:102A900083B093F8D530002B00F0908095F8EB3E92
:102AA000002B40F08B8000F5004393F87037002B2B
:102AB00040F08480D5F8080F03685B6998470028C8
:102AC0007CD1404BD3F8080F03681B6898470B284C
:102AD00074D004F5E0479FED3C7AD7F8443AD3ED43
:102AE000C57AF0EEE77AF4EEC77AF1EE10FA65D522
:102AF00019F0C6FA95F8E02C01A919F09FF8002802
:102B00005CD0D5F82C0F443075F0DEFF0346B7EEED
:102B1000001A9B20DFED2D0A93ED000A38F0ACFF80
:102B2000B5EEC00AF1EE10FA48DDDDED017A9FED59
:102B3000287AF0EEE77AF4EEC77AF1EE10FA3DD596
:102B400004F58056D7F83C0A06F6984393ED848A3C
:102B50000368D3F89C309847DFED1E7A9FED1E7A0C
:102B6000A0EE678AB0EEC88AB4EEC78AF1EE10FA1A
:102B700024D506F69846D6ED857AFDEEE77A17EE6F
:102B8000903A002BB8BF5B4207EE903AF8EEE77A36
:102B9000F4EEC77AF1EE10FA10D59FED100AD5F8D1
:102BA0002C0FC2F06FFFD5F82C3F04F5A3509FED1A
:102BB0000B0AD3ED0C0A1030AAF08EFC03B0BDEC6A
:102BC000028BF0BDE88200300000003400000000FD
:102BD0009A99193FD4023739C2B8B23D0AD7233C7B
:102BE00000F5A04008B5D0F82C0F03685B69984742
:102BF000F6EE007A20EE270AB5EEC00AF1EE10FAE2
:102C000048BF9FED010A08BD0000000038B500F57F
:102C1000E0450446B7EE001A7C2004F5A044DFED41
:102C2000110A2DED028BD5F83C3A93ED370A38F0B6
:102C300023FFD4F82C0FB0EE408AD5F8445A03682D
:102C400005F5BA755B69984738EE400ADFED067AFC
:102C50002846BDEC028B20EE270ABDE83840A7F0DD
:102C60001DB800BF0000000000007A4400F5A0433A
:102C7000B3F9683743B900F54050B0F95E0E00284B
:102C8000B8BF404280B2704783EAE370A0EBE370C4
:102C9000F8E7000038B52DED028B044681F09AFB71
:102CA0000368DB68984720B99FED310ABDEC028BC1
:102CB00038BD304B04F54055DFED2F8A5920D3F84D
:102CC000643BB0EE681ADFED2A0AB3F90A3000EE71
:102CD000103AB8EEC00A38F0CFFE4FF4C8720021A7
:102CE000B5F9660EB0EE408A38F02EFFA5F8660EF4
:102CF000204615F07DF9B5F9663E07EE900AB8EE6C
:102D0000E77A07EE903AF8EEE77A77EE676AB4EE84
:102D1000E68AF1EE10FA11D5204638EE668AFFF702
:102D2000A5FF07EE900AB8EEE70ADFED147A20EE71
:102D3000270A20EE088A88EE260AB7E777EE877A18
:102D4000B4EEE78AF1EE10FAAEDDB5F95E3E38EE8C
:102D5000678A9FED0A7A78EEE77A00EE103AB8EECD
:102D6000C00A20EE070A20EE088A88EE270A9DE7AF
:102D700000000000E882003000007A440AD7233CBB
:102D80007047000070470000002070470020704727
:102D900000207047002070470020704700207047D7
:102DA00000207047002070470020704770470000E7
:102DB00000F5795034307047004870478482180815
:102DC00000F5A040D0F8080F03681B681847000002
:102DD000034808603621117008221A60704700BF4E
:102DE0000453180800F5E0409FED0A7AD0F8503AF5
:102DF0000120D3ED0C7AF4EEC77AF1EE10FABEBFE3
:102E0000D3ED027A9FED047A67EE877AC1ED007AFE
:102E1000704700BF000000340AD7233C00F5A040F3
:102E2000D0F8080F0368DB6E1847000000F5004378
:102E300093F8113B002B14BF1B2003200B1A5842A0
:102E40005841704700F5A04090F8210FC0F3800072
:102E50007047000000F5A040D0F8080F0368DB6D54
:102E60001847000000F5A040D0F8080F03685B6D1C
:102E70001847000000F5A040D0F8080F03681B6D4C
:102E80001847000000F5A04300F50840D3F8083FBC
:102E900008301B1A584258417047000000F5A04006
:102EA00010B5D0F8080F0C4603685B6E98470120F8
:102EB00084ED000A10BD000000F5A04010B5D0F868
:102EC000080F0C4603681B6E9847012084ED000A2A
:102ED00010BD000000F5A04010B5D0F8080F0C465A
:102EE00003689B6E9847DFED047A012020EE270AE5
:102EF00084ED000A10BD00BF0AD7233C15F05CBC6E
:102F00008BF0FCBD16F05CBE04F00EBF90F0A2BAD0
:102F10006FF002B835F08CBB72F026BE1EF08EB991
:102F200084F060BA80F040BE7EF0FABA14F05CBD66
:102F300015F054BD07F09CBE16F09ABD06F032BEE7
:102F400006F080BB06F0A6BA14F05CBE8DF0FABBAA
:102F500097F054BF11F0BEBFFFF792BD14F0FCBD57
:102F600093F068BF15F06EBC03F030BF14F080BD65
:102F700081F0E2B863F0C2BD2BF07CBF07F0A6BAC7
:102F800003F0B2BA84F03EBA15F0A4BC07F01EBE3E
:102F900005F06ABA07F0A4BF06F00EBB07F01ABB33
:102FA00014F018BDFFF748BD36F008B82DE9F0471A
:102FB00000F50E46054688469146B0369A460024EE
:102FC000374657F8040B08B303681B689847404519
:102FD00019D157F8040C03689B6C98474946FEF7D3
:102FE00089F980B957F8040C0368DB6C9847042210
:102FF00051461DF1A1FC30B904F50E542C3455F89E
:103000002440383431E00134052CDAD141462846D9
:1030100007F090FE0446B8BB074656F8043B7BBB5E
:10302000484607F50E5416F177FD814604215046B7
:103030001DF1AAFC2C340646B9F1000F0CD058B192
:10304000442021F077FE074620B133464A464146E8
:103050000FF0ECFC45F8247055F8244044B948467C
:1030600016F1FAFC304616F1F7FC2046BDE8F08771
:1030700005F5A04595F8E13E013385F8E13EC0E74E
:103080000137052FC9D1F0E70024EEE700F5E04055
:1030900008B5D0F8500ABDF033F9012008BD000092
:1030A00010B400F5084400F5A0400834D0F8080F2B
:1030B000A04203D15DF8044B09F0C0BD00205DF8CB
:1030C000044B704700F5084300F5A0400833D0F8E2
:1030D000080F984201D109F0CFBD704715F0E4B850
:1030E00006F07EBF0BF05EBE0BF090BC0BF024BC74
:1030F0001FB500F5A04304460391D3F8080F0368F9
:103100005B6A984760B10023DFED060A04F50E40C4
:103110000399B0EE600A1A46783000930EF09CFDD9
:1031200004B010BD0000000000F5A04313B5044634
:10313000D3F8080F8DED010A03685B6A98479DED8F
:10314000010A18B90024204602B010BD04F50E4053
:1031500078300DF09DFF04460028F3D0012102488D
:10316000FFF7ECFBEFE700BFE83200307FB5044625
:1031700068460D46164620F07BFF04F5A0436946DD
:10318000D3F8080F0368DB6D98476946284621F09D
:10319000D3F810B9002004B070BD6946284621F06C
:1031A000D7F80028F6D0284620F0A6FF054630467E
:1031B00020F0A2FF8542EDD12368314620461B6AEC
:1031C0009847E8E700F5A04370B50646D3F8080F26
:1031D00086B00C4603685B6A98470546C0B1226812
:1031E00006F50E40636803A9D4ED027A7830DFED6E
:1031F0000A0AF1EE677A0392049301220023B0EEEB
:10320000600ACDED057ACDE900321A460EF0ECFEEB
:10321000284606B070BD00BF00000000F0B514469F
:1032200000F5A04207460D462DED028BD2F8080F9F
:103230008DB0B0EE408A0268F0EE608A0593526A63
:103240009047064648B36A6807F50E40D5ED027A06
:10325000079278306268F1EE677A29680A92012253
:10326000CDED087A0292D4ED027A9DF854209FEDBC
:103270000D0AF1EE677A0691019268EE800A2168E4
:1032800028EE000A9DF85020099106A9009209AA8B
:10329000059BCDED0B7A0EF043FE30460DB0BDEC34
:1032A000028BF0BD35FA8E3C30B50C4600F5A041DE
:1032B00005462DED028BD1F8080F8BB0B0EE408A99
:1032C0000168F0EE608A0392496A0293884738B336
:1032D00094ED027A05F50E409DF84410B1EE477A60
:1032E00094ED005A94ED016A78309FED0F0AB7EE25
:1032F000C55AB7EEC66A0191B7EEC77A9DF840107D
:1033000068EE800A029B009128EE000A039A04A945
:103310008DED045B8DED066B8DED087B0EF0CAFB29
:103320000BB0BDEC028B30BD35FA8E3C00F5A043EE
:1033300070B50646D3F8080F90B00D4603681446E2
:103340005B6A984798B395ED027A06F50E4063687C
:103350000AA9B1EE477A95ED005A95ED016A7830E9
:10336000DFED140AB7EEC55AB7EEC77A2268B7EE9A
:10337000C66A059300230492B0EE600A04AA009383
:10338000CDED070ACDED080ACDED090A8DED0E7BD6
:10339000D4ED027AF1EE677ACDE9013307ABCDEDDA
:1033A000067A8DED0A5B8DED0C6B0EF0F5FA10B020
:1033B00070BD00BF00000000F0B51C4600F5A04342
:1033C00007460E4615462DED028BD3F8080F91B037
:1033D000B0EE408A0368F0EE608A5B6A9847002886
:1033E0003ED096ED027A07F50E406B680AA9B1EE61
:1033F000477A2A68059378306368B7EEC77A96ED06
:10340000005A08939DF86830B7EEC55A96ED016AE8
:1034100002939DF86430B7EEC66A9FED130A0492DA
:10342000019368EE800A226828EE000A9DF8603059
:10343000079204AA009307AB8DED0E7BD5ED027ABF
:10344000F1EE677A8DED0A5BCDED067AD4ED027A66
:10345000F1EE677A8DED0C6BCDED097A0EF09CFAEA
:1034600011B0BDEC028BF0BD35FA8E3C00F5A043E7
:1034700070B506462DED048BD3F8080F88B0F0EE3A
:10348000408A0368B0EE609AF0EE419A5B6AB0EE53
:10349000618A9847054600B39FED120A00244FF059
:1034A0007E5304A829EE801A079469EE000A04935B
:1034B00028EE800A069405943CF0E4F89FED0A0A91
:1034C00006F50E40002301AA28EE000A04A9783070
:1034D0000194029403940EF069F9284608B0BDECFB
:1034E000048B70BD35FA8E3C0000C84200F5A04345
:1034F00030B505462DED048BD3F8080F89B0F0EEFA
:10350000409A0368B0EE609AF0EE418A5B6AB0EED2
:10351000618A98470446F0B14FF07E5304A80493A3
:1035200000230793069305933CF012FB9FED0C0AD2
:1035300001A8CDED019A8DED029ACDED038A3DF003
:1035400013FF05F50E40B0EE480A012301AA04A9B5
:1035500078300EF02BF9204609B0BDEC048B30BD5D
:1035600035FA8E3C094A0B4692F8EB2E2AB100221E
:103570008A604A600A600120704700F5E040D0F898
:103580003C2A783207CA83E80700F4E7E882003073
:10359000684B70B5044640F8043B8BF0CDFB00252A
:1035A00004F1100004F577561DF024FA04F16800C8
:1035B0006EF040FA04F5907029F04AFE04F5AA6016
:1035C0001BF0A0FD04F5DF6021F03AFC04F5246057
:1035D00034F048FE04F668708BF05CF904F5815015
:1035E0000C36183068F0F8F904F59B5072F09EF82C
:1035F00004F5A050183096F0F1FE04F5A1501430F7
:1036000083F06EFD04F5A3501030AAF0C9FD04F557
:10361000D850B2F013F804F5D8501C306EF0C4FD49
:1036200004F5E05010308CF073FD04F5805304F580
:10363000E250414A83F8345C04F5E153043014331A
:10364000136060F023FF04F5E4502946183016F0AB
:1036500097FE04F50B5038308FF00CFF04F50C503A
:103660002830A7F03BFE04F532503430A8F0F8FBC8
:1036700004F548503830AEF0FFFE04F54D501030E0
:10368000B1F036F904F54E503430B1F06BFD04F56D
:1036900050500C30A6F038FD04F5525034301AF07A
:1036A000E7FC04F558501830A8F052FD04F55950C5
:1036B0003830B3F05FF904F5675020490C3066F0FC
:1036C00007FD04F56750243097F032FC04F56B5089
:1036D0001030B3F023F804F56C502830C8F040FFE8
:1036E00004F56F50143083F04BF904F5405383F820
:1036F000385C04F571550C3528460C3575F0E0F949
:10370000AE42F9D104F577500D4D1830B3F086F87C
:1037100004F577503C3075F03DF82B6813B109483B
:10372000C8F0D0FE2046084966F0D2FC20462C6046
:1037300070BD00BF7088190848D6003030271A08BD
:103740009CCA0030AC4C18080887190810B514F052
:10375000C9FB80F03FFE0368BDE810405B68184776
:10376000FFF7F4BF10B5044606F0D4FF204615F06D
:10377000E1FA204604F0E6FC2046BDE8104004F0E3
:1037800027BE0000FFF7EEBF70B500F5BE4504464A
:10379000583528461CF0F8FF22F02EF990F9253014
:1037A00093B390F844337BB304F5A04304F5DF668C
:1037B000D3F82C0F443075F087F90346B7EE001AA2
:1037C0009B20DFED120A93ED000A38F055F994F9C9
:1037D000303728460021012B04F6541408BF86ED2B
:1037E0000F0A1CF067FDDFED0A7A94ED287A304667
:1037F00020EE270ADFED077AA7EE270A84ED280AD4
:10380000BDE8704022F008B870BD00BF00000000A5
:10381000CDCCCC3D6666663FFFF7B6BF10B5012143
:10382000044615F0C3FAA0B1184BD3F8080F03688B
:103830009B6A984768B9204602F062FD04F5104380
:1038400093F89D342BB9204602F060FD204602F02B
:1038500065FD4FF40011204615F0A8FA40B104F5BB
:10386000104393F89D341BB936F06AFB34F008FC22
:103870004FF48021204615F099FA28B136F060FB0C
:10388000BDE8104034F00ABB10BD00BFE882003034
:10389000FFF7C4BF70B500F5E046044686B09FED63
:1038A000620AD6F83C0A6C303DF00AFD04F5E4509B
:1038B00003A98DED030A1830CDED040A8DED051A2C
:1038C00016F0FAFB0221204615F070FAB0B1012182
:1038D000204615F06BFA88B9544BD3F8080F0368EB
:1038E0009B6A984750B9204602F00AFD04F5104340
:1038F00093F89D3413B9204602F008FD01212046BB
:1039000015F054FA70B9494BD3F8080F03689B6A55
:10391000984738B904F5104393F89D3413B92046FD
:1039200002F0FCFC0121204615F040FA10B92046B7
:1039300002F04CFD4FF40031204615F037FA30B15B
:1039400004F5A043D3F82C0F03689B6C98474021E3
:10395000204615F02BFA60B104F59B50019071F0F0
:10396000EDF904F58053019893F934340BB171F0FB
:10397000A9FB4FF48061204615F018FA18B104F540
:103980009B5071F075FA2021204615F00FFA58B1BE
:1039900004F5A045D5F8080F03681B69984720B3C4
:1039A000D6F8440ABAF090F88021204615F0FEF9C6
:1039B00040B336F0C5FA34F095FA1021204615F0E0
:1039C000F5F920B104F57B50343093F063FB4FF4EC
:1039D0000041204615F0EAF918B304F5F5405830D7
:1039E00006B0BDE8704083F091BE20460FF00EF99E
:1039F0000028D5D1D5F8080F03685B6998470028DF
:103A0000CED0D1E74FF48021204615F0CFF9002821
:103A1000CFD14FF40021204615F0C8F90028C8D1B5
:103A2000CBE706B070BD00BFE02E6542E8820030F3
:103A3000FFF730BF10B50121044615F0B7F910B1FA
:103A4000204602F0C3FC8021204615F0AFF948B1B2
:103A50004FF48021204615F0A9F918B936F070FA14
:103A600034F01CFA4FF40011204615F09FF930B1E4
:103A700004F5A350BDE810401030A9F0C5BD10BD3D
:103A8000FFF7D8BF10B5044606F07AFB204606F0D3
:103A9000C7F9204606F0BAFB204616F053FA204636
:103AA000BDE8104004F024B9FFF7ECBF00F5BD43BA
:103AB000002201216333104610B513F8014F14B1F1
:103AC00001FA02F4204301321B2AF6D110BD000096
:103AD0002DE9F0434FF6FF7187B0044615F066F903
:103AE00038B12046FFF7E2FF07210246204602F0E8
:103AF0009DFC04F5A045D5F82C3F93F8D5309BB933
:103B00002046FEF789FFD5F82C0F04F5804304F515
:103B10004052016892F87A2E4E6A93F89818B0478E
:103B2000D5F82C0FC1F07AFF82F028FE04F510467C
:103B300082F05AFA204616F059F895F8EB3E04F553
:103B4000004204F5E04783F0010382F88D361F4AF6
:103B5000537196F89D345BB9D7F83C8AD8F8003099
:103B6000D3F874906EF08CFA6DF0DEFE4046C847D4
:103B7000D7F8447A6EF084FA6DF0D6FE07F5BA777E
:103B80003846A5F059FE96F89C34CBB995F94C3BD4
:103B9000B3B10F4B06AA049401241B68986A03680A
:103BA0001D6D0C4B05930623CDE901344FF4C06322
:103BB0000093094B12E90600A84720B186F89C44FF
:103BC00007B0BDE8F08305481CF0F0FF9DC9003048
:103BD00088C70030DD3006086E211908C04C18086F
:103BE000FFF776BF2DE9F04100F5805600F5A044BF
:103BF000DFED1B7A054606F6984304F5746804F673
:103C00004477D3F85C22C8F80020D3F868223A60E1
:103C100093ED860A30EE270AB7EEC00A37F0FCFEB5
:103C2000B7EEC00B04F648734FF6FF71284683EDDC
:103C3000000A04F64C73D8F8002004F575641A6085
:103C40003B68236015F0B2F838B1D6F8A42E2846A8
:103C50000921BDE8F04102F0C1BBBDE8F08100BF21
:103C6000DB0F494038B500F5A0450446D5F83C3F88
:103C7000002B4FD095F8EC3E002B4BD0002385F85D
:103C8000EC3E80F0A7FB0368DB689847002841D032
:103C9000D5F85C3BB3F90A2006EE102AD5F8602B64
:103CA000B2F90A20B8EEC66A07EE902AD5F83C2F82
:103CB000012AF8EEE75A2ED105F5746292ED007AEA
:103CC00005F6447292ED005A67EE257A65EEC56AF4
:103CD000E5EE067AE7EE066A04F5E45090EDA07A88
:103CE00090ED9D6A27EE877AA6EE867ABDEEC77ABA
:103CF00017EE102A5A8190ED9D7AD5F8603B67EE59
:103D0000877A90EDA07AE6EEC77AFDEEE77A17EEB5
:103D1000902A5A8138BD05F64C72D2ED007A05F52D
:103D2000756292ED007A65EEC76AE7EE866A67EE25
:103D3000A57AE7EE067ACFE738B5054600F5A04448
:103D40002DED028BE1B1284604F6487513F022FFF1
:103D5000B0EE408A95ED000A30EE480AB7EEC00A90
:103D600037F072FEB7EEC00BDFED187AB0EEC00A86
:103D7000B4EEE70AF1EE10FA10D5BDEC028B38BDB7
:103D8000D4F83C3F022BF8D113F0EAFEF2EE047AAD
:103D9000B4EEE70AF1EE10FAD5D5EEE79FED0C0A86
:103DA00085ED008A38EE008AB0EE480A17F184FFEC
:103DB00004F64C7304F5756483ED000AB0EE480A0E
:103DC00018F116FE84ED000AD7E700BFC2B8B23D75
:103DD000DB0F494000F5E4500121183018F0B4B869
:103DE000FFF7F8BF10B5044614F0EEFC1021204692
:103DF00014F0DCFF98B1204602F0CEF94FF4001128
:103E0000204614F0D3FF50B936F09AF834F038F960
:103E100004F5A350BDE810401030A9F0F5BB10BD6B
:103E2000FFF7E0BFF8B5044606F058FF224B4FF607
:103E3000FF76254604F17C004FF0FF3745F8383B0C
:103E40001E4B6465C4E916341D4BC4E918341D4B80
:103E5000A36620F00DF904F1980020F009F904F1AF
:103E6000B40020F005F9184B04F1D000A4F8CC60A0
:103E7000C4F8C83020F0FCF8144B15492846C4F8A3
:103E800080721D6066F024F904F52570A4F8747042
:103E9000A4F8906020F0ECF804F52C7020F0E8F81D
:103EA00004F5337020F0E4F80023204684F8E03273
:103EB000C4F80433F8BD00BF80B01808E530060828
:103EC000E9300608ED3006080000FFFF70C9003039
:103ED000F83E190810B5044606F000FF0A4B04F13D
:103EE0003C0023600123238720F0C2F804F14C003A
:103EF00020F0BEF804F15C0020F0BAF804F16C0088
:103F000020F0B6F8204610BD30BD18082DE9F0436A
:103F1000044689B0FFF73CFBA44B04F57A5004F546
:103F2000A045236004F5B64628304FF07C5702F0D8
:103F300085FC04F5795305A906F188002833059717
:103F40004FF000094FF00108C5F8743B062385F8CF
:103F5000783B74F097FE06F1A400C7F037FC04F537
:103F6000B746192304A906F15400049785F8C43B09
:103F700004F5B84785F8BC9B74F084FE06F1700028
:103F8000C7F024FC2837182385F8088C384606AE7D
:103F900085F8103CB2F036FD854B3146381DC5F82A
:103FA000283C8DF8188067F09FF804F5B940814FE0
:103FB000103062F053FD04F5B9405430B2F00CFDFE
:103FC0007D4B04F5B9403146C5F8D43C6C300697BA
:103FD00074F058FE04F5B940069704F5BA47314627
:103FE000783074F04FFE1037744B07F10C00C5F8B1
:103FF000103DC7F0EBFB1E234FF4E16085F8748E93
:10400000C5F87C3EA5F8809E20F09AFEC5F8780E93
:1040100004F5BD400430C7F0D9FB04F5BD4048307D
:10402000C7F0D4FB664B1A6802B91F60384604F526
:10403000104764494FF07E5866F04AF86437624B87
:1040400004F5BE40C5F8087FC5F8103D0C30B4F04B
:10405000FDF905F5746304F5BE4005F64C75C3F82B
:1040600000804FF40071594B5830C5F8008004F5BA
:10407000E0450793564B0694009396E80C001BF01E
:104080005BFF04F5C94070309DF0D2FB04F5F440AD
:1040900003A9CDF80C800C3074F01EFE04F5F4403A
:1040A00003A9CDF80C80203004F5F74874F0EAFD40
:1040B00004F5F44008F168082C301FF0D9FF04F52E
:1040C000F4404FF4004158301CF09AFD04F5F540DF
:1040D000583083F071F904F5F6405C3099F0C6F978
:1040E00004F5F740183067F035F93A4B04F5F7401E
:1040F000C5F8983B2C3096F023FE04F5F740364B7C
:1041000048303649186065F0E3FFFF2334494046E4
:1041100085F8FC3B85F8043C65F0DAFF314B1E68FE
:1041200016B13148C8F0CEF904F5F840C3F8008064
:1041300004F505450C306FF049F904F50440D0351D
:10414000B830BBF0BFF804F50540C830BAF04CFFFA
:104150002846A4F0D3FC294604F5074004F50045A1
:10416000C2F04EFC214B04F50742DFF898C0C5F8B9
:1041700000370623603285F854371D4BC3F800C062
:104180003346142698B2013306FB00C1097C00298E
:10419000F8D1184B1880184B1880184BD3F80080B2
:1041A000B8F1000F30D01648BCE700BF4C571808D4
:1041B000244C18080000A040684C180864AD190889
:1041C00000CF0030E8A8190838581808E130060870
:1041D0003C571808844C180850D6003000D01908F5
:1041E00064251A0814D70030CC4C180830A71808DA
:1041F00058CA003056CA00302CCA003000CA0030FD
:10420000ED4C1808949C180804F507401A606D4B93
:1042100003A9743004F50B46039374F033FD04F5E1
:1042200007405036943006F059FD674B04F50740BF
:10423000C5F89437D03006F051FD644B04F50840C2
:10424000C5F8D0370830FFF7EDFD304606F046FDE3
:104250005F4B06F138000026C5F8503BC5F0D6FE8E
:104260005C4B04F50D40C5F8883B383006F036FD50
:10427000594B04F50D40C5F8383D783006F02EFD59
:10428000564B04F50D4085F8B08DC5F8783DB43037
:1042900006F024FD524B04F50D40C5F8B43DEC305A
:1042A00006F01CFD4F4B04F50E40C5F8EC3D05F63D
:1042B00024633C301E605E609E6006F00FFD4A4B3A
:1042C00004F50E40C5F83C3E783006F007FD474B3C
:1042D00004F50E40C5F8783E05F57C65C43006F05F
:1042E000FDFC434B04F50F4045F8FC3C083006F05C
:1042F000F5FC404B04F50F4045F8B83C443006F05F
:10430000EDFC3D4B04F50F4045F87C3CDC302E6065
:104310006E6004F51045FFF7DDFD384606F0DEFC63
:10432000364B284604F514476B66A030383710F03A
:10433000ADFE04F51140683006F0D0FC304B04F5BA
:104340001140C5F86831A03006F0C8FC2D4B04F5CB
:104350001140A5F8D881C5F8A031EC3006F0BEFCBC
:10436000294B04F51240C5F8EC312830FFF7B2FDB7
:10437000264B002204F51240C5F828320123D03024
:1043800085F8AD320023C5E9AE23C5E9B023C5E900
:10439000B2230BF01BFF04F5134005F27445A03067
:1043A00012F024FA384606F099FC194B07F1480040
:1043B00045F83C3C2E606E60C7F008FA204609B014
:1043C000BDE8F083CDCC4C3D44AC1808F8AC1808DF
:1043D00034B11808D4B1180844B31808F4B3180855
:1043E000A4B418084CB51808A8B7180858B8180885
:1043F00050BA1808F8BA1808A8BB1808ACBE1808B4
:1044000094B21808E8C21808B0B91808F8BD18081E
:10441000BCC3180838B5054B0A4601461C6823681A
:1044200020461D68024BA847002038BD88C70030D1
:10443000E832003038B5037904463BB905682DB140
:10444000284632F0C5FE284620F07CFC204638BDC8
:104450002B4B70B50360044600F565502C301FF0FF
:1044600093FD04F5405393F8A82342B9D3F8A4531D
:104470002DB1284632F0ACFE284620F063FC04F54E
:10448000D85004F6EC75B1F0EDF804F5B45004F62C
:104490008C760430FFF7CEFF04F5B3501C30FFF7E5
:1044A000C9FF04F5B3501430FFF7C4FF04F5A15061
:1044B000143082F02DFEB54204D0183D284632F06B
:1044C00085FAF8E70F4B04F63C50C4F8403AFFF782
:1044D000B1FF04F63450FFF7ADFF04F62C50FFF7A0
:1044E000A9FF04F53D6075F02FF904F63C3075F036
:1044F0002BF904F6A82075F027F9204670BD00BFFF
:1045000070881908102D190838B5104B044603603F
:1045100000F5004393F8F42642B9D3F8F0562DB1D4
:10452000284632F055FE284620F00CFC04F5A04346
:10453000074AD3F8780EC3F8102D08B120F006FC16
:104540002046FFF785FF204638BD00BF4C571808AE
:1045500064AD190810B5C7F00BFC064C064B18608B
:104560002046FFF7D3FC2046044A0549BDE8104029
:1045700017F19CBBE832003088C700303C35013071
:10458000094506080120704790F830308B4286BFFD
:1045900000EB8100406B00207047000090F8303045
:1045A0008B4286BF00EB8100406B0020704700000B
:1045B000FA207047034BD3F83C0F431E5842584132
:1045C000704700BFE8820030034BD3F83C0F831ED6
:1045D00058425841704700BFE8820030034BD3F87F
:1045E0002C0F08B1BFF0CCBE01487047E882003004
:1045F0002458180870B5436A04464D4D43F4E05200
:104600004262826A42F4E0528262C26A42F4E0523A
:10461000C262D5F8442AE2B143F4F8434362D5F8C4
:10462000440AB8F03BFD38B1A36A43F48043A36267
:10463000E36A43F48043E362D5F8440AB8F020FE0D
:1046400038B1A36A43F40053A362E36A43F400530E
:10465000E362384892F02AFC18B1636A43F0806341
:104660006362344892F0CEFB18B1A36A43F08063D2
:10467000A362304892F04CFC18B9E36A43F08063BF
:10468000E3622D4B1D6845B11921284667F08AFA6F
:1046900018B1636A43F480736362284E96F87C3BDA
:1046A0006BB1A36A43F48073A36245B11921284614
:1046B00067F0C4FA18B1E36A43F48073E362204BF5
:1046C00093F9B8248AB1D4E9091242F0800241F08A
:1046D0008001A262616293F9B82432B193F8B825DF
:1046E0001AB1E26A42F08002E26293F8B034013B10
:1046F000012B0BD8D4E9092343F4800342F4800250
:10470000A362E36A626243F48003E362636A43F094
:1047100080436362A36A43F08043A362D6F82C3FD0
:1047200093F8C1301BB9E36A43F08043E36270BD84
:10473000E8A20030DC71003064CA0030E88200304A
:10474000E8B2003013B54FF45C70019120F0F2FA3A
:10475000044620B101997EF0C3F9024B2360204644
:1047600002B010BDE05818080020704770470000E4
:104770000320704708207047034B187810B9034B8B
:1047800093F8FA0E704700BF34C90030E882003059
:104790007047000008B50C4BD3F8440A70B91023D9
:1047A0000A4A43F04000D2F82C2F22B192F8D520CB
:1047B0000AB143F0C00040F0010008BDB8F06EFC43
:1047C0000028ECD01823EBE7E8A20030E8820030A4
:1047D00038B5C5780B4604463522352D4FF000011B
:1047E000184628BF35251BF18BF904F10C012A4628
:1047F000BDE838401BF13AB900B5002389B00293F7
:104800000393049305930693079317F039FC02A9C9
:1048100017F0E4F9A0B117F033FC00F55D7005ABBB
:1048200007C883E8070018463DF068F9F1EE047AFE
:1048300020EE270AFCEEC07ACDED017A9DF8040047
:1048400009B05DF804FB00001FB5184C94F802167F
:1048500004F2B44019F01AFE78B194F8021604F28A
:10486000B44019F0A5FF40B194F8021604F2B44028
:1048700004B0BDE8104019F0E7BF00230193029394
:10488000039317F0FDFB01A917F0A8F920B101A8C7
:104890003DF034F904B010BD2AF02AFBB02290F8A4
:1048A000F43202FB030090ED3B0AF3E7E8620030CC
:1048B00008B50D4BD3F82C0FA8B1443074F004F9AF
:1048C0000346B7EE001A9B2093ED000ADFED070ABE
:1048D00037F0D2F8DFED067A20EE270ABDEEC00AE7
:1048E00010EE103A18B208BDE88200300000000057
:1048F0000000C8422DE9F04FDFF8E0808DB004469B
:10490000354F042508F5804617F8019BB8F9843E19
:1049100009F1FF3A43FA0AF3D90746D594F828007B
:1049200075F0AAFF834694F8280076F091FF00F115
:1049300021039B4506D294F828000DB0BDE8F04F46
:1049400077F03CBCBAF1030F2FD8DFE80AF002354C
:104950003A3FD6F83C0A03689B68984700F1A003E9
:104960005A69D3F800A0D3F804E0D8681969D3F8DD
:1049700018C008925A6A1B6ACDF825206222CDF829
:104980002930212306900791C22194F82800CDF800
:104990000CA0CDF810E0CDF814C08DF82490CDE92E
:1049A0000032192303AA75F0E5FF013D15F0FF055C
:1049B000AAD10DB0BDE8F08FD6F83C0A0368DB68D9
:1049C000CBE7D6F83C0A03681B69C6E7D6F8443A39
:1049D00003F50573C4E700BFC4591808E862003046
:1049E00013B504460748019109F0FCFE30B901995E
:1049F000204602B0BDE8104077F036BD042002B07A
:104A000010BD00BFF0BA0030014809F08FBC00BFF4
:104A1000F0BA003037B5044609480D46D0F8903852
:104A2000DB0706D5114600F58E400192C2F0A6FBC9
:104A3000019A2946204603B0BDE830407CF0FEBB19
:104A4000E872003010B588B0044679F011F90C4BCB
:104A5000D3F82C0F38B90B4A0621204608B0BDE820
:104A6000104079F0EDB869461E22BFF091FC6B460C
:104A7000054A0621204679F0E3F808B010BD00BFD2
:104A8000E88200306C5818085DDD1A08034A92F875
:104A9000583B013382F8583B77F0BEBFE8820030C4
:104AA0000148BAF021BE00BFA0B7003007B50846E4
:104AB00001911FF079FC38B10448019902F04AFFD6
:104AC000002003B05DF804FB0420FAE794C700302F
:104AD000F7B58B8B06460C461746CD2B1DD1D1ED75
:104AE000067AFCEEE77ACDED017A9DF80430022BD0
:104AF00013D10E4D95F8511B05F6D82082F092FC8B
:104B000058B195F8511B05F6D82082F093FC20B9D6
:104B100094ED020A064802F0F9FE3A462146304674
:104B200003B0BDE8F04078F00DB800BFE8A2003057
:104B300094C70030162A10B40C4605D0542A03D06E
:104B40005DF8044B77F0ACBC0323012023705DF8C3
:104B5000044B7047074B10B540F6CD3493F90C2C3D
:104B600040F6CD13002A08BF1C4677F00BFF204308
:104B700010BD00BFE8A200301FB517F081FA04464F
:104B800068461FF075FA6946204616F07DFF0C4B0B
:104B900093F8F10E90B103F50053DDED017ADFEDEE
:104BA000096AD3F8443AB8EEE77AD3ED0D7AE7EE26
:104BB000267AFDEEE77A17EE903A18B204B010BDEF
:104BC000E88200300AD7233C10B5044620F0BAF83A
:104BD000204610BD10B50C4C94F8EB3E7BB9D4F8D0
:104BE000080F03685B6D984758B9D4F8080F03683D
:104BF0001B6D984700280CBF0220032010BD012028
:104C0000FCE70420FAE700BFE882003008B50E4B4D
:104C100093F8F10EB0B1D3F8080F03685B6E9847B4
:104C2000DFED0A7AB2EE047AB4EEE70AF1EE10FA9A
:104C300058BFB0EE670AC0EE077AFCEEE77A17EECF
:104C4000903A98B208BD00BFE882003000FF7F476D
:104C500010B44C69012C05D101465DF8044B0348A2
:104C600003F060BC5DF8044B77F0F2BEE832003030
:104C70002DE9F341B1F9043006460C461546002BE8
:104C800035DB1C4F4FF000089FED1B0A4FF47A7381
:104C9000CDE90028B1F90220D7F85C1B7CF040FE7A
:104CA00001239FED150A3046B4F90020D7F8601BA8
:104CB000CDE900534FF47A737CF032FE9FED0F0A7A
:104CC0004346B4F90420D7F8641B3046CDE90058B8
:104CD0007CF026FE9FED080A4FF47A73B4F90620A3
:104CE000D7F8681B3046CDE900587CF019FE02B0B9
:104CF000BDE8F081E88200300000FA4400007A4408
:104D00000C4B07B593F8F10E80B1D3F8080F036888
:104D10001B6E984736F012FEF6EE007A20EE270A58
:104D2000FCEEC07ACDED017A9DF8040003B05DF889
:104D300004FB00BFE88200307FB500230393049397
:104D4000059317F09DF903A916F048FFD8B117F0A5
:104D500097F9D0EDDD0A90EDDE0AF1EE600AB1EED2
:104D6000400A18F117F8DFED097A20EE270A36F02D
:104D7000E5FDF6EE007A20EE270AFCEEC07ACDEDD6
:104D8000017A9DF8040007B05DF804FBE02E65424F
:104D9000114B07B593F8F10ED0B103F50053D3F8DA
:104DA000440A00F546703CF0A9FEF1EE047A20EECC
:104DB000270ADFED0A7AB4EEE70AF1EE10FA58BFDF
:104DC000B0EE670AFCEEC07ACDED017A9DF80400E2
:104DD00003B05DF804FB00BFE882003000007F43B1
:104DE0000B4B93F8ED247AB9A3F5805213F8DF3C0E
:104DF0009B0609D192F8EB3E43B992F8F13E002BA5
:104E000014BF04200120704705207047032070471D
:104E1000E892003008B5074B93F9783E032B03D096
:104E2000BDE8084078F084BF034A022178F008FF0B
:104E3000042008BDE862003084581808094BD3F8F4
:104E40009028920701D477F01FBB03F54053DFEDA4
:104E5000067A03F5236393ED000AB8EEC00A20EE4C
:104E6000270A7047E87200300AD7233C10B594B087
:104E7000044603A81FF0FCF81D4B03A9D3F8080F44
:104E80000368DB6D984780B3002103A81FF0CEF9BB
:104E900058B394F82840C7F043FB059B9622DDEDFC
:104EA000047A57210893069BF8EEE77A9FED117A72
:104EB0000993002367EE877A07900B9320460C93A3
:104EC0000D930E930F931093119312934FF6F85383
:104ED000CDED0A7AADF84C3000238DF84E303323F7
:104EE000CDE9003207AA75F045FD14B010BD00BF32
:104EF000E88200300AD7233C684B30B505462DEDDB
:104F00000A8BD3F8080F91B003685B6A98470028B2
:104F100055D0634B1B68062B00F2AC80DFE803F032
:104F20000404045377924F005E4840F6F8540DF0A5
:104F3000FBF89FED5D8A90ED027B90ED00ABB0EE4B
:104F400048BAF7EEC79BB7EECAABB0EE489AF0EEA0
:104F500048AAF0EE48BAB0EE48CA90ED047BF7EEEE
:104F6000C78B95F82850C7F0DBFA00238C22B1EEEE
:104F7000687A03900D93B1EE499A0E930123B1EE36
:104F8000488A55218DF83E30332328468DED04AAFA
:104F9000CDED059A8DED067A8DED07CACDED08BAF7
:104FA0008DED099A8DED0ABACDED0BAA8DED0C8A27
:104FB000ADF83C40CDE9003203AA75F0DBFC11B03E
:104FC000BDEC0A8B30BD37484FF440640DF0ACF8AF
:104FD00090ED027B90ED00ABF7EEC79BB7EECAAB4E
:104FE00090ED047B2F48F7EEC78B0DF0A1F890ED04
:104FF00000CAD0ED01BA90ED029A2A480DF09CF853
:1050000090ED00BAD0ED01AA90ED028AA9E7DFED9C
:10501000268A40F6074423480DF08AF890ED00CA2E
:10502000D0ED01BAF0EE689A90ED029AB0EE68AA5F
:105030001C480DF081F890ED00BAD0ED01AA90ED7A
:10504000028A8EE79FED189A40F63F4415480DF00E
:1050500073F8F0EE49BAB0EE49CA90ED00BAF0EE3E
:10506000498AD0ED01AAF0EE499A90ED028AB0EE9D
:1050700049AA76E79FED0C8A0024F0EE48AAB0EE2C
:1050800048BAB0EE489AF0EE48BAB0EE48CAF0EE30
:10509000488AF0EE489AB0EE48AA62E7E88200300B
:1050A000A0C8003060C1003000000000324A2DE985
:1050B000F0412DED048B92F8F13E8AB0002B55D0D3
:1050C00002F500579FED2D7AD2F8086FD7F83C3AD9
:1050D00090F828803046D3ED1D7A93ED1B9A67EE49
:1050E000877AD3ED1C8A29EE079A68EE878AFDEE4F
:1050F000E77A17EE903A1CB233681B6E9847BDEE04
:10510000C00A304610EE103A1DB233685B6E984705
:10511000DFED1B7AB0EE408AD7F8443AB4EEE70AE6
:1051200030465F6B3368F1EE10FA9B6E58BFB0EEFD
:10513000678A98470023B7223E214046BCEEC88AC2
:1051400006938DED039ACDED048A18EE103A05977B
:105150008DED070AADF824301A23ADF82040ADF8E4
:105160002250CDE9003203AA75F004FC0AB0BDEC70
:10517000048BBDE8F08100BFE8820030E02E65427C
:1051800000FF7F47584B2DE9F047A3F17402A6B00A
:1051900089460646109203F65C0218251192A3F187
:1051A0003802129203F5AE62139203F5E062149294
:1051B00003F5CE62159203F2BC62169203F2D4722A
:1051C000179203F2AC52189203F2E452199203F5CB
:1051D00052721A9203F23C721B9203F5A6621C9261
:1051E00003F698121D9203F516621E9203F6E4125E
:1051F0001F9203F52262209203F23462229203F698
:105200009832239203F543622592384AD2F86C17FC
:10521000D2F87C2A219124920522CDE90E3303F5A0
:10522000D56353F8041B09B10135EDB2013A12F010
:10523000FF02F6D109F1FF37FFB2BD4234D9172F73
:1052400036D826AB03EB870353F8608CD8F80030D0
:1052500040469B6C9847D8F80030044640461B688F
:105260009847002F39D0012F214B04BF03201C4643
:105270000023029096F82860232221460DF11300A6
:1052800003938DF810508DF811908DF812303CBBBF
:105290001AF136FC86222E2340F2B3113046CDE9B6
:1052A000003202AA75F066FB284626B0BDE8F087FA
:1052B000A9F1190842F2AC33DFF83CA053FA88F8A0
:1052C0005AF828000028EFD003689B6C98470446E2
:1052D0005AF8280003681B68C2E71B20054CC7E783
:1052E0001BF13EFBD6E700BFF0BA0030E882003089
:1052F000C1321A08A8581808E83200301D4B2DE9B1
:10530000F04F2DED028BD3F83C3A8DB090F8284049
:10531000D3F88480D3F88870D3F88C60D3F8905099
:1053200093ED258AD3F898B0D3F89CA0D3F8DC90FD
:10533000C7F0F6F800231622029053218DF82C3086
:10534000252320468DED078ACDF820B0CDF824A086
:10535000CDF82890CDF80C80049705960695CDE9F8
:10536000003202AA75F006FB0DB0BDEC028BBDE861
:10537000F08F00BFE8A2003070B58A7A06464B7AFB
:105380000C4643EA0223CA7A43EA02439D2B21D109
:10539000134D95F8511B05F6D82082F043F8C8B19B
:1053A00095F8511B05F6D82082F050F8022811D14B
:1053B00095F8511B05F6D82082F03CF850B9D4ED91
:1053C000057A9FED080AF8EEE77A074827EE800A8B
:1053D00002F09CFA21463046BDE8704077F01CBAD6
:1053E000E8A200300AD7233C94C70030054BD3F81D
:1053F0002C3F2BB193F8CA00002808BF0220704749
:1054000002207047E882003008B5034BD3F8080F3C
:1054100003681B68984708BDE8820030014B93F889
:10542000F10E7047E882003070B52C4E05460C46F0
:10543000D6F8080F2DED028B036886B091ED018A36
:105440005B6A984750B9BDEEC88A18EE103ADB0780
:1054500004D4022006B0BDEC028B70BDD4E9040177
:1054600037F028FE0028F4D002A81EF001FE02AAA0
:10547000214628467CF04CF90028EAD0184902A8B9
:105480001EF09EFF03460028E3D1DFED160A024618
:10549000009002A9B0EE600A13480CF0DDFBD8B111
:1054A000D6F8080F03685B6A9847044608B10020E5
:1054B000D0E7022204210D4806F062F860B1DFED6A
:1054C000090A2346224602A9B0EE600A0648009463
:1054D0000CF0C2FB0028EAD10420BBE7E8820030D0
:1054E00014AD00300000000060C10030E832003030
:1054F00008B591F820200B46032A18D1D1ED027A85
:105500009FED0C7AF0EEE77A93ED060A0A4BF4EE83
:10551000C77AD3F8080FF1EE10FA4CBF0121002131
:1055200013F054FF002814BF0020042008BD0220FF
:10553000FCE700BF00000034E882003010B52DED1C
:10554000028BD1ED007A82B00C46F5EEC07AF1EE16
:1055500010FA04DA042002B0BDEC028B10BD9FEDFE
:105560001C7AF4EEC77AF1EE10FAF3D891ED030A43
:105570009FED188AF0EEC07AF4EEC87AF1EE10FAD8
:105580001FD5D4ED037AD4ED010AF4EEC87AD4ED38
:10559000027A94ED000AFDEEE77A0F48F1EE10FA78
:1055A000CDED017ADFED0D7AACBF012200229DF92D
:1055B000041060EEA70A20EE270A02F01DF9002071
:1055C000C9E7F7EE000A36F013F90028C2D0D8E791
:1055D0000000B4430000003494C7003035FA8E3C1C
:1055E00091ED010ADFED197AB4EEE70A07B5F1EEA5
:1055F00010FA29DBD1ED007AFCEEE77ACDED017AE5
:105600009DF80430042B04D8DFE803F007071218D4
:105610001E00042003B05DF804FB0D4BD3F8080F07
:105620000368DB6E9847002814BF00200420F1E7D0
:10563000074BD3F8080F03681B6FF3E7044BD3F84D
:10564000080F03685B6FEDE70220E3E7000000341A
:10565000E882003008B5D1ED007A9FED157AF0EEC2
:10566000E77AF4EEC77AF1EE10FA1DD5D1ED017AA2
:10567000F0EEE77AF4EEC77AF1EE10FA14D50222D2
:1056800003210C4805F07CFF80B10A480121FDF799
:1056900055F9094890F84438012B03D000F504600F
:1056A0003FF038FE002000E0022008BD0420FCE7A7
:1056B00000000034E8320030E8B2003010B5D1ED1F
:1056C000007AFCEEE77A17EE903A9CB2012C02D0F9
:1056D000022C06D04CB9214605488BF0C1FC0020B5
:1056E00010BD044803F0CEFCF9E70420F8E700BF42
:1056F000B0AE0030E83200301FB5D1ED017A0B7C3E
:10570000FCEEE77ACDED027AD1ED007A0093FCEE63
:10571000E77AD1ED030A91ED020A01469DF80830BF
:10572000CDED037A9DF80C20024812F03FF805B049
:105730005DF804FBE832003010B50A4C94F8213FC4
:10574000DB070CD402220521A4F5A04005F018FFC8
:1057500028B90222A4F5A040114605F011FF00204F
:1057600010BD00BFE882003010B5D1ED007A0446CC
:10577000FCEEE77A17EE903A13F0FF0310D1104BCE
:10578000D3F8080F0368D3F88430984708B1002095
:1057900010BD0C4A2046062178F052FA0420F7E7A3
:1057A000012B0AD1064BD3F8080F0368D3F88830D1
:1057B00098470028EBD1044AECE70220E8E700BF55
:1057C000E8820030B4581808C458180801F10C03D6
:1057D0009FED0A7AF1EC017AF4EE677AF1EE10FAB5
:1057E0000AD6F0EEE77AF4EEC77AF1EE10FA03DCAF
:1057F0009942EFD1012070470020704700007A44A1
:1058000030B5002305462DED028B8DB00393049334
:10581000059316F035FC03A916F0E0F960B316F015
:105820002FFC00F55D7306AC95F8285093E807004F
:1058300084E80700DDED060A9DED070AF1EE600A37
:10584000B1EE400A17F1A6FA2046B0EE408A3CF0CD
:1058500055F9089B0122DFED0A7AA8210B930C234E
:1058600028EE278A28468DED0A0ACDE9003209AADA
:105870008DED098A75F07EF80DB0BDEC028B30BD60
:10588000E02E65422829F7B505460E4641D00AD8D4
:1058900024294AD027292DD03146284603B0BDE817
:1058A000F0407CF0DDBA4029F6D1262176F098FC54
:1058B000044620B395F828102148A3F075FA214B2F
:1058C0001F68EFB12621284676F08AFC0446B8B15D
:1058D00000230DF1060231462846ADF806307DF072
:1058E00029FA68B1BDF80620384695F828109AF0D4
:1058F000F9FF05E0122176F073FC044618B9002484
:10590000204603B0F0BD95F828100F486CF08CFFCE
:10591000F6E7162176F064FC04460028EFD095F8EF
:10592000281009486DF05AF8EAE70C2176F058FC87
:1059300004460028E3D02846FFF762FFE0E700BFF7
:10594000B8B8003010D70030F4AE003038B5164C7F
:105950000D4694F8213FDB070AD4D4F82C3F93F886
:10596000D5303BB9012204F628401146FCF740FE31
:10597000002038BD94F8EB3E022273B10521A4F556
:10598000A04005F0FDFD0028F2D0012195ED000AB0
:10599000D4F8080F13F01AFDEAE70921A4F5A04096
:1059A00005F0EEFDE4E700BFE882003010B5204CC2
:1059B00094F8213FDB070DD4D4F82C3F93F8D53071
:1059C00043B194F8EB3E3BB10122082104F6284094
:1059D000FCF7CCFE002010BDD1ED007A9FED157ACA
:1059E000F0EEE77AF4EEC77AF1EE10FA0BD5022268
:1059F0001121114805F0C4FDA0B902220E4811463C
:105A000005F0BEFDE6E7D4F8080F03681B68984769
:105A10000428DFD0D4F8080F03681B6898471428BF
:105A2000E5D1D7E740F6C411044809F071FDD1E78C
:105A3000E882003000000034E832003020C000303E
:105A400070B58B8B05460C46C12B3CD8BB2B0CD8B4
:105A5000542B6AD02ED8113B99B2052918D921466A
:105A60002846BDE870407DF021BDBC3B052BF6D833
:105A700001A151F823F000BF655B0608735B0608BF
:105A80005F5A06085F5A06080F5B0608195B06088E
:105A9000052BE4D801A151F823F000BF4F5B0608A5
:105AA0005F5A06085F5A06085F5B0608C15A060877
:105AB0002B5B0608732B22D0B22B24D0552BCED1D2
:105AC0000222092145E04AF21146B34237D00AD8F2
:105AD000D12B26D0B3F5967F35D0D02BBFD1BDE8E2
:105AE0007040FFF7EBBD4AF21246B34223D04AF2B0
:105AF0001346B342B3D1BDE87040FFF757BFBDE8CE
:105B00007040FFF71BBDBDE87040FFF769BD21463F
:105B1000BDE87040FFF788BC2146BDE87040FFF744
:105B200023BEBDE87040FFF7E7BD21462846BDE82B
:105B30007040FFF7DDBCBDE87040FFF707BFBDE870
:105B40007040FFF7F9BDBDE87040FFF783BD02224A
:105B500005210A4805F014FD48B9042070BD022251
:105B60000621F6E70221064806F0FAFFF4E70020D6
:105B7000F4E70221024806F0BFFFEDE7E83200300B
:105B8000F0BA0030F6EE007A08B591ED007AB4EE86
:105B9000E77AF1EE10FA06DD012205210348FCF751
:105BA000E5FD002008BD0420FCE700BF108F003099
:105BB00030B52DED028BCD7893B00C462722272DE2
:105BC0004FF0000108A828BF272519F199FF04F11B
:105BD0000C0108A82A4619F149FF464BD3F8080FD3
:105BE00003685B6A984748B19DF846509DF9463076
:105BF000690607D5012140480BF052FD13B0BDECFA
:105C0000028B30BD00244FF07E52002B049207948B
:105C10000694059427DA04A839F09AFFEA0705F0FC
:105C200006030194029403942BD4002BE2D10D9B24
:105C300001930E9B02930F9B03932F480BF0AEFD35
:105C40009DED100A0446F8B1B7EE001A40F2F330A9
:105C5000FFEE000A35F010FF234601AA04A92648EA
:105C60000BF0A4FDCAE7099B04A804930A9B0593C3
:105C70000B9B06930C9B079339F070FF0028CDD146
:105C8000B8E7062BB6D1D8E7DFED1C0AB7EE001A4D
:105C900040F2F63035F0F0FEF6EE000AB0EE408A43
:105CA00035F0A6FD18BBB6EE007A154BDFED156A90
:105CB000D3F8483AB4EEC78AF1EE10FA0ADD38EEAE
:105CC000478A93ED060A20EE260A38EE088A28EE67
:105CD000000AC1E7D3ED077A37EE488A67EEA67A65
:105CE00038EE088AF0EEE77A27EEC80AB4E79FEDAF
:105CF000030AB1E7E882003060C100300000000014
:105D0000E8A200300AD7233C2DE9F0472DED028BA5
:105D1000A2B08246084614A9FEF75AFD8A4BD3F872
:105D2000080F03685B6A984750B19DF88420012AE8
:105D30000BD0D31F022B08D9012184480BF0B0FCF3
:105D400022B0BDEC028BBDE8F087BDF8803003F0D7
:105D5000070703F0380803F4E07603F4806503F4E2
:105D600000649B0501D5002EE6D09FED758B8DED6F
:105D7000088B8DED0A8B8DED0C8B002F3CD19DEDAA
:105D8000177A083A9DED166AB1EE477A9DED155ADD
:105D9000B7EEC66A012AB7EEC55AB7EEC77A8DEDDF
:105DA000085B8DED0A6B8DED0C7B07D808A9684860
:105DB00016F0C0FB8DED080B8DED0A1B9DF88430AD
:105DC000073B022B18D88DED0E8B8DED108B8DEDD2
:105DD000128B16F055F90EA914F09CFE0028ABD0DA
:105DE0000EA908A83BF00CF99DED0C7B9DED126B04
:105DF00037EE467B8DED0C7B4FF00009CDF814900B
:105E0000CDF81890CDF81C90B8F1000F1CD1DDED45
:105E10001A7A05A9189B5046F1EE677A0593199BEB
:105E2000CDED077A0693FFF7D1FC002884D09DF8CA
:105E30008430083B012B07D805A9454816F066FBBE
:105E40008DED050ACDED060ACDF83890CDF83C90E1
:105E5000CDF84090B6B91B9BDDED1D7A0E931C9BCF
:105E6000F1EE677A0F939DF88430CDED107A083B00
:105E7000012B07D80EA9364816F048FB8DED0E0A07
:105E8000CDED0F0AFDB99DF884309DED1E0A083B4B
:105E9000012B8CBF00230123CCB9DDED1F0ACFB944
:105EA000B8F1000F3AD1B4FA84F4B5FA85F502934B
:105EB00005AA64090EAB6D0908A901940095234851
:105EC0000BF06AFD3CE700239FED220AE4E7DFEDDB
:105ED000210AE4E7B8F1000F0FD10122B4FA84F4EB
:105EE00005A91A486409CDE90132B5FA85F30EAA6D
:105EF00000945B090CF014F822E7002E7FF41CAF2D
:105F000001220EA91148CDE90032B4FA84F3B5FAA2
:105F100085F25B0952090BF0A1FF11E7002E3FF457
:105F20000BAFB5FA85F208A908485209CDE9003748
:105F3000B4FA84F35B090BF0BDFD01E7AFF3008019
:105F40000000000000000000E882003060C1003066
:105F5000804F0030000000002DE9F047A4B08246D9
:105F6000084616A9FEF734FC704BD3F8080F0368F7
:105F70005B6A984760B1BDF88840A30504F0070844
:105F800004F4E07707D537B9012169480BF088FBA5
:105F900024B0BDE8F0870CAE30461EF069F8B8F1C9
:105FA000000F23D1DDE9170137F084F80028EBD08A
:105FB00009AA9DF88C1050467BF094FB0028E3D092
:105FC000DDED197A10AD9FED5B7A099B284667EEEF
:105FD000877A0093FDEEE77ADDE9171217EE903A23
:105FE0001EF064F895E80F0086E80F00002214F018
:105FF00038090692079208920FD1DDED1C7A06A9A6
:106000001A9B5046F1EE677A06931B9BCDED087AFA
:106010000793FFF7DBFB0028B6D009920A920B9298
:106020004FB9DDED1F7A1D9BF1EE677A09931E9B38
:10603000CDED0B7A0A9314F480650CBF9DED200A18
:106040009FED3D0A14F400640CBFDDED210ADFED85
:106050003A0AB8F1000F35D1B9F1000F56D13046E8
:10606000CDED050A8DED040A1EF046F803289DEDDE
:10607000040ADDED050A87D00022002310A930466E
:10608000CDED050A8DED040ACDE91023CDE91223EB
:10609000CDE914231EF0F0FA00283FF475AFB4FAEE
:1060A00084F4B5FA85F3DDED050A06AA64099DEDD1
:1060B000040A5B0910A9CDF8049000941C480BF069
:1060C000E7FC65E7B9F1000F0FD10123B4FA84F4BE
:1060D00009AA06A964091648CDE90193B5FA85F322
:1060E00000945B090BF01CFF52E7002F7FF44CAFCC
:1060F0000123B5FA85F209A90D485209CDE90073CB
:10610000B4FA84F35B090BF0A9FE41E7002F3FF4DA
:106110003BAFB4FA84F3B5FA85F23146CDF800808E
:106120005B09034852090BF097FD31E7E882003024
:1061300060C100300000C8420000000030B48D7A19
:1061400004464B7A0A4643EA0523CD7A43EA0543DF
:10615000562B1CD008D8522B13D0542B14D02046C9
:10616000114630BC7CF0E0B903F18073863B23F02C
:106170007F43012BF3D890F82810064830BC6CF010
:10618000F9BC30BCFFF714BD30BCFFF7BDBD30BC5F
:10619000FFF7E2BEF4AE0030F0B5044600F5F8407B
:1061A000002301220C302DED028B91B06946009343
:1061B0006DF0A2FA08B94F4B009304F5A04704F51F
:1061C000E045D7F8080F03685B699847002840F05E
:1061D0008B80D5F8443A93EDBE7B93EDC88AF7EEF9
:1061E000C78B04F5B84601A91436304612F088FC76
:1061F00018B970F019FA3F4B01933722002102A819
:1062000019F17EFCA3238DF8083095238DF8093011
:10621000C6F08EF9D5F83C3ACDF80B00D7F82C0F24
:10622000D3F8DC20D3F8E0304430CDF80F10CDF8AF
:106230001320CDF8173072F047FC0346B7EE001A72
:10624000DFED2D0A9B2093ED000A35F015FCD7F801
:106250002C0F10EE103ACDF81B3003685B6998479D
:1062600010EE103A3046CDF81F3018EE903ACDF8C7
:106270002330D5F8443A93EDB27BB7EEC77B17EEE7
:10628000103ACDF8273005F608231B68CDF82B30DF
:10629000019BCDF82F3012F04FFC9FED187A10EED5
:1062A000103A372202A928EE078ACDF83330009B36
:1062B00004F59B50BDEEC88ACDF8373018EE103A81
:1062C000ADF83B30D5F8443AD3EDC27A67EE877A21
:1062D000FDEEE77A17EE903AADF83D306FF0DEFA5A
:1062E00011B0BDEC028BF0BD9FED038AF0EE488A41
:1062F00077E700BF2292CA7F000000000000C8427A
:1063000000F5E040D0F83C0AB3F01CB900F5E040DD
:10631000D0F8441AD0F83C0AB3F07AB970B54FF40B
:106320008051044612F042FD00284ED004F5E046AC
:1063300004F59B55D6F83C0A03689B68984767218B
:1063400000F1A00228466FF049F9D6F83C0A03682C
:10635000DB689847682100F1A00228466FF03EF9FB
:10636000D6F83C0A03681B699847692100F1A0022E
:1063700028466FF033F9D6F8442A6A21284602F5F8
:1063800005726FF02BF92021204612F00FFDE0B1CD
:1063900004F5A043D3F8080F03681B69984778B148
:1063A000D6F8442A28466C2188326FF017F9D6F8BF
:1063B000442A28466D21B432BDE870406FF00EB912
:1063C00020460CF023FC0028EAD170BD08B515F07A
:1063D00057FEBDE8084015F02DBB00007FB50E4606
:1063E0004FF6FF710446154612F0E0FCE0B11022B2
:1063F0000021684619F184FBA3238DF80030952312
:106400008DF8013003238DF80230C6F091F8102288
:10641000CDF80300CDF8071004F59B5069468DF8C0
:106420000B6003956FF0BAFA04B070BD7FB50E46ED
:106430004FF6FF710446154612F0B8FCE0B1102289
:106440000021684619F15CFBA3238DF800309523E9
:106450008DF8013004238DF80230C6F069F810225F
:10646000CDF80300CDF8071004F59B5069468DF870
:106470000B6003956FF092FA04B070BD30B52DED4E
:10648000048B89B004460D461C22002101A8F0EEC1
:10649000409AB0EE609AF0EE418AB0EE618A19F14E
:1064A0002FFBA3238DF8043095238DF805300623A8
:1064B0008DF80630C6F03CF81C22CDF80700CDF868
:1064C0000B1004F59B5001A98DF80F50CDED049AE7
:1064D0008DED059ACDED068A8DED078A6FF0DEF918
:1064E00009B0BDEC048B30BD10B54FF480110446EB
:1064F00012F05CFC30B104F5E450BDE810401830F7
:1065000013F0C2BE10BD00002DE9F04F2DED028B3F
:106510008DB080462F2200216846F0EE408AB0EE12
:10652000608A11EE10BA11EE90AA12EE109A12EED5
:10653000907A13EE106A13EE905A14EE104A19F185
:10654000DFFAA3238DF8003095238DF8013009235D
:106550008DF80230C5F0ECFF18EE903ACDF803004C
:10656000CDF807102F22CDF80B30694618EE103AFF
:1065700008F59B50CDF813B0CDF80F30CDF817A02B
:10658000CDF81B90CDF81F70CDF82360CDF82750C3
:10659000CDF82B406FF082F90DB0BDEC028BBDE859
:1065A000F08F000030B52DED088B8BB004460D4602
:1065B000282200216846B0EE40BAF0EE60AAB0EEA4
:1065C00041AAF0EE619AB0EE429AF0EE628AB0EE25
:1065D000438A19F195FAA3238DF8003095238DF89D
:1065E00001300A238DF80230C5F0A2FF2822CDF831
:1065F0000300CDF8071004F59B5069468DF80B5049
:106600008DED03BACDED04AA8DED05AACDED069A68
:106610008DED079ACDED088A8DED098A6FF03EF970
:106620000BB0BDEC088B30BD2DE9F0438FB01446A4
:10663000054689463122002101A89846DDE91676F3
:1066400019F15EFAA3238DF8043095238DF80530F7
:1066500008238DF80630C5F06BFF3B683122CDF87A
:10666000070005F59B50CDF81D307B68CDF80B1069
:1066700001A9CDF82130BB688DF80F90CDF82530F9
:1066800033688DF81C80CDF82930736894ED007B59
:10669000CDF82D30B368B7EEC77BCDF831308DED36
:1066A000047A94ED027BB7EEC77B8DED057A94ED0D
:1066B000047BB7EEC77B8DED067A6FF0EFF80FB075
:1066C000BDE8F08370B52DED068B8CB01446054601
:1066D0000E462C22002101A8B0EE409AF0EE608A0E
:1066E000B0EE418AB0EE61AAF0EE429A19F108FAD2
:1066F000A3238DF8043095238DF805300B238DF8F6
:106700000630C5F015FFDFED1A7A2C2294ED007AE1
:1067100029EE279ACDF8070027EE277ACDF80B103F
:1067200068EEA78A01A928EE278A05F59B508DED12
:10673000077A94ED017A8DF80F6027EE277A8DEDB8
:10674000049ACDED058A8DED068A8DED087A94EDDB
:10675000027A8DED0AAA67EE277ACDED0B9ACDED80
:10676000097A6FF09BF80CB0BDEC068B70BD00BFD2
:10677000E02E65422DE9F04188B080461B220021C1
:1067800001A810EE107A10EE906A11EE105A11EE78
:10679000904A19F1B5F9A3238DF8043095238DF8AB
:1067A00005300C238DF80630C5F0C2FE1B22CDF853
:1067B0000700CDF80B1008F59B5001A9CDF80F701C
:1067C000CDF81360CDF81750CDF81B406FF066F888
:1067D00008B0BDE8F0810000AD20704730B5044638
:1067E00089B0144B1E2204F59B556946D3F82C0F33
:1067F000BDF0CEFD6A46104928466FF0EBF904F56E
:10680000A043D3F8080F03681B68984704F540536A
:106810000146284693F8382C6FF000FA04F5E4504E
:10682000183015F09FFE04F5907027F091FA09B02A
:1068300030BD00BFE88200305DDD1A08F8B51123D5
:10684000424A04464C3000F8483C40F68425404B10
:1068500040F6845640F8142C4FF0804240F8443CF7
:10686000002340F8102C40F8343C40F8303C40F80D
:106870002C3C40F80C3C374B374F40F8083C374B2A
:1068800040F8043C90F0EEF804F6F4107DF0B0FB14
:10689000334BC4F8F43960197DF072FE675130351E
:1068A000B542F8D104F6885004F580567FF098FD83
:1068B00004F5C05000212B4D1030C1F043F804F511
:1068C000C650C6F8C4580830B1F0DAFDA5F5E96342
:1068D00004F5D050C6F8103A1C3096F0CBFAA5F566
:1068E0000C7304F5DF50D035C6F8D43B9FED1E1A6B
:1068F0000430DFED1E0A9FED1E0AC6F8E05BB3F020
:10690000EDFD9FED191A04F5DF509FED1A0AF0EE28
:10691000410A1C30B3F0E2FD9FED131A04F5E0507C
:106920009FED140AF0EE410A1430B3F0D7FD04F5E0
:10693000E3500430B8F0D2F920460F4963F0C8FBA9
:1069400020460E4963F0C4FB2046F8BD0000C84154
:10695000504200300AD7233CF8A618080000E04057
:106960000CA71808B8C50030000000009A99993E9D
:106970000000B44300804A43F4981808B49B1808F8
:1069800000F57851782230B5044693B02C310125BA
:106990006DF09CF804F57850B7EE000A0022022151
:1069A0003C3062F09FFF002304F567512D4A4520DB
:1069B0002431CDE9005362F0F1FE04F56F5100235C
:1069C000FA201431284ACDE9005562F0E7FE274944
:1069D0000B68D8070DD404F55852254B0D601832BA
:1069E0001A6004F56C522832DA6004F5A0521832AD
:1069F0009A6104F57A5003221D490125283062F07E
:106A00003BFF00231B4A04F59B51FD20CDE90053B9
:106A100062F0C4FE184B1A68D20705D404F5D854A6
:106A2000164A1D601C341460154D0121134802AC38
:106A300062F03EFF0FCD0FC40FCD0FC40FCD0FC4BA
:106A400095E80F0084E80F000022042102A862F0FC
:106A5000A1FE63F02FFD0B4A138843F0010313805E
:106A600013B030BDB81E1A08F4BC19088CC700302A
:106A7000C4250030588F190890C70030E825003031
:106A8000E040180838CA003070B52A4CA4B0064659
:106A9000B7EE000A6D4694E80F0085E80F0000216C
:106AA000284662F0CDFD96F91C6BD6B910340CADBA
:106AB0000FCC0FC50FCC0FC50FCC0FC594E80F003E
:106AC00085E80F00324604210CA862F063FE9FEDBA
:106AD0001A0A1A4863F090FEB7EE000A184863F0ED
:106AE0008BFE184C04AD9FED180A0FCC0FC594E82F
:106AF0000F0085E80F00002104A862F0A1FD00212D
:106B00009FED110A284662F09BFD04F1100100245C
:106B100060220CA818F1AAFF0CABB7EE000A002106
:106B20001819103462F08CFD602CF5D17FF0C4F997
:106B300024B070BD2041180800000000D498180847
:106B4000E3981808704118080000344238B5002452
:106B5000054D28191034B7EE000A002162F070FDCF
:106B6000D02CF6D138BD00BFC4A318080F299DBF93
:106B7000302303FB0100903000207047014B93F954
:106B80006F0E7047E8620030024B93F8210F00F05F
:106B900001007047E8820030044BB3F8343EDB0755
:106BA0005ABF0069C0F3401000207047E86200300F
:106BB000014BD3F8680B7047E882003008B50368D2
:106BC0009B68984730B9044B93F9200FB0FA80F0D6
:106BD000400908BD0020FCE7E882003038B50C1EF3
:106BE0002EDB184DE3B295F8782B9A4228D3D5F8CE
:106BF000743B0122A5F5A040195D04F0C1FCF8B179
:106C00007DF0E8FB03217EF0B5FEC8B97DF0E2FB24
:106C10000D217EF0AFFE98B9A5F50052A5F5A04074
:106C200092F9543EE340DB0756BF92F96E1E0221F3
:106C3000E140BDE8384058BF01F00101FBF790BECC
:106C400038BD00BFE8820030022910B5044606D1E5
:106C5000014635220948BDE8104004F091BC084BBC
:106C6000D3F8080F03681B689847844205D17DF06C
:106C7000B1FBBDE810407DF09BBA10BDE83200309A
:106C8000E882003029B1022907D1044BC3F8001F64
:106C90007047024B0122C3F8002F7047E882003092
:106CA00031B1022907D1044B012283F8042F704728
:106CB000014B83F8041F7047E882003010B52DEDBA
:106CC000048B90F890330446F3B19FED1B8A0023A8
:106CD000F0EE488A80F8903315F0D2F9F0EE480AC9
:106CE000B0EE680A012115F055FA6FF09DFC2621DF
:106CF0006FF0D6FB7AF072FF104A0621BDEC048BD0
:106D0000BDE8104075F00AB87DF0B2FAB0F90A306B
:106D100020469FED0B9A08EE903A7DF0B3FAB0F959
:106D20000A30F8EEE88A08EE103AB8EEC88A68EE43
:106D3000898A28EE098ACFE70000000094A4180889
:106D4000D402373910B50446E1B1022919D1124BEA
:106D5000D3F8080F03681B6B984738B97AF03EFFE9
:106D60000E4A0621BDE8104074F0D8BF7AF036FF15
:106D70000B4A062174F0D2FF01230A4A84F89033AB
:106D8000137210BD90F89033002BFAD0054B197296
:106D9000BDE81040FFF792BFE8820030A0A41808B9
:106DA000C2A418089DC9003008B50023054A80F820
:106DB000903313727AF012FF034A0621BDE80840AF
:106DC00074F0ACBF9DC90030D4A4180873B590F816
:106DD00090330546A3B31B4CD4F8080F03681B6B14
:106DE000984728B9284602B0BDE87040FFF7DCBFDD
:106DF00094F8F26E36B17AF0F1FE134A042174F081
:106E00008DFFEFE704F50054F3EE047AD4F83C3A32
:106E100093ED1B7A87EE270A93ED1C7AC7EE270ABB
:106E20008DED010ACDED000A15F02AF93146DDEDB0
:106E3000000A9DED010A02B0BDE8704015F0AAB944
:106E400002B070BDE8820030E8A418086D2913B5BF
:106E500000F3EE8001290DDC02B0BDE810407EF0A9
:106E600071BBA1F1B2040123A34013F0150FF3D0BD
:106E700002B010BD8B1E6B2BEED801A454F823F08A
:106E8000716E060887700608716E0608716E060836
:106E9000596E0608716E0608596E0608596E060886
:106EA00087700608596E0608716E06088770060816
:106EB00087700608596E0608716E0608716E06081E
:106EC000716E0608596E0608596E06088770060826
:106ED000716E060887700608596E060887700608E6
:106EE00087700608596E0608596E0608596E06081E
:106EF000596E0608596E060887700608716E0608F6
:106F0000596E0608596E0608596E0608716E060815
:106F1000596E060887700608596E0608596E0608ED
:106F2000716E060887700608596E0608596E0608C5
:106F3000596E0608716E0608716E0608716E0608B5
:106F4000596E0608596E0608716E0608596E0608D5
:106F5000596E0608716E0608716E0608716E060895
:106F6000596E0608596E0608716E0608716E06089D
:106F7000596E0608596E0608596E0608596E0608BD
:106F8000596E0608596E0608716E0608716E06087D
:106F9000716E0608716E0608716E0608716E06083D
:106FA000596E06088770060887700608596E06082D
:106FB000596E0608596E0608596E0608596E06087D
:106FC000596E0608716E060887700608596E060825
:106FD000596E0608596E0608596E0608596E06085D
:106FE000596E0608596E0608596E0608596E06084D
:106FF000596E0608596E0608596E0608596E06083D
:10700000596E0608716E0608596E0608596E060814
:10701000596E0608596E0608596E0608596E06081C
:10702000596E0608596E0608596E060887700608DC
:10703000B62923DCB1293FF714AFA1F197030A2B3E
:107040003FF60AAF0A2B3FF607AF01A454F823F02E
:10705000716E0608716E0608596E0608716E060894
:10706000596E0608596E0608596E0608596E0608CC
:107070008770060887700608716E0608A1F1DB03A9
:10708000012B3FF6E9AE8379009300237EF018FAD6
:10709000EEE600BF70B50B688AB00C46632B00F3B8
:1070A000D380012B05DC21460AB0BDE870407DF09D
:1070B000E9BE023B612BF6D801A252F823F000BFD3
:1070C000B3720608C5720608E5720608EF72060874
:1070D000A770060821730608A7700608A77006089F
:1070E000D9730608A7700608A7700608D5720608A7
:1070F000FF730608A7700608D37306083D740608D8
:1071000043740608A7700608A77006085B74060893
:107110006B7406087B740608A7700608A37406083B
:10712000B7740608A7700608A7700608A7700608B7
:10713000A7700608A7700608CB740608DF74060857
:10714000A7700608A7700608A7700608E574060869
:10715000A7700608EB740608A7700608A770060853
:1071600007750608A7700608A7700608A770060826
:10717000A7700608A7700608A7700608A77006087B
:10718000A7700608A77006088B750608A770060882
:10719000A7700608497406084F7406085574060857
:1071A000A7700608A77006080D750608137506086F
:1071B000A7700608A7700608A7700608A77006083B
:1071C000A7700608A7700608797506087F75060877
:1071D0008575060891750608977506089D75060859
:1071E000A7700608E3750608A3750608A7700608C9
:1071F000A7700608A7700608A7700608A7700608FB
:10720000A77006084776060867760608A77006087E
:10721000A7700608A7700608A7700608A7700608DA
:10722000A7700608A7700608A7700608A7700608CA
:10723000A7700608A7700608A7700608A7700608BA
:10724000A77006087D760608A02B1DDC962B7FF71D
:107250002AAF973B092B3FF626AF01A252F823F045
:107260008376060893760608A7700608A9760608AE
:10727000A7700608A7700608A7700608A77006087A
:1072800075760608C7760608B62B00F0FD810ADC85
:10729000B22B00F0BA81B42B7FF405AF0979AA486C
:1072A000C1F07AFA03E0DB3B012B3FF6FCAE012490
:1072B00033E00B79022BFAD135220E21A34804F0DA
:1072C0005FF9F4E70979003918BF01219F48FBF7FE
:1072D00047FBECE709790129F8D0022914BF002106
:1072E0000221F3E709790620FFF7AEFCDFE70B790F
:1072F000022BDCD1964DD5F8080F0368DB6A98475E
:1073000004460028D3D0D5F8643BB3F90A30002BEB
:10731000CDD1A5F26470FFF7D1FC20460AB070BD54
:107320000B79022BC3D18A4D8A4BD5F8082F9A428C
:10733000BDD0D5F82C3F93F8D530002BB7D005F54C
:107340004054B4F97438012B05DCD5F8643BB3F92B
:107350000A30002BABD005AE1C22002103A818F187
:10736000CFFB30461CF084FEB4F974387A4C012B04
:1073700013DC162303A904F5C250ADF80E30D4F87F
:10738000303A642BB8BF642306933BF019FA20B15E
:107390006FF04AF927216FF083F804F62C230FCB06
:1073A00086E80F00D5F8643B03A96C48B3F90A30AE
:1073B000002BCCBF10231523ADF80E303BF000FAA4
:1073C00000283FF474AF6FF02FF927216FF068F8B1
:1073D0006DE70979032087E70B795D4D022B03D018
:1073E000002385F87C3B62E719215D4864F0DAFBF5
:1073F00004460028F4D0012385F87C3B8DE70C7906
:10740000012C0BD0022C12D0002C7FF450AF554B26
:1074100083F8A04E6FF008F92B21D7E7514B83F882
:10742000A04E6FF001F92C216FF03AF875E74D4B43
:1074300083F8A04E6FF0F8F82D21C7E709790F20E7
:1074400052E7097909204FE7097904204CE70979C7
:10745000052049E70979172046E70979881E414246
:107460004141414889F0FCFD21E70B79022B7FF473
:107470001EAF364801F006FE19E70C79012C06D044
:10748000022C09D0002C7FF412AF2146E9E72146F7
:10749000354889F0E5FD40E70121334889F0E0FDFA
:1074A000E7E72D4BD3F83C2A0B79991E4B424B4111
:1074B00082F82030FBE609798B1E59425941264B50
:1074C000D3F83C0AB4F098F8F1E60B79204A013B76
:1074D000012B8CBF0023012382F8F83EE7E60979EF
:1074E000112001E709791220FEE60B79012433B15E
:1074F000022B7FF4DCAE1D4B83F8404F0DE71B4A97
:1075000082F8403F09E709791520EDE6097918204E
:10751000EAE60F4BD3F8080F154B98427FF4C7AE3D
:1075200001900FF005FD24790198012C08D0022C60
:1075300020D0002C7FF4BBAE21460FF099FDB6E6BB
:1075400000210FF00DFDE8E670BE0030E83200309B
:10755000E8820030F0BA0030E8A2003028BB0030EA
:1075600020430030E8620030B0AE0030E8B20030B6
:1075700088C600300121E0E709790020B4E60979E6
:107580001020B1E609790220AEE609790120ABE6C8
:1075900009791620A8E609790720A5E609790B20C4
:1075A000A2E60B79022B4F4B0ED1012483F87047D2
:1075B0006FF03AF84A216EF073FF7AF00FFB4A4AF7
:1075C000062174F0ABFBA8E6002283F870276FF069
:1075D0002BF84B216EF064FF7AF000FB434A062142
:1075E00026E00C79012C09D0022C0CD0002C7FF461
:1075F0005EAE01213E4811F0ABFA58E600213C484E
:1076000011F0A6FA89E62146F4E70B799BB1022B2B
:107610007FF44DAE374BD3F8080F0368D3F88430AE
:10762000984700287FF443AE7AF0D8FA324A042112
:1076300074F074FB3BE62F4BD3F8080F0368D3F8C4
:107640008830984733E62B4BD3F8080F2B4B9842E2
:107650007FF42DAE0B79022B02D10FF01FFE26E630
:107660000FF0FAFC23E60979FFF70CFB244804F03D
:107670009DFC1CE62179FFF713FB18E609791B2016
:1076800032E621791C202FE609791E48FFF75AFBC4
:107690000DE62379022B7FF40AAE1B48FCF7A2FA11
:1076A0007AF09CFA194A9AE721797DF063FA184832
:1076B000AFF00EFA044600283FF4F9AD0D4B01225D
:1076C00083F8FD2E29E62379012433B1022B7FF4C0
:1076D000EEAD084B83F8384B1FE6064A82F8383B7C
:1076E0001BE600BFE8B2003008A5180819A5180865
:1076F000FC8E0030E88200302BA5180888C60030C8
:107700007CBA0030847B0030E832003044A5180891
:10771000108F0030002313B504460093019314F03A
:10772000AFFC694613F05AFA30B104F1080168461B
:1077300035F05CFC02B010BD024BD3F83C3A93ED3F
:107740001D0AF7E7E8A200301FB5002304461148E0
:1077500001930293039311F0C5FAB8B114F090FCB1
:1077600001A914F05FFA88B101A839F02BF9F7EEFE
:10777000007AB4EEE70AF1EE10FA07DDDDED010A5A
:107780009DED020A15F106FB84ED080A94ED080A46
:1077900004B010BDE8320030074B93F9550E0228B3
:1077A00005D0032806D0003818BF0120704781F0AB
:1077B0000100704704207047E862003003688B4284
:1077C0000CD00429C0E9001302D0072904D0704767
:1077D000034B1B680362704700238362704700BF3E
:1077E00098510030024608B5FFF7D6FF0146104613
:1077F000BDE80840FFF7E2BF70B5044616460D46E7
:107800002DED048BF0EE408A9FED2F9AB0EE608A4A
:10781000C4F086FEE0611EB3236813B92B4B1B68CE
:107820006362B7EE000A002DFFEE007A20FE270A01
:1078300060EE288AC4ED058AB4EEC98A244BD3F8D9
:107840003C0AF1EE10FA32DAB2F08CFE84ED060A50
:1078500020460321BDEC048BBDE87040FFF7AEBFAE
:1078600094ED090A38EEC00AB7EEC00A34F0ECF81D
:10787000B7EEC00B002D84ED050A0BDAB4EEC90A91
:10788000F1EE10FAD8DBDFED137A30EE670A84ED03
:10789000050AD1E7D0D0DFED107AB4EEE70AF1EEB9
:1078A00010FAC9D8DFED0B7A30EE270AEFE7B2F015
:1078B00059FEB4EE480AF1EE10FA48BFB0EE408A25
:1078C00084ED068AC4E700BF000000349851003000
:1078D000E8A20030DB0FC940000000B410B52DED68
:1078E000028BF0EE408A0446B0EE608AC4F018FEC7
:1078F0000621E061C4ED098A204684ED0A8ABDECC8
:10790000028BBDE81040FFF759BF000010B50446D8
:107910002DED028BB0EE408AC4F002FED4ED097A60
:107920009FED0B7AE061E8EE077AB7EEE70A34F0F4
:1079300073F8B7EEC00B00232046062184ED090A38
:10794000A362BDEC028BBDE81040FFF737BF00BF5C
:1079500035FA8E3C70B58B6806460C46144D73B9EB
:10796000CB6863B9496851B91248FFF73BFF95F8F6
:10797000511B05F6D820BDE870407FF00DBF95F88B
:10798000511B0D487FF056FD48B906F1080120460D
:107990001CF0F6FD18B102210648FFF70FFF224642
:1079A00095F8511B0448BDE870407FF0E9BE00BF68
:1079B000E8A2003094C70030C0AD0030072108B500
:1079C000FFF7FCFE80ED0A0A08BD000008B5036859
:1079D000032B23D1D0ED057A9FED127AF0EEE77AF2
:1079E000F4EEC77AF1EE10FA1AD50F4B90ED090AB2
:1079F000D3ED007A30EE670AB7EEC00A34F024F80F
:107A0000B7EEC00BDFED097AB0EEC00AB4EEE70ABC
:107A1000F1EE10FA94BF0120002008BD0120FCE720
:107A20000020FAE7000000349851003035FA0E3D8E
:107A300038B503680446023B082B5DD8DFE803F045
:107A4000050C2F32415736575700FFF763FE84ED80
:107A5000090A94ED090A38BDC4F062FDE369DFED5F
:107A6000290AC31AE06194ED050AF82007EE903A5E
:107A7000F8EE677A67EEA07AD4ED060A20EEA71A30
:107A800067EEE00A33F0F8FFD4ED057A77EEC07ABE
:107A9000C4ED057AD4ED097A37EE800AD7E7FFF70F
:107AA00053FED4E7184B1B686362D2E7174DD5F835
:107AB000500AB8F03FFC0028CBD0D5F8503A9B6B69
:107AC000F2E7C4F02DFDE3699FED0E7AC31AD4ED01
:107AD0000A6AE06107EE903AF8EE677A67EE877A15
:107AE00094ED097AA6EEA77A84ED097AB1E7074BFF
:107AF000D3F83C3A5B6FD7E7044BD3F8443AD3F85A
:107B0000B032D1E76F12833A3C920030E8A20030E5
:107B10000368092B08D8DFE803F0050A0505050509
:107B2000070705100023836290ED0A0A7047044B93
:107B3000D3F8443AD3F8B432F5E7C36AF3E700BFA9
:107B4000E8A2003070B5384D0446D5F8080F2DED89
:107B5000048B036888B0B0EE408AD3F88C30984725
:107B600000284ED0D5F8080F05F500569FED2F9A46
:107B700003689B6F9847D6F8443AD6F83C0AF0EE73
:107B8000408AD3EDAA9A0368D3F89C309847F0EE68
:107B9000400AD6F8443AD5F8080FD9EE890A93ED91
:107BA000AB1A036821EE091A1B6D8DED041ACDED99
:107BB000050A98470390D5F8080F0268526D904760
:107BC00028EE098A0090B0EE680A039B07A9BDEE73
:107BD000C88A9DED041ADDED050A05F60C3018EE95
:107BE000102A12B2B7F092F878B10A212046FFF7B6
:107BF000E5FD9FED0F7ADDED077A67EE877AC4ED3C
:107C00000A7A08B0BDEC048B70BD23680A2BF8D14A
:107C1000002361682046A36211B9FFF7E3FDF0E796
:107C2000FFF7CCFDEDE700BFE88200309F0CB345C5
:107C3000D4023739F8B500230D460446244ECB62F2
:107C40007CF0C8FB0368DB689847002834D0214FDC
:107C5000D7F8080F0368D3F88030984760B3D7F897
:107C6000080F03F073FE85ED0B0AB0EEC00ADFEDDE
:107C70001A7AB4EEE70AF1EE10FA03D4092130467D
:107C8000FFF79CFD95ED0B0A2846FFF75BFF1048B8
:107C9000FFF7CEFE0E4884ED000AFFF739FF336888
:107CA00084ED010A0A2B0FD8DFE803F00C10101046
:107CB0001010100C100C0C003368092BE2D10021BD
:107CC0000348DDE70223A3602046F8BD0123FAE75D
:107CD00094C70030E882003000000034034B0122DA
:107CE0001A6000229A60DA601A61704794C7003007
:107CF00013B5044601A910F06BFE04F5E04320B96A
:107D0000012283F8812B02B010BD03F674329DED81
:107D1000017AD2ED007AB4EEE77AF1EE10FA54BFB0
:107D200001220022EDE7000010B5044600F50540F1
:107D3000D030A1F0F9F904F50740BDE81040BFF0DC
:107D4000F3B9000008B50F22084803F019FC60B928
:107D50000F220621054803F013FC30B90F22092138
:107D60000248BDE8084003F00BBC08BDE832003013
:107D700070B5154E04460D4696F8213FDA0622D519
:107D80006FF3041386F8213FA6F500566EF04CFC05
:107D9000002214216EF0A4FB96F8383C0E2B12D171
:107DA000022D0AD0032D0AD0012D0CD194F85410C5
:107DB0002046BDE87040FFF7C5BF0621F8E794F8FC
:107DC00054100329F4D070BDE882003010B50E4C79
:107DD00049B9D4F8080F03681B689847A0F113034A
:107DE0005842584110BDD4F8080F03681B689847E3
:107DF0001328EED00E221321A4F5A04003F0C0FBFF
:107E00000028E6D1EEE700BFE882003030B50D462D
:107E100089B01146FFF7DAFF044640B304A81CF00E
:107E200027F914F02DF904A913F02EFE28B12869C2
:107E3000059B8342D4BF00200120DFED176A174B5A
:107E40009FED176AD3F8482ADFED167ACDED016A67
:107E5000CDED026A70B192ED067A27EE067A67EEF2
:107E6000277A01A91048CDED037A07F057FA20468A
:107E700009B030BD92ED077AA3F58041D3F8302ADE
:107E800027EE067AD1F83C3E9A42B0EEC77A67EE0A
:107E9000C77A67FEA67AE4E700000000E8A2003097
:107EA0000AD7233C0000C84250C40030F0B50F464A
:107EB00085B011460646FFF789FF044658B10025F4
:107EC00001AA39463046019502950395BFF038FA6C
:107ED000044618B90024204605B0F0BDDDED017A56
:107EE0009FED1B7AF0EEE77A0395F4EEC77AF1EE98
:107EF00010FA08D5DDED027AF0EEE77AF4EEC77AF3
:107F0000F1EE10FAE6D401A839F0F8FD01A839F035
:107F10003FFA104B9FED107A01A9D3F8483A0F4869
:107F2000D3ED057A67EE877A9FED0D7A67EE877A53
:107F30009DED017A27EE277A8DED017A9DED027A8B
:107F400067EE277ACDED027A07F0E8F9C3E700BFC4
:107F500000000034E8A200300AD7233C50C40030AF
:107F60000000C84270B50E46114605462DED028B45
:107F700084B0FFF72BFF044600283CD09FED2A8AEF
:107F800001AA314628468DED018A8DED028A8DEDDC
:107F9000038ABFF0D5F9044668B3244BDFED245AB9
:107FA000D3F8482A9FED236A92ED057ADDED017A38
:107FB00027EE257ADDED036AF4EEC86A27EE067A2D
:107FC000F1EE10FA67EE877ACDED017ADDED027AF7
:107FD00027EE877A8DED027A12DD92ED067A67EE52
:107FE000257A67EE867A67EEA67A01A91248CDED6A
:107FF000037A07F093F9204604B0BDEC028B70BD04
:10800000D2ED077AA3F58041D3F8302A67EEA57A3E
:10801000D1F83C3E9A42F0EEE77A67EE867A67EE58
:10802000A67A67FE887AE0E700000000E8A2003048
:108030000AD7233C0000C84250C400302DE9F0416B
:108040003D4F14460646884697F8213FDA0616D477
:10805000D7F8080F43F01003012587F8213F036884
:108060001B68984786F85400D7F8080F03681B6808
:108070009847092805D100242046BDE8F081002555
:10808000F2E7D7F8080F03681B6898471228F2D068
:10809000D7F8080F03681B6898470E28EBD0012C0F
:1080A00012D8062C38D801A353F824F0798006089A
:1080B000198106080B8106081F8106082B81060816
:1080C000E1800608018106081C4801F031FE002805
:1080D000E7D001220A211A48FAF748FB00241BE0E6
:1080E000002DC9D00E220621144803F049FA00B928
:1080F00000246EF099FA224614216EF0F1F9BBE7E4
:10810000002DB9D00E220521EEE72A464146304621
:10811000FFF77CFE0028E1D0002DADD0E9E72A462C
:1081200041463046FFF7C2FEF4E72A464146304654
:10813000FFF718FFEEE700BFE8820030E8320030BA
:10814000108F003000F540532DE9F04700F5E4585A
:10815000044600F5004508F118082DED068B93F94B
:10816000B63E84B033B100F5A046D6F82C3F93F864
:10817000D5707FB900214046A5F8641714F024FAA1
:1081800095F86517404604B0BDEC068BBDE8F04796
:1081900014F024BA04F5E044C4F0C2F982460DF1AB
:1081A0000409D4F8440A9FED878A90EDC59AB4F08B
:1081B00075FF002800F0D080D4F8443A03F54673E8
:1081C00093E8070089E8070048468DED038A39F0F7
:1081D00095FCF0EE408AD6F8080F03681B689847B4
:1081E000122840F0BC80002385F864378DED008AAA
:1081F00013F046FF694612F019FDD6F8080F036820
:108200005B69984728B1D6F8643BB3F90A30002B74
:108210000CDC96F8EB3E4BB1DDED007A05F26C73A9
:10822000C5F868A7F1EE677AC3ED007A95F8643770
:10823000DBB1D5F8680741F28833AAEB000A9A450A
:1082400010D8DDED007A05F26C73F1EE677A93EDEC
:10825000007A77EEC77AB6EE007AF4EEC77AF1EEDE
:1082600010FA02DD002385F86437D4F83C3AD3EDE8
:108270001B9A93ED1CAA8DED018A8DED028A8DED7E
:10828000038A13F0FDFE494613F0CCFC824668B128
:10829000484638F0A1FBF7EE047AB4EEE70AF1EEB7
:1082A00010FA4CBF4FF0010A4FF0000AD4F8440A0C
:1082B000B4F0F4FE30B1F7EE047AF4EEE78AF1EEB2
:1082C00010FA0AD9BAF1000F57D1D6F8080F03688F
:1082D0001B689847022857D00027D4F8440AB4F006
:1082E000CFFF0446002866D0B5EEC09AF1EE10FA32
:1082F00060D5FFEE007AB4EEE79AF1EE10FAACBF6B
:108300004FF001094FF0000913F0BAFE96F8E02C87
:1083100003A913F093FC50B1DDED037A9FED2A7AA7
:10832000F0EEE77AF4EEC77AF1EE10FA45D9B9F13A
:10833000000F08BF002795F86417404685F8657759
:1083400014F042F995F86517404614F047F904B067
:10835000BDEC068BBDE8F087F0EE488A3BE7D6F827
:108360002C3F93F8D530002B3FF440AF96F8EB3E0E
:10837000002B3FF43BAF012336E7D4F8440AB4F0B6
:108380008DFE0028A1D1A8E7B0EE4A0A13F194FCB3
:10839000B0EE408AB0EE690A13F18EFCDFED0B7A85
:1083A00020EE080AB4EEE70AF1EE10FACCBF01277E
:1083B000002792E70024A146A6E7B9F1000FBAD141
:1083C000002CB6E7000000009A99193F55CF7D3F79
:1083D00038B5044610F086FC04F5E455183548B964
:1083E000204610F04DFC014620B92846BDE8384033
:1083F00013F066BA04F5A044D4F8080F03681B6DA7
:10840000984720B9D4F8080F03685B6D9847014678
:10841000EBE7000030B5044689B004F5E455684642
:108420001BF026FE04A818351BF022FE69462846DC
:1084300013F02AFBB0B104A9284613F0E7FB88B17A
:1084400004A968461BF042FE236800226946D3F85F
:10845000B4302046984728B104F5AD4001213830AA
:10846000BFF0B8FD09B030BD00F5805292F8202F62
:10847000D2070CD400F5A042D2F82C2F92F8D510D8
:1084800009B1FFF7C7BF0368D3F8B030184770478A
:1084900030B587B0044602A801911BF0E9FD04F550
:1084A000E45002A9183013F0EFFA019A18B9002528
:1084B000284607B030BD236802A92046D3F8B4305F
:1084C000984705460028F2D004F5AD400121383028
:1084D000BFF080FDECE70000F0B5044685B00F4624
:1084E000154604F5E45668461BF0C2FD6946183689
:1084F000304613F08BFB10B9002005B0F0BD3946B3
:10850000304613F049F90028F6D0002DF5D004F5D7
:108510008054284694F8203F43F0020384F8203F1B
:10852000EBE700002DE9F04F2DED0A8BBDB00446BE
:1085300024220D4618A8002117F1E2FA2422002176
:1085400021A817F1DDFA04F5A047242200212AA86A
:1085500017F1D6FA2422002133A817F1D1FA00230B
:1085600097F8EF8E01200F93CDE90D33B8F1000F8E
:1085700028D197F8583B87F8EF0E08931DF03CFA86
:1085800090F925301BB390F8443303B304F5DF664C
:10859000C24630461DF040F95FFA8AF194F81E3762
:1085A0008B421DD930460AF1010A1DF013F98146AC
:1085B0000028F1D1CA4A0221284675F041FB87F80C
:1085C000EF9E01203DB0BDEC0A8BBDE8F08FC54A9F
:1085D0000221284675F034FB002387F8EF3EF0E7D0
:1085E00004F5B8430121283318460BEE903AF9F709
:1085F00043FE814608B9BC4ADDE720460FF072FC15
:10860000D7F8643BB3F90A90B9F1000F01D0B74A2B
:10861000DEE797F8EBAEBAF1000F07D1B44A0221BA
:10862000284675F00DFB87F8EFAECAE720469FEDB0
:10863000B18A01F095FE04F5BE434A460CA95833B1
:1086400018460CEE103A17F085FE00284FF08F0107
:1086500013AA14BF02230123ADF854900493F1230D
:10866000CDE913390A234FF00009CDE90031032386
:108670004D2195F8280072F07DF99F4B01220621CB
:1086800028465A729D4A75F0DBFA049B062128465B
:10869000022B0CBF9A4A9B4A75F0D2FA04F540535C
:1086A0004946304683F8629E1DF000F85FFA89F172
:1086B00094F81E378B420CD913AA30468DED138ADD
:1086C00009F101098DED148A8DED158A1CF06CFEFF
:1086D000ECE74FF0000A4FF07C0B30461DF09CF8A1
:1086E0005FFA8AF994F81E274A4519D94946304657
:1086F0001CF04CFD3CAAC0B20C230AF1010A0BFB92
:10870000004003FB092C00F28C70ACF1900C07C800
:108710008CE807003CAA02EB890909ED2F8ADFE704
:1087200041F288310AA82EF095FAD7F82C0F9FED68
:10873000719A0368F0EE499A9FED73AADB6A984735
:108740000121D7F82C0FBBF01DFD704BDFED70AA97
:1087500001211B68D86A039303681B689847C3F01C
:10876000DFFE0690C3F0DCFE079004F5A047089AF0
:1087700097F8583B934240F0D38094F83E1A304625
:108780001DF028F8002800F0CB80D7F82C3F93F894
:10879000D5300593002B00F0C38041F288310BA83F
:1087A0002EF058FAC3F0BCFE069BC01A132840F204
:1087B000D580C3F0B5FE069020460FF093FB7DF008
:1087C000DDFF81467DF064FFD7F8643BD7F82C0FBE
:1087D000B3F90A3000EE103AB8EEC00A20EE0A0AE9
:1087E000BDF046FB48467DF05BFF30461DF014F8B7
:1087F0001CEE100A17F0C8FFD7F8643BA220B7EEB2
:10880000001AB3F90A30DFED3B0A00EE103AB8EE79
:10881000C00A20EE0A0A33F02FF9B4EEE90A00226A
:108820000CA91CEE100AF0EE408AF1EE10FA58BFC7
:10883000F0EE409A17F08EFD08B900230C939DEDE1
:108840000C8ADFED347AB4EE498AF1EE10FAF4EED8
:10885000E78A48BFB0EE498AF1EE10FA80F28C80C8
:108860004FF000099FED2C9ADFED2C8A5FFA89FA10
:1088700094F81E37534540F28B810C2718ABB0EEAD
:10888000490A09F1010907FB0AF7D81938F018FD60
:1088900051463046CDED110A8DED121A8DED100ABC
:1088A0001CF074FC7C23C0B2B0EE680A03FB0040ED
:1088B00000F28C7038F004FD3CAB13A910A81F44E3
:1088C0008DED130ACDED140A8DED151A38F0CCFCA0
:1088D00007ED240A47ED230A07ED221AC6E700BF79
:1088E00049A7180838A7180877C6180857A71808FE
:1088F00069A71808000000009DC9003074A7180877
:1089000089A718080F4918086F12833A88C70030E2
:108910000000C84200000034A4707D3F0AD7233C09
:10892000D7F82C0F0368DB6A98470021D7F82C0F83
:10893000BBF028FC039B0021D86A03681B6898479A
:10894000B8F1000F40F059812846C44A052175F05E
:1089500077F9414630461CF0A9FE6DE1039BB0EE6D
:10896000498A0521986A03685B6898470BA82EF02E
:108970007DF9B0EE489AF8E600274FF00C0A04F5AE
:10898000E7695FFA87FB94F81E375B451CD95946A7
:1089900030461CF0FBFB0AFB0BF13CAB7C22C0B267
:1089A00001370B4402FB0090A3F16C0B099318AB49
:1089B0005430194438F06EFC099B03ED1B0ACBEDD3
:1089C000010A8BED021ADCE7049B4FF00009012B32
:1089D00042D14FF00C0A9FEDA2BA9FEDA29A94F8F3
:1089E0001E375FFA89F7BB4240F284800AFB07F723
:1089F0003CABB0EE680A09F1010903EB070821ABB3
:108A0000D81938F06DFC33AB08ED120AB0EE4B0A02
:108A1000D81948ED110A08ED101A38F051FC2AABAC
:108A20008DED100AB0EE490AD819CDED110A8DED81
:108A3000121A38F045FC13A910A88DED130ACDEDDC
:108A4000140A8DED151A38F025FC08ED090A48EDD9
:108A5000080A08ED071AC2E7F0EE088A9FED809A2F
:108A60009FED80BA94F81E275FFA89F39A4266D97F
:108A70009DED0C0AB4EEE80AF1EE10FA37DB4FF088
:108A80000C0808FB03F83CAB03EB080721AB03EB36
:108A9000080038F025FC33AB07ED120AB0EE490AA6
:108AA00003EB080047ED110A07ED101A38F008FC37
:108AB0002AAB8DED100AB0EE4B0A03EB0800CDEDAA
:108AC000110A8DED121A38F0FBFB13A910A88DEDD9
:108AD000130ACDED140A8DED151A38F0DBFBDDF825
:108AE000148007ED090A47ED080A07ED071A09F196
:108AF0000109B7E74FF000084FF00C0994F81E3752
:108B00005FFA88F7BB4241D933AB08F1010809FB92
:108B1000073038F0F3FF1BEE900AF0EE408AADF01C
:108B2000D3FF07EE900A3CABB8EE677A03EB8707FA
:108B3000C8EE877A67EEAA7A47ED2F7ADEE74FF024
:108B400000094FF00C0A94F81E375FFA89F7BB4210
:108B50001ED933AB09F101090AFB073038F0CEFF0B
:108B6000C8EE297A1BEE900A67EE808AADF0ACFF62
:108B700007EE900A3CABB8EE677A03EB8707C8EEC6
:108B8000877A67EEAA7A47ED2F7ADCE7DDF8148062
:108B9000C3F0C6FC079BC01AB0F5FA7F29D9C3F011
:108BA000BFFC04F5A0430C9AB121D3F8643BDDED82
:108BB0000D7A5B891392FCEEE77A339AADF85C305C
:108BC000149217EE903A349AADF85E301423159251
:108BD000359A07901692F022CDE9003213AA95F843
:108BE000280071F0C7FEA3F009F995F82810A2F04B
:108BF00091FD0BA82EF03AF8BBE64FF000084FF0BD
:108C00000C09049930461CF051FD5FFA88F194F884
:108C10001E378B4208D933AB304608F1010809FBF7
:108C200001321CF0C1FBF0E730461CF0CFFB0E4ACE
:108C30000621284675F004F80C4B002520465D728D
:108C400001F080FB04F57950223061F00DFB0AA899
:108C500087F8EF5E2EF00AF82846B3E42F8D1A0845
:108C6000A4707D3F0AD7233C91A718089DC9003006
:108C700010B5838F044643B96BF03EFF92224FF448
:108C800080116BF0F1FE638FA387A08F10BD0000F1
:108C90002DE9F3414E4F0446D7F8E83ADA0700F1E0
:108CA000948000F5A045D5F82C3F93F8C120002A08
:108CB00040F08B8093F8D530002B00F0838095F83E
:108CC000EB3E002B7ED100F5004393F87037002B6C
:108CD0007BD100F5E046D6F83C0A6C3037F072FEE6
:108CE000DFED3C7AB4EEE70AF1EE10FA6ADCD6F872
:108CF0003C3A9FED397AD3ED377AF4EEC77AF1EE4C
:108D000010FA04D5D5F82C3F1B7A002B5AD0B5EEBB
:108D1000007AF4EEC77AF1EE10FA53D400230193EF
:108D200013F0AEF995F8E02C01A912F087FF0028A6
:108D300048D0DFED2A7A9DED017AB4EEE77AF1EEC4
:108D400010FA3FDBD6F83C3A9FED257AD3ED367A20
:108D500067EE877AB3EE0E7AF4EEC77AF1EE10FA88
:108D600030DA204E04F16800338801333380FFF796
:108D70007FFF3388834228D34FF00008A6F8008095
:108D80006DF052FC012219216DF0AAFBD5F82C0FD1
:108D900003689B699847431C04F5BA40124A414650
:108DA000103072F0BBFFD5F82C3F012283F8C120B0
:108DB000D7F8E83A5B0708D504F5A050183091F0D1
:108DC00051FB02E0074B00221A8002B0BDE8F0819F
:108DD000E8820030235E8C3D6666663F000000340A
:108DE000E02E6542CEC70030A8A718084A4BF0B560
:108DF0002DED028BD3F8E83A85B004469B071FD4CB
:108E000000F5E046DFED458AD6F83C0A03681B69A9
:108E10009847D0ED017AF4EEE87AF1EE10FA0FDB24
:108E200004F5A04304F50745D3F82C2F743592F8C8
:108E3000C11049B1002303A9284603936FF046FEF1
:108E400005B0BDEC028BF0BD92F8D520002AF1D020
:108E500093F8EB3E002BEDD104F5004797F87037FF
:108E6000002BE7D1D6F83C0A03681B699847D0F875
:108E7000B030D6F83C0A039303681B69984704F5A1
:108E80008C7200F1B00128466FF00EFFDDED037A21
:108E9000B0EEC08AF0EEE77AF4EEC87AF1EE10FA9E
:108EA00003D503A928466FF011FED6F83C0A0368E3
:108EB0001B699847D0ED040AF4EEE80AF1EE10FAC7
:108EC000BEDBF6EE087A60EEA77AF4EEC87AF1EE31
:108ED00010FA1AD5C3F024FBD7F8803742F210728B
:108EE000C31A9342ACD99FED0E0A0021C7F8800740
:108EF00004F5BA4028EE000A0A4A1030B7EEC00A5C
:108F00008DED000B72F00AFF9AE79DED030A32F037
:108F10006FFC0028DED193E7E882003000000034C7
:108F20000000C842C4A7180810B5044600F5F74071
:108F3000483088F0A7F804F5F74001216830BDE813
:108F4000104097F0ADBE0000F7B500F5E0440546CF
:108F500094F9C83B63B300F5A04694F8DC2B05F503
:108F6000F74796F8EB3E483783F0010363F3C302FB
:108F7000002384F8DC2B019313F082F896F8E02CA0
:108F800001A912F05BFE9DED010A384688F0FAF85F
:108F900005F5004393F8703753B9384688F09EF8CA
:108FA000D6F82C3F93F8D53023B9334B00221A80E2
:108FB00003B0F0BD94F8DC3BDB07F9D4D6F8080F1A
:108FC0000368DB6B98470028EFD096F8EB3E002B48
:108FD000EBD1294E33884BB9B4F9CE3B33B164227F
:108FE00013FB02F3D4F8302A9A42E1DB384688F0CA
:108FF000E5F8D4F83C3A9FED217AD3ED367A67EE66
:10900000877AB3EE0E7AF4EEC77AF1EE10FA05D84D
:109010003388002BCCD0013B3380C9E705F16807CA
:1090200004F608243846FFF723FE3388D4ED007A8F
:10903000984284BF013333803388012B104B02D117
:10904000C3ED007AB4E793ED007AB4EEE77AF1EE7F
:1090500010FAAAD93846FFF70BFE33888342A7D30C
:10906000002333806DF0E0FA02220C216DF038FA13
:109070002846FFF759FF9BE7CCC70030E02E65423A
:10908000C8C7003000F5E04208B592F9C83B63B3A9
:1090900000F5A04393F8EB3E73B100F5BA40134AD4
:1090A0000621103072F03AFE6DF0BEFA03220F2155
:1090B000BDE808406DF014BAB2F9CE3B8BB1642123
:1090C000D2F8302A13FB01F39A420ADA00F5BA40CB
:1090D000074A0121103072F021FE6DF0A5FA02223C
:1090E000E5E7BDE80840FFF71FBF08BDDCA718088B
:1090F000EEA7180870B500F5A0450446544E2DEDB6
:10910000028BD5F82C3F8CB093F8D5303BB195F855
:10911000EB3E23B900F5405393F97E3E2BB9002373
:1091200033800CB0BDEC028B70BD00F5004393F8AA
:109130007037002BF3D101F07DFB002874D1D5F8F6
:10914000080F0368DB6B98470028E8D004F5F4406B
:109150000C306FF011FD38F0D1FCF0EE087AF0EE33
:10916000408AB4EEE70AF1EE10FAD8DA04F5E453D7
:109170009FED388AD3ED9C7A93ED9B0A20EE270A67
:1091800013F1A0FDF2EE0E7A20EE080AB4EEE70A23
:10919000F1EE10FAC3D904F5E043F3EE0E7AD3F8FA
:1091A0003C3A93ED367A27EE088AB4EEE78AF1EE80
:1091B00010FAB4D904F5E450002309A91830099332
:1091C0000A930B9312F02EFD002835D1358804F157
:1091D00068000135ADB23580FFF74AFDB5EB400FB1
:1091E0009FDB6DF021FA01220C216DF079F900224C
:1091F000194BB7EEE80AB7EEC88A04F5BA40002169
:109200001030CDE90623154B00228DED040BCDE97E
:1092100002238DED008B124A72F080FD01220C2199
:109220001048F9F7A3FA7CE7D5F8080F03685B6DDF
:109230009847002883D172E709A838F05FFCF2EE66
:10924000047AB4EEE70AF1EE10FABFDB67E700BF7D
:10925000C4C70030E02E65420000084000003E40D8
:1092600004A81808108F0030F0B500238BB0044616
:1092700000F5E450079302AA089304F5A046099369
:1092800005AB03A91830019307AB009304AB12F0B0
:1092900045FB054686F8040D18B9002528460BB095
:1092A000F0BDC3F035F9D6F8083D9FED2D7A07469D
:1092B000C31A04F5B94006AA02A907EE903A6C3029
:1092C000F8EE677A67EE877ACDED067A6FF0ECFC00
:1092D00004F5B94004F57A5406AA03A978308DED57
:1092E000020A6FF0E1FCC6F8087DD4ED007AF5EED5
:1092F000C07AF1EE10FAD0D9DDED086A9DED077A5B
:10930000D6F8902C87FE267ADDED096A87FE267A4C
:10931000F4EEC77AF1EE10FA94BF0123002312B1E4
:1093200096F8942C92B937EEA77AB4EEC70AF1EE0C
:1093300010FA0BDB0233DBB29DED027AF4EEC77A52
:10934000F1EE10FA09D8002BA7D0A7E7B4EEE70A90
:10935000F1EE10FAF0DB0133EDE7012B9ED89CE72C
:10936000BD3786352DE9F04700F5A045044695F850
:10937000213F43F0040385F8213F6DF055F90122A8
:1093800011216DF0ADF8D5F82C3F93F8D530002BB6
:1093900051D02A4B012204F5405820465A7398F9BF
:1093A0007D9E09F033FC074638B1B9F1000F04D0B7
:1093B00004F50E40C43009F011FC214BD3F8080F1E
:1093C00003681B69984798B998F97D3E033B18BF1D
:1093D000012304F5BA461036B9F1000F01D007B9E0
:1093E00043B13046174A0221BDE8F04772F096BCFF
:1093F0000023EEE798F97D1E81B1022903D195F88B
:10940000213FDB0704D50621204609F0EBFB05E0F0
:109410000622204602F0B4F80028F4D0D5F8080F50
:1094200003689B6C9847084A034602213046BDE812
:10943000F04772F073BCBDE8F08700BF9DC90030F3
:10944000E882003038A8180845A8180800F5A0429E
:1094500008B592F8213F590717D56FF3820382F8B8
:10946000213F0A4B5A7B42B1002200F5BA4002214B
:109470005A731030064A72F051FC6DF0D5F8002294
:109480001121BDE808406DF02BB808BD9DC9003022
:1094900068A81808F0B5054685B005F5E457684694
:1094A0001AF0E6FD69461837384612F0AFFB80B176
:1094B00005F57A53384CD3ED007AF5EEC07AF1EE2B
:1094C00010FA08D80023354A28462380D373FFF7C3
:1094D000BDFF05B0F0BD2846FFF7C6FE064628468C
:1094E0000FF0CEFB10B928460FF0A2FB002EA37898
:1094F00018BF00200343DBB2A370002BE9D06378D0
:10950000A8BB83BB23780133DBB2082B237003D1C4
:109510004EB3384612F082FA2378092B02D138462E
:1095200012F074FA2378092B1DD94FF48573238028
:109530006DF07AF8022210216CF0D2FFC2F0F0FF39
:109540006368C01A47F23053984209D905F5BA400A
:10955000134A0221103072F0E1FBC2F0E1FF6060BB
:109560002846FFF7FFFE62780C4BDA73B1E72678E6
:10957000002EF8D0013EF6B22670002BF3D0002E5C
:10958000F1D166706DF050F8324610216CF0A8FFF2
:109590002846FFF75BFFE6E7D0C700309DC90030E3
:1095A00080A8180800F5A04393F8213F5B0701D578
:1095B000FFF7D8BE7047000073B5044600F5E450CD
:1095C00001A904F5A045183011F0E6FF0646D5F8CC
:1095D000D83C83420CD004F5E043D3F83C0AB2F007
:1095E000A5FBC5F8D86C6DF01FF83E216CF058FF54
:1095F00004F5805695F9DC1C96F9B42F96F8B43F23
:1096000091421BD0FF2B19D004F5E043D3F83C0A5C
:10961000B2F08CFB96F8B43F85F8DC3C6DF004F8B2
:1096200095F8DC2C18216CF05BFF04F5BA4095F935
:10963000DC3C0421024A103072F070FB02B070BDB5
:1096400090A818082DE9F0438FB00546C2F068FFD6
:10965000002305F5E4580646059308AA069308F189
:109660001808079305A90893404609930A930B939A
:109670000C930D9304AB019303AB00930BAB12F06F
:109680002DF9DFED477A9DED077A0746B4EEE77ACC
:10969000F1EE10FA30DB9DED0A7AB4EEE77AF1EEE6
:1096A00010FAACBF0124002405F5A049404699F802
:1096B000043D002B08BF002712F022F98046EFB9C5
:1096C000444699F9803A012B29D164B1D9F82C3F4D
:1096D00093F8D5403CB1D9F8080F03685B69984707
:1096E00080F00100C4B299F8E03CCBBBCCB9C9F81A
:1096F000E46C0FB0BDE8F0830024D5E7002CDFD088
:1097000005F5B94078306FF0DFF9F7EE007A90EDAB
:10971000007AB4EEE77AF1EE10FAD2DCD0E700245A
:10972000E1E7D9F8E40C301AB0F57A7FE1D9C9F84D
:10973000E83C012405F5E04389F8E04CD3F8443ACD
:1097400083F8C8436CF070FF22461D216CF0C8FE00
:10975000144A05F5BA400221103072F0DFFAC8E76A
:1097600014B1C9F8E86CC4E7D9F8E80C43F69823BB
:10977000361A9E42BDD905F5E043C9F8E44C89F894
:10978000E04CD3F8443A83F8C843C9F8E84C6CF08D
:109790004BFF22461D216CF0A3FE034AD9E700BF10
:1097A00000000034A8A81808C2A818080B4B012212
:1097B00010B504465A72C2F0B3FE04F50042D2F866
:1097C0005C37C31A142B08D9C2F85C0704F5E250C1
:1097D000BDE8104004305BF065B810BD9DC9003095
:1097E0002DE9F743044600F5795000230DF10701F8
:1097F00004F5A04638308DF8073061F0A3FCD6F8A8
:109800002C0F90F9C030026883B3083BD569DBB2F6
:10981000012B2BD93221A84704F1100004F5BA48D6
:1098200017F05EF91F4B4FF0000908F110081F6890
:10983000F86A0368DB69984701281ED1C2F070FE00
:1098400041F28733A0EB090205469A4205D9A946A1
:10985000154A0621404672F061FA2046FFF7A6FF3E
:10986000B86A032103685B689847E1E704F5405351
:10987000D269B3F8941E9047CEE70121D6F82C0F99
:10988000BAF080FCD6F82C0F03681B6B98477CF06D
:109890007DFAF86A012103681B6803B0BDE8F04354
:1098A000184700BF88C70030E0A8180870B5044604
:1098B00000F5BA40184A06211030184E2DED028BE3
:1098C0009FED178A72F02AFA2046FFF789FF20469B
:1098D000FFF76CFF20460EF005FB33680321986A02
:1098E00003685B6898477CF049FF05467CF0D0FE32
:1098F00004F5A043D3F8642BD3F82C0FB2F90A2057
:1099000000EE102AB8EEC00A20EE080ABCF0B0FA49
:1099100028467CF0C5FEDAE704A9180888C700309D
:109920006F12833A2DE9F047044600F5BA402B4AFE
:109930000621103004F5A046DFF8A89041F2873ADE
:109940002DED028B72F0EAF92046FFF749FF7CF01B
:1099500015FF05467CF09CFEB7EE000AD6F82C0FEA
:10996000BCF086FA28467CF09BFEC2F0D9FD074683
:10997000C2F0D6FDC01BD9F80080504517D99FED25
:10998000188A28467CF084FEB0EE480AD6F82C0FE0
:10999000BCF06EFA28467CF083FE2046FFF706FFF7
:1099A000D8F82800032103685B689847E9E7284650
:1099B0007CF06EFEB7EE000AD6F82C0FBCF058FA19
:1099C00028467CF06DFE2046FFF7F0FED8F8280010
:1099D000032103685B689847CAE700BF34A91808E9
:1099E0000000000088C700302DE9F34100F5A046D3
:1099F0000446D6F82C3F93F9C030032B2BD06525B5
:109A000000F50048344F013D15F0FF050CD0D8F8A3
:109A100058374BB93B681421986A03685B689847CC
:109A200020460EF05FFAEEE704F5B8400121283039
:109A3000F8F722FC04F5405393F9783E70B953B11E
:109A4000092B08D08DF8070004F579500DF10701B6
:109A5000383061F077FB02B0BDE8F081032B34D8D9
:109A6000DFE803F002252D30D6F8643BB3F90A2075
:109A700040F2B5339A422ADD04F5795001250DF103
:109A8000070138308DF8075061F05CFB04F5BA40EF
:109A9000124A0221103072F041F9114B5D720E4BE7
:109AA0001C68A06A052103685B689847F9E7D6F847
:109AB000643BB3F90A2040F2B5339A4207DD2046F1
:109AC000FFF7F4FE2046FFF72DFF092BC3D000233C
:109AD0008DF80730B8E700BF88C7003058A91808CC
:109AE0009DC9003000F5BA400B46024A04211030EF
:109AF00072F014B978A9180810B504466CF094FDFA
:109B0000002205216CF0ECFC04F5BA40034A042164
:109B10001030BDE8104072F001B900BF84A91808E8
:109B20000B4613B54AB100F5BA4000920421054A2C
:109B3000103072F0F3F802B010BD02B0BDE8104072
:109B4000FFF7D0BF9CA9180800F5BA40064A0421C7
:109B5000103008B572F0E2F86CF066FD00220821C2
:109B6000BDE808406CF0BCBCB0A9180838B5044684
:109B70000D46C2F0D5FC04F5A0433DB9D3F8182F2B
:109B8000C3F81C0F0AB9C3F8180F38BDD3F81C2F3F
:109B9000801A642882BF0022C3F81C2FC3F8182F34
:109BA000F3E7000038B5044612F06AFA4FF480413A
:109BB00011F0A4FA04F5A043054693F8F52E82426D
:109BC0001AD004F5BA4483F8F50E103460B16CF085
:109BD0002BFD02220B216CF083FC084A2046022157
:109BE000BDE8384072F09AB86CF01EFD2A460B2191
:109BF0006CF076FC024AF1E738BD00BFC8A918082E
:109C0000E4A9180838B50A460C460621054601F0B5
:109C1000B7FC28B1054A137843F00803137038BD28
:109C200021462846BDE8384008F0DCBFBCC90030FA
:109C300038B50A460D461521044601F0A1FC28B1AD
:109C4000094A137843F00803137038BD04F5BA408D
:109C50000421064A103072F061F829462046BDE81A
:109C6000384008F0BFBF00BFBCC90030F4A91808D5
:109C700038B50A460D461521044601F081FC28B18D
:109C8000094A137843F00803137038BD04F5BA404D
:109C90000421064A103072F041F829462046BDE8FA
:109CA0003840FFF7AFBF00BFBCC900301CAA18087E
:109CB00038B50A460D461B21044601F061FC28B167
:109CC000094A137843F00803137038BD04F5BA400D
:109CD0000421064A103072F021F829462046BDE8DA
:109CE0003840FFF78FBF00BFBCC9003032AA180848
:109CF00038B50A460D461121044601F041FC28B151
:109D0000094A137843F00803137038BD04F5BA40CC
:109D10000421064A103072F001F829462046BDE8B9
:109D2000384008F05FBF00BFBCC9003044AA180823
:109D300038B500F5A04494F8F95E15B10125284620
:109D400038BDD4F8080F03681B689847032807D06C
:109D500004D802280DD194F8EB5EF0E71B28FAD165
:109D600094F8E93E002BEAD194F8EB5E002DE5D1A2
:109D7000E5E794F8F33E002BE0D1ECE738B500F5C9
:109D8000A045044695F8213F43F0080385F8213F9C
:109D900000F5E043D3F8480AB6F024FF0128014655
:109DA0001ED0022802D040B9194B1AE0194B1A4AAA
:109DB00004F5BA40103071F0B1FF6CF035FC0122AF
:109DC00017216CF08DFB2046FFF7B2FF60B104F560
:109DD000B840012215212830BDE83840F8F7C6BC4C
:109DE0000E4B0D4A0221E3E7D5F8080F03681B6804
:109DF0009847062806D104F50F40BDE83840DC300E
:109E00000AF024B920460B21BDE83840FFF7FABE1E
:109E100083AA180861BC180858AA18086DAA18085F
:109E200070B500F5A0450646D5F8182FD5F81C3FAB
:109E30009B1A41F28832934211D9D5F8080F036872
:109E40009B6D9847044695F8213FC3F3C003A34296
:109E500013D034B13046BDE87040FFF78FBF002407
:109E6000F1E76CF0E1FB224617216CF039FB95F825
:109E7000213F64F3C30385F8213F70BD0B461146B3
:109E800010B50446072B07D8DFE803F02A041316A1
:109E9000191C242708F0A6FE04F5A043D3F8843A41
:109EA0009B061DD504F5A050BDE81040183090F079
:109EB000D9BAFFF7A7FEEFE7FFF7DAFEECE7FFF707
:109EC000B7FEE9E700F5B840012214212830F8F781
:109ED0004DFCE1E7FFF7ECFEDEE7FFF709FFDBE70C
:109EE00010BD000070B504466CF09EFB01220521F8
:109EF0006CF0F6FA04F54053204693F8623E072BC7
:109F000096BF304A0125D55CFFF712FF68B12E4A93
:109F100020462E49FFF704FE04F5B8400122102127
:109F20002830F8F723FC002516E004F5A046D6F803
:109F3000080F03685B6D9847A8B104F5C04393F818
:109F4000ED2482B193F9EC34012B0CDC204A214939
:109F500001252046FFF7E4FD294620460322BDE8FF
:109F60007040FFF78BBFD6F8080F03685B6D98470A
:109F700018B1D6F8843A190715D4D6F8080F036833
:109F80001B689847032803D1D6F8843ADA070DD422
:109F9000D6F8080F03685B6A984768B90B492046F2
:109FA000FFF7A0FDD8E70A4A0849D1E70A4A07495E
:109FB0002046FFF7B5FDB6E7D6F8843A5B07EDD546
:109FC000064AF4E73CAB180890AA1808FDD0190817
:109FD0009AAA1808ADAA1808BDAA1808CDAA180888
:109FE00070B5044615466CF01FFB012206216CF08B
:109FF00077FA2046FFF79CFE98B104F5B84001229D
:10A00000072100252830F8F7B1FB134A13492046F1
:10A01000FFF786FD294620460422BDE87040FFF781
:10A020002DBF04F5A046EDB2D6F8080F03685B6DAE
:10A03000984758B1D6F8843A1B0707D535B1084A76
:10A04000204606490125FFF76BFDE3E7034920465B
:10A05000FFF748FDDEE700BF90AA1808EAAA180833
:10A060009AAA1808F8B504466CF0DEFA0122082115
:10A070006CF036FA04F5A0467AF01AF804F540536D
:10A0800093F8513E072B96BF364A0225D55CD6F889
:10A090002C3F93F8D5705FB933492046FFF722FD76
:10A0A0000025294620460522BDE8F840FFF7E6BE18
:10A0B0002046FFF73DFE60B104F5B84001221221B1
:10A0C0002830F8F753FB294A27492046FFF728FD97
:10A0D000E6E7D6F8080F03685B6D984778B104F59A
:10A0E000C04393F8ED2452B193F9EC34012B06DC14
:10A0F0001F4A204920460125FFF712FDD1E7D6F877
:10A10000080F03685B6D984718B1D6F8843A1907B1
:10A1100013D4D6F8080F03681B689847032803D1A7
:10A12000D6F8843A9A070BD4D6F8843ADB0609D4D9
:10A130000D492046FFF7D6FCB3E70D4A0A49D9E797
:10A140000D4AC1E7D6F8080F0368DB699847064651
:10A150000028EDD1094A204603493546FFF7E0FCC7
:10A160009FE700BF44AB1808C2301A0890AA18082D
:10A170009AAA1808E4AA1808F2AA180807AB18083F
:10A1800000F5405370B593F9513E0446BBB300F55A
:10A19000A045D5F8706E96B3C2F0C2F905F52E63EE
:10A1A000DFED177A861B93ED000A8D209FED151ABF
:10A1B00020EE270ADFED140A31F05EFCBCEEC00A87
:10A1C00010EE103A9E420CD295F8213F9A0716D510
:10A1D00020460021F8F712FC2046BDE87040FFF74A
:10A1E000B3BC0CD995F8213F9B0708D42046012128
:10A1F000F8F704FC2046BDE87040FFF733BF70BDA0
:10A2000000007A440000804F00000000F8B50646C8
:10A2100011F036FF4FF4802106F5A04410F06EFFD8
:10A220000546C2F07DF994F8243F0746AB420DD0B5
:10A2300006F5BA4084F8245F1030002D3DD0394B2C
:10A24000394AC4F8287F022171F068FD94F8243F50
:10A2500043B394F8253F2BBBB4F9F63A4FF4B070F2
:10A260009FED320A07EE903A9FED311ADFED310A89
:10A27000F8EEE77A27EE800A31F0FEFBBCEEC00A6A
:10A28000D4F8280F10EE103A3F1A9F420AD9012342
:10A2900006F5BA40284A022184F8253F1030214BA8
:10A2A00071F03CFD94F9F53A002B94F8213F0BDC5A
:10A2B0006FF3451384F8213FF8BD1A4B1F4AC4F8C9
:10A2C000285F84F8255FBEE7C3F34012AA42F3D0AB
:10A2D00065F3451384F8213F9B06EDD5184BD3F861
:10A2E000080F03681B6998470028E5D06CF09CF9BB
:10A2F00001221F216CF0F4F83046FFF719FD40B140
:10A3000006F5B840012221212830BDE8F840F8F7D1
:10A310002DBA94F8F51A30463222BDE8F840FFF71E
:10A32000ADBD00BF20AB18085CC8190800007A4416
:10A330000000804F000000002FAB180837C8190834
:10A34000E882003008B50122034B1A70C2F0E0F831
:10A35000024B186008BD00BFD9C70030DCC7003011
:10A36000014B00221A707047D9C700302DE9F04127
:10A370000446C2F0CDF82A4B0546B4F8BE20198831
:10A38000284E91420ED01A80274B18603378A3B123
:10A39000002434706CF048F922461321BDE8F041E6
:10A3A0006CF09EB83378214FDBB93B782BB11E4B54
:10A3B0001F4A1B68C31A934201D8BDE8F0810123EC
:10A3C000337004F5A043D3F82C0F90F8D53013B1B7
:10A3D0000368DB6A98476CF027F9012213216CF0BF
:10A3E0007FF83B78002BE8D03378002BE5D00E4A7D
:10A3F00010491368EB1A8B42DFD904F5A0441560AD
:10A40000D4F82C0F90F8D530002BD6D00021B9F01D
:10A41000B9FED4F82C0F0368BDE8F0419B6A1847D9
:10A42000DAC70030D8C70030DCC70030D9C70030E9
:10A4300080841E0040420F00F8B50546C2F070F857
:10A4400005F54054D4F8CC3AC31A272B38D994F8E0
:10A45000C83AABBB05F5A047C4F8CC0A94F8306AFB
:10A46000D7F8080F03685B6D9847014640B997F825
:10A47000EB1E29B9D7F82C3F93F8D51081F00101D4
:10A4800005F56750243091F06BFB84F8C90AA0B938
:10A490009EB194F8303A83B90A4B93F8EB3E33B946
:10A4A00005F5BA40084A0521103071F037FC6CF010
:10A4B000BBF8002209216CF013F8012384F8C83A94
:10A4C000F8BD00BFE88200304CAB1808F8B500F5C5
:10A4D0004055044695F8C83A4BB100F5A047D7F867
:10A4E0002C3F93F8D5301BB9002385F8C83AF8BD46
:10A4F00095F8C92A002AF7D0334B93F8EB3E2BB9D5
:10A5000000F567503149243090F078FD95F9EA69FB
:10A510004EB197F8EB3E73B104F5B84001220F211C
:10A520002830F8F723F96CF07FF895F8C92A09214B
:10A530006BF0D6FFD8E7D7F8080F03685B69984738
:10A5400050B197F8F33E3BB197F8213FDA0703D4B7
:10A5500095F8303ADB07DFD504F5675095F8C91A4E
:10A56000243091F09FF8DFED1A7AB4EEE70AF1EEAD
:10A5700010FA05DD0A220921204601F001F8D2E790
:10A58000023E032E11D801A353F826F075A5060844
:10A590009DA50608BBA50608C1A506080A22152127
:10A5A000204600F0EDFF0028BDD10A2206212046FA
:10A5B00000F0E6FF0028B6D1DCE70A221121F6E719
:10A5C0000A221521F3E700BFE882003064AB1808C7
:10A5D0000000C84270B500F5A04300F5E045044610
:10A5E00086B093F8E01CD5F8440AB3F0D7F804F528
:10A5F000AE407030AEF010FD02A819F039FD04F540
:10A60000E45002A9183011F03FFA049BC5F8343A1F
:10A61000059BC5F8383A11F033FD01A910F006FB8F
:10A62000E8B1DDED017A04F5F4469FED117A04F509
:10A6300080542C36022267EEC77A3046FDEEE77A68
:10A6400017EE901A17EE905A19F016FD94F8203F65
:10A65000DB0706D401222946304619F00DFD06B06D
:10A6600070BD0121304619F0E1FD0028F2D0F6E777
:10A670000000C84270B500F5004486B00D4616468D
:10A68000B4F88C378B4203D1D4F88837934221D069
:10A69000C1F046FFD4F88437C31A132B1AD9C4F873
:10A6A0008867A4F88C57C4F884076BF0BDFF044694
:10A6B000C1F03EFF084B094A1B68CDE90453084B23
:10A6C0000193084BCDE9020100932046064B074950
:10A6D0006BF036FD06B070BDE0C7003070AB1808F7
:10A6E00088AB1808D37F18089F5F180883AB180839
:10A6F00038B500F5A0450C4695F8F23E8B4207D0E0
:10A7000021B16BF091FF11216BF0CAFE85F8F24E7A
:10A7100038BD000070B500F5A045064600F5E044E0
:10A720002DED048BD5F82C3F93F8D530002B49D074
:10A7300095F8EB3E002B45D1D5F8080F03685B690F
:10A740009847002843D1D4F83C0A6C3036F03AF9E7
:10A7500006F5F440D4F83C3AB0EE409A0C30D3ED14
:10A76000368A6EF009FA37F0C9F9D4F8443AD5F8C8
:10A77000080FB0EE408AD3EDC59A03685B6D984729
:10A78000DFED297AB4EEE79AF1EE10FA02DC95F8E3
:10A79000043F03B178B3DFED257A68EEA78AF3EEC4
:10A7A0000E7AF4EEE78AF1EE10FA24DCF0EE087A85
:10A7B000B4EEE78AF1EE10FA1DDCF5EEC09AF1EE88
:10A7C00010FA18DAD4F83C0A0368DB6F0EE0D5F80B
:10A7D000642BD4F83C0AB2F90A200368002A03DC8F
:10A7E000D5F8002F022AF0D1D3F88030BDEC048BCD
:10A7F000BDE870401847D4F83C5A40F23B20B7EE11
:10A80000001ADFED0B0A2B68D3F88460D4F8443AC1
:10A8100093EDA40A31F030F928463346BDEC048BA1
:10A82000BDE87040184700BF235E8C3DE02E6542B6
:10A830000000000000F5A04090F8040F70470000F1
:10A840002DE9F04100F5A04605460C4696F8EB3E92
:10A850008B4244D0234B00221A6000293BD06BF07E
:10A86000E3FE122184F001086BF01AFE86F8EB4E2D
:10A8700005F54057A1F084FD4146A1F059FDB8F11E
:10A88000000F06D097F83A3C1BB9C1F049FEC7F853
:10A890003C0C87F83A8C14B3B7F8343E5B071ED5EE
:10A8A000D6F82C3F93F8D530CBB1D6F8080F036813
:10A8B0005B69984798B9D6F8080F202103689B690F
:10A8C000984760B105F5B84001220D212830BDE858
:10A8D000F041F7F74BBF6BF0A7FE1C21C2E7BDE8C4
:10A8E000F08100BFE0C700302DE9F04F00F5A04532
:10A8F00000F5004304462DED088BD5F82C2F85B0CC
:10A9000092F8D56001931EB90121FFF799FF0BE082
:10A9100095F8EB3E002B5DD0D5F8080F03681B6D52
:10A9200098470646002839D04FF0000B95F8EB1EEB
:10A93000A14EB1B9D6ED007A04F16800B8EE678A8D
:10A94000FEF796F907EE900A9FED9C7AF8EEE77A0B
:10A9500067EE877AB4EEE78AF1EE10FAACBF012118
:10A9600000212046FFF7C4FE95F8EB2E0AB14BF00C
:10A97000010B95F8F22E0AB14BF0020B019B93F8F4
:10A9800070270AB14BF0080B32685946204605B0D3
:10A99000BDEC088BBDE8F04FFFF76CBED5F82C3F3F
:10A9A000204693ED0C8AF8F71BF9B4EEC80AF1EED5
:10A9B00010FAB9D5D5F82C3F93F8A130032BB3D1B9
:10A9C0006AF09AF84FF4801142226AF04DF831464D
:10A9D00020469AE7019991F87097B9F1000F02D0DB
:10A9E000754A1360A0E700F5E04A92F80780DAF8AC
:10A9F0003C0A03689B6F984707460090D5F8080FFC
:10AA000003685B69984720B1D5F8003F022B00F03E
:10AA1000C880B8F1000FF7EE00AA0CBF4FF0000B92
:10AA20004FF4007B17B14BF4806B009604F5F747A9
:10AA3000DFED63BAB3EE0EBA6837384696F050F9D8
:10AA40000130DAF83C0A0CBF012302236C3008EE17
:10AA5000103A35F0B7FFDAF83C2AB4EEEB0ADFED36
:10AA6000597A04F5F440D2ED369AB0EE40AAF1EEF0
:10AA700010FA00F10C0069EEA79AC8BF4BF4807B76
:10AA8000F4EECB9AF1EE10FAC8BF4BF4807B6EF077
:10AA900073F837F033F8B8EEC88A0022B0EE409A67
:10AAA000B4EEC80A0392F1EE10FA98BF4BF0800B97
:10AAB00011F0E6FA444A03A992F8E02C11F0BEF82E
:10AAC000DDED038A2046F0EEE88AB4EEE88AF1EE86
:10AAD00010FAC8BF4BF0400B0DF0F0FE002842D139
:10AAE0004BF0200BB246384696F0FAF801284BD1CD
:10AAF0004BF0100BB146304EB8F1000F4FD0009B19
:10AB0000002B4CD0B4EEEBAAF1EE10FA47DCF4EED9
:10AB1000CB9AF1EE10FA42DCB4EEC89AF1EE10FADC
:10AB20003DD8B4EEE88AF1EE10FA38DDBAF1000F44
:10AB300035D0B9F1000F32D0D6ED007A04F16800BB
:10AB4000B8EE678AFEF794F807EE900AF8EEE77A17
:10AB500067EEAA7AB4EEE78AF1EE10FA1AD53268F7
:10AB600001323260E2E604F5B74008306DF0ACFF28
:10AB7000F0EE007A90ED007AB4EEE77AF1EE10FA9A
:10AB8000AED44FF0000AAEE7384696F0A9F801308F
:10AB9000B1D1ADE701212046FFF752FEC6E6002203
:10ABA000DFE7B8F1000FF0EE08AA0CBF4FF0000B82
:10ABB0004FF4007B37E700BFE0C70030CDCC4C3E00
:10ABC000235E8C3DE02E6542E882003000F5FF53A5
:10ABD0009FED257A70B5143388B0044602AD04F5B4
:10ABE000F44693E8070085E80700DDED047A0C36AB
:10ABF00077EE877A9FED1D7ACDED047AD4ED2B7A2E
:10AC0000F0EEE77AF4EEC77AF1EE10FA12D569F0B9
:10AC100073FFA2224FF4801169F026FFB4F9A2302D
:10AC2000F7EE006A07EE903AF8EEE77A86EEA77A3A
:10AC300084ED2B7AD4F8AC3001AA29463046019332
:10AC40006EF058F82046FFF74FFE2046FEF77CF9DD
:10AC50002046FEF74FFA2046FEF71AF82046FEF788
:10AC6000C5F808B070BD00BF0AE81C410000003400
:10AC700010B504461D202DED028B7BF075FA40B314
:10AC800004F5A043D3F8080F03689B6F984704F5B9
:10AC900081501921B0EE408A183060F079FF022807
:10ACA00014D00338012806D804F5B74008306DF0F9
:10ACB0000BFF90ED008A04F5F740B0EE480ABDECBA
:10ACC000028B6830BDE8104096F090B89FED028A84
:10ACD000F1E7BDEC028B10BD000000000F4A0260DE
:10ACE0000F4A02F17C01426002F504528160026267
:10ACF000A2F574720B4942620432C160043182626F
:10AD0000043201610839C2620432416106490263BA
:10AD10008161064A06494263C16170477CC81808D0
:10AD20001471003030AD0030804F003000340030FE
:10AD300024AD0030F8B504460E461C296AD8DFE879
:10AD400001F0140F181C27242E20692A6932696922
:10AD5000363A3E42464A4E51555A5E61696966002E
:10AD600000F5074494342046F8BD00F510446434DF
:10AD7000F9E700F50744D034F5E700F50844083456
:10AD8000F1E700F50D447834EDE700F50F44F6E700
:10AD900000F50E44F7E700F50E44C434E3E700F590
:10ADA0000F44DC34DFE700F50D44B434DBE700F595
:10ADB0000D44EC34D7E700F50B445034D3E700F5ED
:10ADC0000F444434CFE700F50D443834CBE700F5A9
:10ADD0001144A034C7E700F511446834C3E700F517
:10ADE0001144E6E700F512442834BCE700F5A04022
:10ADF000D0F86C47B7E700F50E443C34B3E700F5F4
:10AE00001344E6E700F5A040D0F87C4AABE700F534
:10AE10001444DAE700F50E470025B03757F8040B65
:10AE200050B103681B689847B04205D105F50E552F
:10AE30002C3554F8254096E70135052DEED1002438
:10AE400091E7000073B50B68054608460C469B6CFD
:10AE500016469847034605F5BA400E4A0421009667
:10AE6000103070F05BFF6BF0DFFB23680546204677
:10AE70001B6898470A21024628466BF031FB064BB7
:10AE800093F8F13E23B1054A137843F0040313709D
:10AE900002B070BD8CAB1808E8820030BCC900302D
:10AEA00070B518230C4A05460E4669F04FFA80B17A
:10AEB00031462846FFF73EFF30B10146074A284693
:10AEC000FFF7C0FF002070BD3146284669F0EAF860
:10AED000F8E70120F7E700BF1CAC1808ACAB180876
:10AEE00010B5002300F5A04400F5E04084F8203CB4
:10AEF000064BD0F83C0A93F8EB1EAFF0A7FBD4F852
:10AF0000080F0368BDE81040DB681847E88200308E
:10AF100070B5054608680C46164603685B69984795
:10AF200088B1306803685B69984760B905F5A0434C
:10AF3000D3F82C2F92F8D5202AB193F8EB3E13B911
:10AF40002846F7F763FE04480EF0A4FA2068036869
:10AF5000BDE870409B681847F0C8003070B500F538
:10AF6000A04504460C4ED5F8080F0368DB699847E6
:10AF70003074D5F8080F03681B689847F070D5F84F
:10AF8000080F0368DB6C9847014604F5E250BDE802
:10AF90007040043059F01CBD9DC9003070B52DEDD6
:10AFA000048B0646F0EE408AB0EE609A0C461546D9
:10AFB00079F010FA0368DB68984728B90023BDECE4
:10AFC000048B23602B6070BD736A186879F0FCFBFA
:10AFD000B36AB0EE408A186879F0F6FBF0EE491AD1
:10AFE000F0EE400A2946B0EE681A2046B0EE480A54
:10AFF000BDEC048BBDE8704031F028BE70B5002375
:10B0000006462DED028B88B0F0EE408A029306AD25
:10B01000039379F0DFF9036802ACDB68984758B90D
:10B0200094E8030085E803009DED060ADDED070ABC
:10B0300008B0BDEC028B70BD736A186879F0C4FB70
:10B04000B36AB0EE408A186879F0BEFBF1EE407A40
:10B050009FED1A7A8DED038ACDED027AF0EEC07A7B
:10B06000F4EEC77AF1EE10FA06D5B0EEC88AB4EE67
:10B07000C78AF1EE10FAD3D42146114811F046FAEE
:10B080008DED020ACDED030AB0EEC00AF0EEE00A43
:10B090002046B4EE600AF1EE10FA30FE200A35F0D8
:10B0A000F3FB04A88DED040ACDED050A35F094FC00
:10B0B000204688EE800A35F017FCB1E70000003426
:10B0C000804F0030094B93F8EB0E68B1B5EEC00A23
:10B0D000F1EE10FA07D9D3F82C3F93F8A100C31E64
:10B0E0005842584170470020704700BFE882003046
:10B0F000036A1B6893F8D50030B1044B93F8E92E2E
:10B100001AB193F8EB0E704701207047E8820030C7
:10B1100010B5036A04461868D1B10221B9F042F8AB
:10B12000E3699FED0C1A1868F0EE410A0368B0EE6F
:10B13000410A1B6B9847E369074A00211868D2ED62
:10B14000000A03689FED030A9B6EBDE81040184794
:10B150000121E3E7000000001871003010B5036A18
:10B1600004461868002930D00221B9F01BF8E369C1
:10B170001868AFF03BFA236A1B6893F8A130012BE3
:10B1800004D8E36901211868AFF0FCFF636918680F
:10B19000B3F01AF963691868B3F0AAF963699FED0F
:10B1A0000C0A1868B3F0ACFB63691868B3F022FCB2
:10B1B000E3699FED071A1868F0EE410A0368B0EEE4
:10B1C000410A1B6BBDE8104018470121CDE700BFC5
:10B1D0000000000013B5044601A914480DF0F8FB67
:10B1E00010B19DED010A0BE063691868B1F056FFDC
:10B1F00040B90F4B03F5236393ED000AB8EEC00A84
:10B2000002B010BD01AA03210A4819F01FF8002856
:10B21000E7D1074BDFED087A03F5236393ED000ACE
:10B22000B8EEC00A20EE270AEAE700BFE832003095
:10B23000E8A2003014AD00300AD7233CF0B5044634
:10B240002DED048B8FB0002940F01E818368DFED67
:10B25000908A03F580538F4EB3F9C238642BB8BF80
:10B26000642307EE903A0368B8EEE78A9B6F98472D
:10B270006268204628EE288AB2F93030B4EEC08ADF
:10B28000F1EE10FAD4BF96F8F25E0125002BCBBF89
:10B290005B42636907EE903A1B68CCBFF8EEE77A31
:10B2A000D3ED9F7AB2F92E30C8BF67EEA87A002B93
:10B2B000B8BF5B429BB25B4208EE103AA368B8EE9F
:10B2C000C88A03F58053B3F9C23828EE288AB4EE51
:10B2D000678AF1EE10FA37FE888A642BB8BF6423C0
:10B2E00007EE903A23689B6FB8EEE79A9847636938
:10B2F000626B1B6899EE280AD2ED001A93EDA11A31
:10B30000D3ED0C0A31F018F86368F0EE480A40F209
:10B310007E20B3F92E30002BB8BF5B429BB25B425C
:10B3200001EE103AB8EEC11A21EE281A30F0A4FB53
:10B330006369B0EE408A1868B1F0B0FE96F8F73E47
:10B340000746002B40F08D805348B4F0DBF800280E
:10B3500000F08780002F00F084800022002302A9E3
:10B360004D48DFED4E9ACDE90223CDE90423B4F038
:10B370004FF9002800F08580636906AE1B6803F56D
:10B380002E730FCB86E80F00314602A835F01CFE65
:10B3900068468DED0A0B8DED0C1BB7EEC00BB7EEBA
:10B3A000C11B8DED000A8DED011A35F015FBF0EE95
:10B3B000408A3B4E0AA9CDED0A9A96ED009AA6F175
:10B3C0002400CDED0B9AA6F2DC46CDED0C9AB4F03C
:10B3D00049F9F4EEC98AF1EE10FA08DDB0EEC99A27
:10B3E000DFED307AB4EEE79AF1EE10FA4DD5DDEDEF
:10B3F0000C7A9FED2D7AF4EEC77AF1EE10FA30DD7B
:10B40000B0EE007AF4EEC77AF1EE10FA29D5B6F86C
:10B41000F4345B0725D46368DFED247AB3F92E306A
:10B42000DFED236A002BB8BF5B429BB208EE103AF7
:10B43000B8EEC88A68EE277A87EEA67A27EE288AC1
:10B44000B5EEC08AF1EE10FA48BF9FED148A38EECF
:10B45000678ADFED187AB4EE678AF1EE10FA37FEEC
:10B46000888A6369B0EE480A29461868B2F068FD18
:10B47000636918680FB0BDEC048BBDE8F040B3F011
:10B48000B9BAF0EE698A94E700259FED048AE8E7EF
:10B490000AD7233CE8820030A0B70030000000004B
:10B4A000C4B70030000000343333B33E0AD7A33BA7
:10B4B0009A99193ECDCCCCBD036A186803685B69C4
:10B4C0001847000038B505462C482DED028B0CF0CE
:10B4D0008FFDEB6A041E4FF47A721B684FF0000177
:10B4E000D8BF4FF4FA74F6EE008AB3F90A0030F0D0
:10B4F0002BFB84422FDD07EE900AB8EEE77A07EEC9
:10B50000904AF8EEE77A27EE287A87EE278A2B68AA
:10B510002846D3F89030984740F2823030EE680ADF
:10B52000F5EE087AB7EE001AB1EE400AFEEE000A18
:10B5300080EE270A30F0A0FAF7EE007A77EEC07AB4
:10B5400028EE000A20EE080A20EE080AA7EE880A74
:10B55000BDEC028B38BD031BC4F57A7407EE103ABC
:10B5600007EE904AB8EEC77AF8EEE77A27EE287A27
:10B5700087EE278A38EE288AC9E700BFE832003014
:10B580002DE9F04F00F5004900F5A04605460F46AD
:10B5900090462DED028B99F8904783B089F890275B
:10B5A000D6F8080F03681B689847B84223D105F501
:10B5B0004053B8F11A0F83F8388C09D140B905F51A
:10B5C000E04506F6BC26D5F83C3A3268C3F8FC20C4
:10B5D000974B93F8F13E33B90124204603B0BDECFC
:10B5E000028BBDE8F08F4445F6D0924A137843F0C1
:10B5F00002031370F0E7B8F1020F0CD01B2F12D129
:10B6000005F508404146083003B0BDEC028BBDE8AB
:10B61000F04F01F0D9BA39462846FFF741FC0446FD
:10B620000028EBD1D9E739462846FFF783FB0446CB
:10B63000019020B93946284668F034FDCDE7D6F8A8
:10B640002C3F93F8D5B003688BF0010A5B699847EB
:10B6500005F50D43019AB4339A4208BF0120BBF1AE
:10B66000000F10D178F0B6FE03689B689847002859
:10B6700031D10198514603685B6898470446002819
:10B6800032D16D4A22E096F8EB3E002B00F0C180EB
:10B69000002800F0BE80DFF898B1DBF8080F0368DF
:10B6A0005B6998470446002840F0B3800198FFF793
:10B6B00009FFB0EE408AABF5A040F7F791FAB4EE7F
:10B6C000C08AF1EE10FA40F3A4805C4A0199284642
:10B6D000FFF7B8FB81E7019803681B6C98470446A5
:10B6E0000028C6D1564AF1E705F5BE4101AA284611
:10B6F00005F5405A0831FFF70BFC0198C6F8080F12
:10B700008AF8388C03681B6898474246014605F55D
:10B710009B506AF083FA05F5BA400021103077F0AB
:10B7200075FEFB1E012B02D9B91F4C424C4189F812
:10B730008E469AF9EA3923B105F56750243090F026
:10B74000CFF9D6F8080F03681B689847C21E05F5A5
:10B75000E04306F68C2150425041D3F83C2A012F99
:10B7600083F8C80A0968C2F8F81006F6BC21D3F8B5
:10B770003C2A0968C2F8FC1001D00B2F06D106F64E
:10B78000A426D3F83C3A3268C3F8FC202846FFF7D9
:10B79000E5FB274B93F8F13E002B7FF426AF1BE728
:10B7A00005F5405393F8E429002A3FF45BAFB3F862
:10B7B000042AD0077FF556AF93F8302A002A3FF4C9
:10B7C00051AFD6F82C2F92F8D520002A3FF44AAF7B
:10B7D00093F8383C0A2B7FF445AF96F8EB4E002CDB
:10B7E0007FF440AF174A71E717480DF08DFA002833
:10B7F000D6D1D6F8080F03685B6998470028CFD0E8
:10B80000019803685B69984704460028C8D10F4A2D
:10B810005CE7019803681B6998470028E4D00A4850
:10B820000DF060FA04460028DED1094A4EE700BF59
:10B83000E8820030BCC90030EE8B1A08D4AB18087F
:10B840000AAC1808F8AB1808E8320030E6AB180864
:10B85000721D1A080148FFF793BE00BFE83200309E
:10B8600010B52DED028B9FED118A82B0044620EEBB
:10B87000080A8DED010A93F045FA636901A9626B2C
:10B880001B6892ED001AD3EDA10A93ED0C0A60EE4D
:10B89000880A92F08BF89DED010ADFED057A20EE23
:10B8A000270A02B0BDEC028B10BD00BF0000C842E9
:10B8B0000AD7233C036A186803689B6A184700008C
:10B8C00010B5036AF0EE407A04461A6892F8D51073
:10B8D00061B91046B8F066FC236A1B6893F8A100B2
:10B8E00018B1012814BF0320022010BD15480378A9
:10B8F00033BBFFF7E7FB18BB134B93F8E91E11B1FD
:10B9000093F8EB1EB1B1F5EEC07AF1EE10FA0FD557
:10B9100093F8F63E63B901211046B8F043FC236A60
:10B920001B6893F8A130012B0CBF02200320DCE739
:10B930000221F1E710460221B8F034FC0420D4E7DC
:10B940000120D2E7F0C80030E882003010B52DEDBC
:10B95000028B044678F03EFD0368DB689847C8B167
:10B96000236B186878F030FFA368DFED0C7A03F5DD
:10B97000805303F6184203F61C4392ED008AD3ED80
:10B98000000A28EE278A31F029F920EE080ABDECDA
:10B99000028B10BD9FED020AF9E700BF35FA8E3C1D
:10B9A000000000000148F7F775B900BFE832003029
:10B9B0000148F8F757B900BFE83200300148FFF7F7
:10B9C000DFBD00BFE8320030F0B52DED028B8FB047
:10B9D0000D46044678F0FEFC036805AEDB68984728
:10B9E00000285BD063681B899B071BD549486DF015
:10B9F0006BF8DFED497A90ED007AB4EEE77AF1EE7C
:10BA000010FA0FDD6AF010FE3D216AF049FD0922AF
:10BA100005214248FFF7B4FD20B909220221204642
:10BA2000FFF7CCFF636893F95030002B36D000232A
:10BA30000593089323691868B6F000FEE369B0EE39
:10BA4000408A18680368DB6E984708AAF0EE400A3F
:10BA50003146B0EE480A2046FFF7A0FADDED057A40
:10BA60009FED2F7AF0EEE77AF4EEC77AF1EE10FA56
:10BA700008D5DDED087AF0EEE77AF4EEC77AF1EE5C
:10BA800010FA0BD4274F97F8F73E23B96AF0CCFD94
:10BA900049216AF005FD012387F8F73EF2EE040A1A
:10BAA0009FED210A95ED047BD5E90223D5E900013C
:10BAB000B1EE477BCDE90A2363698DED0C7BCDE9BF
:10BAC000080108A91868B2F0EDFA63691868B2F0C5
:10BAD0000FFD63691868B2F08DFFE3691D68636943
:10BAE0001868B1F09BFD304610498DED020ACDED8E
:10BAF000030A8DED041AFCF79DF8079B02A928465E
:10BB0000009396E80C00AEF021FE0FB0BDEC028B66
:10BB1000F0BD00BF08AD003000002F44E832003017
:10BB200000000034E88200300000000094C70030BC
:10BB3000F0B5704E0027044696F8F23E2DED028BCC
:10BB40008FB0039704971BB143691868B1F024F9CB
:10BB500078F040FC0368DB689847002855D063689C
:10BB60001B899A071BD564486CF0AEFFDFED637A42
:10BB700090ED007AB4EEE77AF1EE10FA0FDD6AF09C
:10BB800053FD3D216AF08CFC092205215C48FFF73A
:10BB9000F7FC20B9092202212046FFF70FFF636856
:10BBA00093F950308BB35648F8F75CF8E3689FED93
:10BBB000558A20461B68D3ED097AF4EEC87AF1EE77
:10BBC00010FAAABF9FED500AF0EE047A67EE807A71
:10BBD000B6EE000A27EE800AFFF710FACDED040A50
:10BBE0008DED030AB0EEC00AB4EEC80AF1EE10FA09
:10BBF00022D5F0EEE00AF4EEC80AF1EE10FA1BD5F9
:10BC0000424BB3F8F4349B0722D400230AAD86F8E4
:10BC1000FE3E96F8F73E2BB93D48B3F073FCC8B929
:10BC200086F8FE0E606901230A972A460B9703A93E
:10BC30000068B1F017F93DE096F8F73E23B96AF0D5
:10BC4000F3FC49216AF02CFC012386F8F73EDCE77F
:10BC50000023FAE70123002229462D4886F8FE3EFC
:10BC6000002305970697CDE90A23CDE90C23B3F00D
:10BC7000CFFCD4F814C030B9DCF8003003F52E73D3
:10BC80000FCB85E80F00DCF8001005AA204801F56D
:10BC90004071B3F009FD606901230797089705AA71
:10BCA0000093294607AB0068B1F014F996F8FE3E00
:10BCB000002BB7D063691868B2F01AFC6369186882
:10BCC000B1F0ACFCE369284612498DED070ACDEDD1
:10BCD000080A8DED091A1C68FBF7ACFF0C9B07A93D
:10BCE0002046009395E80C00AEF030FD0FB0BDEC9F
:10BCF000028BF0BDE882003008AD003000002F4418
:10BD0000E8320030000000340AD7233CE8B20030AB
:10BD1000A0B7003094C7003013B504460191FFF777
:10BD200007FF0199204602B0BDE81040FFF786BA30
:10BD30001B4B10B593F8F73E86B004466BBB002250
:10BD4000002369461748CDE90023CDE90223CDE958
:10BD50000423B3F06BFA032807D8DFE800F0150ED0
:10BD6000020869462046FFF72FFE06B010BD0D48B9
:10BD7000B3F07EFA30B10128F7D100212046FFF759
:10BD8000CBFFF2E70121F9E768F0B6FE40F2553249
:10BD90004FF4801168F068FEEFE70021EFE700BF85
:10BDA000E8820030B0B8003008B5034619B9064A39
:10BDB00092F9B8241AB91846FFF7AEFF08BDBDE8DE
:10BDC0000840FFF7B5BF00BFE8B200300148FEF7FA
:10BDD00037BD00BFE832003000487047F88F0030B0
:10BDE00043689FED050AB3F9323007EE903AF8EE5A
:10BDF000E77A27EE800A70470AD7233C08B5064841
:10BE0000F6F734FF07EE900A9FED040AF8EEE77AA2
:10BE100027EE800A08BD00BFE83200300AD7233C75
:10BE200043689FED050AB3F9343007EE903AF8EE17
:10BE3000E77A27EE800A70470AD7233C30B51D4DBC
:10BE40008DB000230022044606A9D5F8440ACDE9A6
:10BE50000623CDE90823CDE90A23B1F0F7FB0AA9AF
:10BE6000D5F8440AB1F046FC9FED130A68469DEDF3
:10BE7000087B9DED065BF7EEC76BB7EEC55B9DEDEE
:10BE80000A7B8DED005ACDED016AB7EEC77B8DEDD3
:10BE9000027A35F015FA022203A920468DED030A35
:10BEA000CDED040A8DED051A18F018FE20460DB0F0
:10BEB00030BD00BFE8A200300000C842014B0122A3
:10BEC0001A707047E4C700300020704700207047A8
:10BED0000020704700207047002070470020704706
:10BEE0000020704700207047002070479FED010A36
:10BEF000704700BF000000009FED010A704700BFBF
:10BF0000000000009FED010A704700BF0000000024
:10BF100000207047002070470020704701207047C4
:10BF200000207047002070470020704701207047B4
:10BF300000207047012070470120704700207047A3
:10BF40000120704701207047002070470020704793
:10BF50000048704734AC18080048704734AC1808E3
:10BF6000836803F5805393F82C3CDB0706D5002348
:10BF7000022280F83830024BC3F8002F01207047AE
:10BF8000E882003090F8383053B9836803F5805365
:10BF900093F82C3CDB0742BF034B0122C3F8002F70
:10BFA000002380F838307047E8820030012380F8A1
:10BFB000383070472DE9F04300251E460446884678
:10BFC00017462DED0C8B95B0436AF7EE00CADFEDF6
:10BFD000DABA0295039504950595069507951868B4
:10BFE00078F0F2FBA36AF0EE408A186878F0ECFB78
:10BFF000236BB0EE409A186878F0E6FB28EEA87A3A
:10C00000A368B0EE40BAA9EE097A03F5805303F6AF
:10C01000E83203F6EC33D3ED000AD2ED00AAB7EE16
:10C02000C77A6AEEABAAB1EEC76BB7EEC66BB4EED9
:10C03000EC6AF1EE10FAC2BFCCEE867A68EEA78AFF
:10C0400029EE279AB0EE680A30F0C8FDA36860EECA
:10C050002AAA03F58053B0EE490A03F6E83203F644
:10C06000EC3392ED00AAD3ED000A30F0B7FDA068E2
:10C070002AEE2BAA00F5E05320EE0AAAD3ED009A8F
:10C08000D3ED010AB0EE4B0A30F0A8FD636869EE0B
:10C09000AB9A93F9743060EE299A002B00F0D480AB
:10C0A000E3691B6893ED1B0A93ED1C8AB7EEC00A87
:10C0B0002FF0CAFCB7EEC0CB93209FEDA01ADFEDA6
:10C0C000A00AB0EE4C0A2FF0D7FC6368D3ED1B7AC0
:10C0D00020EE670A8DED020AB7EEC80A2FF0B4FC15
:10C0E000B7EEC0DB97209FED951ADFED950AB0EE15
:10C0F0004D0A2FF0C1FC63680495D3ED1C7A93F9C7
:10C10000743020EE670A022B8DED030A75D1E369C6
:10C11000DFED8CDA1B68D3F85021B2F9002008EE6D
:10C12000102AB8EEC88A28EE2D8AB4EEC8CAF1EEFD
:10C1300010FA3FDD93ED051A38EE4C0AA368DFEDE7
:10C14000820A21EE2D1A03F5DF53626BD3ED027ADA
:10C15000D2ED001A67EEAB7AC7EEA00A30F0ECF829
:10C16000DDED027A77EE807ACDED027AB4EEC8DAB0
:10C17000E3691B68F1EE10FA38DD93ED061A38EE2C
:10C180004D0AA368626B21EE2D1A03F5DF53D2ED41
:10C19000001AD3ED020A60EEABBADFED6B0ACBEE0C
:10C1A000A00A30F0C9F8DDED037A37EE800A8DED94
:10C1B000030A22E0B1EE480AB4EECC0AF1EE10FA1E
:10C1C000D4DD93ED051A30EE4C0AA368626B21EEC4
:10C1D0002D1A03F5DF53DFED5C0AD2ED001AD3ED23
:10C1E000027A67EEAB7AC7EEA00AB7E7B1EE488AEB
:10C1F000B4EECD8AF1EE10FABFDCE36910AD0DF1BB
:10C200003009D3F800C00CF184030FCB85E80F0090
:10C2100008AD89E80F0085E80F0005AB02AA2946A2
:10C220006046AEF063FF636893F97430022B16D159
:10C23000DDED057A7AEEA7AADDED067A3AEE27AAB9
:10C24000DDED077A79EEA79AC8ED00AA87ED00AA7E
:10C25000C6ED009A15B0BDEC0C8BBDE8F083B0EED6
:10C26000C97ADFED3A0AF0EEE87AB0EECBBA8DED9E
:10C27000087AB7EE001AB4EEE77ACDED017A8DEDCB
:10C280000CBAF1EE10FA54BF284601A8D0ED007A9E
:10C29000F4EECB7AF1EE10FAD8BF484690ED000AE2
:10C2A000B5203CEEC00A2FF0E7FBA36905A8D3ED4B
:10C2B000967A20EE270A35F003F88DED071AB0EED6
:10C2C000EA1ABD20F0EEC07A8DED050ACDED060A22
:10C2D0003AEE800A31EE671AB0EEC11AF1EE410A69
:10C2E0002FF0CAFBF0EE40AA9DED060AB0EECA1A86
:10C2F000C220F0EEC07A3AEE000A31EE671AB0EED4
:10C30000C11AF1EE410A2FF0B7FBB0EE40AA9DED45
:10C31000070AB0EEE91AC720F0EEC07A39EE800ABB
:10C3200031EE671AB0EEC11AF1EE410A2FF0A4FB0C
:10C33000F0EE409A88E700BF35FA8E3C920A063F3D
:10C34000920A06BFD4023739C2B8323E000000005C
:10C3500010B52DED028B84B0044603AB01A902AAEF
:10C36000FFF728FE236A186890F8D51000293FD1FE
:10C37000B7F018FF2046FFF7A5F8236AB0EE408A11
:10C380001B6893F8A110012941D0032948D051B965
:10C39000E36901211868AFF075FDE3691868AEF034
:10C3A0000FF99FED248AE3691868A36803F58053A9
:10C3B00093F82C3C9B073AD5AEF0C4FCE3691868AF
:10C3C00003681B6C9DED031ADDED020A9DED010A69
:10C3D0009847E369184AB0EE480A18680021D2ED80
:10C3E000000A03689B6E984704B0BDEC028B10BD39
:10C3F000124B93F8F32E32B9D3F8003F022B04D13D
:10C4000090F8A1300BB90121B2E70221B0E7E3694E
:10C410001868AFF037FDE3691868AEF0E7F8C0E7D9
:10C42000D9790029BFD12046FFF7D0FCBBE70368CC
:10C43000DB6BC7E70000000018710030E8820030B5
:10C440008368DFED077A03F6EC1393ED000AB4EE90
:10C45000E70AF1EE10FA01DAFFF72EB8704700BFD5
:10C460000000003470470000012070470120704731
:10C47000022070470020704700207047012070475D
:10C480000020704781F001007047000001207047D4
:10C490000120704701207047012070470048704715
:10C4A000DCAC180800487047E8AC180830B52DED32
:10C4B000028B436983B004461868B0F0E1FE18B9F6
:10C4C00063691868B2F02EF9636920461D68FFF7AA
:10C4D00095FCB0EE408A2046FFF782FC20468DEDA9
:10C4E000010AFFF79DFCDDED010AB0EE401A284677
:10C4F000B1EE480AB0F0E0FD636920461D68FFF721
:10C500007DFCB0EE408A2046FFF76AFC20468DEDA8
:10C51000010AFFF785FC2846B0EE401ADDED010A5E
:10C52000B1EE480AB0F038FE012003B0BDEC028B3A
:10C5300030BD000030B52DED048B436987B0044653
:10C54000DFED679A1D68FFF759FCB0EE408A204680
:10C55000FFF746FC20468DED010AFFF761FCDDED9B
:10C56000010AB0EE401A2846B1EE480AB0F0A4FD28
:10C570002046FFF71DFAE3691868D0F85031B3F987
:10C58000003008EE103A0368B8EEC88ADB6E9847B0
:10C5900004AAF0EE400A03A928EE298A2046B0EE4C
:10C5A000480AFEF7FBFC2046FFF7D0F92046F0EEE4
:10C5B000408AFFF7F7F92046B0EE408A8DED050A74
:10C5C000FFF71CFCB0EE409A2046FFF709FC2B2039
:10C5D000B0EE401AF1EE490AB0EE480A2FF04CFADC
:10C5E00020468DED050AFFF76BF9042813D8DFE824
:10C5F00000F0032F252A4F00E3691868ADF0E0FF33
:10C60000E36900211868AEF0BDFD63699FED350A4E
:10C610001868B2F075F9E369B0EE681ADDED040A46
:10C6200018689DED030A03681B6B984763691868D7
:10C63000B2F0E0F907B0BDEC048B30BDE369012135
:10C640001868AEF09FFDE3691868ADF0CFFFDCE736
:10C65000254D2B7883B963684520DFED247AB2EE4F
:10C66000041A93ED030ADFED1F0A20EE270A2FF0CC
:10C6700003FA28460CF0F4FE20469DED050AFFF76C
:10C68000EFF805A918488DED050A0CF025FFC2E763
:10C69000236A02211868B7F085FDE36904AA03A99B
:10C6A0001B681348D3F85031B3F9003000EE103A4C
:10C6B000B8EEC00A20EE290A92F098FA20469DEDC5
:10C6C000050AFFF7CDF80B488DED050A0CF09EF931
:10C6D00063699DED050A1868B1F024FC9BE700BF73
:10C6E000D402373900000000F0C800300AD7233CDC
:10C6F00044AE0030FC8E00300020704700207047B0
:10C7000090F80933002B14BF1B2003207047000052
:10C71000002070470120704790F8E002062804D0FE
:10C72000A0F10A03584258417047012070470000A9
:10C73000012070470120704790F80903034A044B19
:10C74000002814BF10461846704700BFA8581808A4
:10C75000C1321A0890F80903034A044B002814BF99
:10C7600010461846704700BF90AD1808C1321A082D
:10C7700090F8E0020B3818BF0120704790F8093399
:10C780002BB9044BD3F8D80A00F001007047002001
:10C79000704700BFE8820030024BD3F8D80AC0F3DC
:10C7A000C0107047E882003090F8E03223B9034BA4
:10C7B000187880F00100704700207047C8C800302A
:10C7C00038B590F8E0420546012C01D0002038BD74
:10C7D000C36818680368DB6998470028F6D1EB68DE
:10C7E00020461B6883F87449F1E70000C368002203
:10C7F00001201B6883F8742970470000002370B57E
:10C800002DED028B80F8093386B0B0F96C30044608
:10C810000D46012B01DC002946D0236A274E1B68F8
:10C8200093F8D53073BB0723254884F8E0320368BA
:10C83000022B02D10021FAF7C1FFE36801259FED29
:10C84000218A1868B0EE480A9FED1A1BB0EE412B02
:10C85000B0EE413BB4F0DAFF04F5217084EDCD8AEF
:10C8600084EDCE8A84EDCF8A84F8085335F062FDDA
:10C87000154805F0CDFB0023144886F8F73EB2F0CA
:10C88000B3FB11E096F8EB3E002BCCD004F138005E
:10C8900038F0F0F805460028C5D12046FFF79CFA8D
:10C8A0000B4A02216FF03AFA284606B0BDEC028B23
:10C8B00070BD00BF0000000000000000E8820030F2
:10C8C00094C700300000000060C10030B0B80030F4
:10C8D00098AD180810B50446094890F84438012B63
:10C8E00003D100F5046035F08FFD064890F8511B28
:10C8F00000F6D8207AF0B4FD002384F8093310BD87
:10C90000E8B20030E8A2003010B5084B04462DED27
:10C91000028BB0EE408AD3F8480AB4F09BFA0120AB
:10C9200084EDCE8ABDEC028B10BD00BFE8A20030C2
:10C9300010B5084B04462DED028BB0EE408AD3F8BB
:10C94000480AB4F097FA012084EDCF8ABDEC028B3F
:10C9500010BD00BFE8A2003010B5084B04462DED15
:10C96000028BB0EE408AD3F8480AB4F091FA012065
:10C9700084EDCD8ABDEC028B10BD00BFE8A2003073
:10C98000C3681B68D868B0F0D1BF000038B5D0F8D4
:10C99000E43204460D461BB9BFF0C2FDC4F8E40200
:10C9A000BFF0BEFDD4F8E432C01A4FF47A73B0FB86
:10C9B000F3F0B4F8E232984209D32046FFF70CFABC
:10C9C0002B88044A06216FF0A9F9012038BD002008
:10C9D000FCE700BFB4AD180808B52DED028B90F848
:10C9E000E0329FED0A8A052B0AD1094BD3F8503A61
:10C9F0005868B0F0BFFE20EE080ABDEC028B08BDFF
:10CA0000C368186803689B699847F4E7E02E65429D
:10CA1000E8A2003090F8E032052B06D1054BD3F8A0
:10CA2000503A58681C3033F0D7BFC36818680368A1
:10CA30001B691847E8A20030836833B9C36823B97B
:10CA40004068003818BF012070470120704700007F
:10CA500090F8E0328B4206D00B2B80F8E01202D126
:10CA60000148FCF79FBD7047E832003073B50123E1
:10CA70001E4E04460A4680F87130D6F8083F8342BD
:10CA800012D10125019284F80953D6F8080F0368E2
:10CA90001B689847019A0146154869F0BFF896F857
:10CAA000F10EB0B9284612E001910321FEF786FF8E
:10CAB000019A05460028E4D184F8710069F0B4FDBC
:10CAC0001B220A2169F00CFD96F8F10E38B902B06C
:10CAD00070BD084A137843F002031370F7E7054A64
:10CAE000137843F004031370DCE700BFE8820030E2
:10CAF00048460030BCC9003030B585B004460D460C
:10CB000001466846FFF79AF9694604F1380038F0A3
:10CB100015FCC0B969F088FD1B220A2169F0E0FC10
:10CB20000C4B93F8F13E23B10B4A137843F0040306
:10CB300013702046FFF750F9084A04216FF0EEF811
:10CB4000002005B030BD2946204605B0BDE8304084
:10CB5000FFF78CBFE8820030BCC90030C8AD1808B0
:10CB600030B585B004460D4601466846FFF766F9C4
:10CB7000694604F1380038F005FCC0B969F054FD8D
:10CB80001B220A2169F0ACFC0C4B93F8F13E23B157
:10CB90000B4A137843F0040313702046FFF71CF987
:10CBA000084A04216FF0BAF8002005B030BD2946CC
:10CBB000204605B0BDE83040FFF758BFE88200309E
:10CBC000BCC9003004AE18087FB505460E460146C4
:10CBD000684605F13804FFF731F96946204638F018
:10CBE000D1FBB8B92046694638F0A8FB044688B99D
:10CBF00069F01AFD1B220A2169F072FC0C4B93F8B4
:10CC0000F13E7BB92846FFF7E7F80A4A04216FF0A6
:10CC100085F804E031462846FFF728FF0446204601
:10CC200004B070BD044A137843F004031370E9E7BD
:10CC3000E88200303CAE1808BCC9003010B590F84E
:10CC4000E0420A2C16D1B0F80E430C8090F8141371
:10CC50001170D0F818231A60029BD0F81C231A60B8
:10CC6000039BB0F920231A80049BB0F922230120F2
:10CC70001A8010BD0020FCE790F8E0320A2B06D1A4
:10CC8000B0F80E338B4204BF012380F80C33704799
:10CC900030B5044687B011480CF024F80546D0B1F1
:10CCA00007230022694684F8E0320023CDE90023FF
:10CCB000CDE90223CDE90423E3681868B4F058F8FD
:10CCC000E36869460022186803689B68984700215A
:10CCD0000348FAF773FD284607B030BDE83200304C
:10CCE00094C7003070B5054644480C462DED028BC4
:10CCF00086B0FFF7A1FE60B967F0FEFE40F2751244
:10CD00004FF4801106B0BDEC028BBDE8704067F0B7
:10CD1000ABBE6B6920461B6893EDB28B17F0ECF944
:10CD20000328B7EEC88B42D1EB6801A91868B4F0AC
:10CD300027F9064600283AD0DDED017A9FED307ADA
:10CD400038EE678AD4ED017AF8EEE77A67EE877AF3
:10CD5000CDED007A2B4BB7EE007ADFED2B7A002178
:10CD600093F8EB3E2948002B07FE877A38EE077AC6
:10CD7000DDED007AB4EE677AF1EE10FA48BFB0EE5E
:10CD8000677A8DED007AFAF719FD6B691868B1F0D2
:10CD9000C9FC31469DED000A1D480CF01DFE002126
:10CDA0002846FFF755FE06B0BDEC028B70BD94E837
:10CDB0000F0002AE86E80F00164B02213046D3F872
:10CDC000342AD3F8383A04926A46059317F03EFAAB
:10CDD00088B969F029FC0222152169F081FBDDED9B
:10CDE000037AB0EE487ADFED066AF8EEE77AA7EE4E
:10CDF000A67A8DED007A0026ACE700BF14AD0030B6
:10CE00000AD7233CE88200300000000094C70030BD
:10CE1000C8C80030E8A20030F0B52DED028BC36821
:10CE20008DB004460F461868B4F080F8002849D148
:10CE30000022002394F8E012CDE90023CDE902237B
:10CE4000CDE9042391B906A92D48CDE90623CDE902
:10CE50000823CDE90A230CF0F1FD38B106AD6E468A
:10CE60000FCD0FC695E8030086E80300D4EDCD7A18
:10CE70009FED248AE368F4EEC87A9FED230A1868D0
:10CE8000F1EE10FA9DED001B27FE800A9DED022BAE
:10CE90009DED043BB4F0BAFC94EDCE0AB4EEC80AA2
:10CEA000F1EE10FA03DBE3681868B3F0D3FF94EDFA
:10CEB000CF0AB4EEC80AF1EE10FA03DBE368186893
:10CEC000B3F0D8FFE36839461868B4F0B9FB0546FB
:10CED00088B10E4B1B68022B09D0032B03D10C4BDE
:10CEE00093F9553E1BB100210848FAF77BFC01215C
:10CEF0002046FFF7ADFD28460DB0BDEC028BF0BD1E
:10CF0000C8C80030000000340000000094C70030A2
:10CF1000E862003010B504462DED028B4369DFED69
:10CF20003E8A1868E3689FED3D8A1B68D3ED090AC5
:10CF300093ED050AF4EEE80A20EE080AF1EE10FA85
:10CF4000ACBF60EE880AF0EE040AAFF0B5FE63698C
:10CF50001868E3681B68D3ED090A93ED050AF4EE3F
:10CF6000E80A20EE080AF1EE10FAACBF60EE880A7B
:10CF7000F0EE040AAFF008FF63691868B0F08EF8AD
:10CF800018B963691868B1F099F9E3681B6893ED03
:10CF9000070A93ED0B1A20EE080AD3ED060A63691F
:10CFA00021EE081A60EE880A1868B0EEC00AB0F0E8
:10CFB00083F8E3681B6893ED070A93ED0B1A20EEE4
:10CFC000080AD3ED060A636921EE081A60EE880AA2
:10CFD0001868B0EEC00AB0F0DFF863691868B0F006
:10CFE0004FF918B963691868B1F09CFB00210C482F
:10CFF000FAF7E4FB0B4893F09DFF0B4B0022204611
:10D00000022183F8F72E83F8FE2EBDEC028BBDE8DB
:10D010001040FFF71DBD00BF000000340AD7233CBD
:10D0200094C70030D0AE0030E88200300C4B10B511
:10D030000446D3F8500A90ED030A00F1180190F865
:10D040005820B3F0A5FA07480368022B02D0082144
:10D05000FAF7B4FB20460521BDE81040FFF7F8BC05
:10D06000E8A2003094C70030F0B5574D99B004469F
:10D070000E46D5F8500A17468DED010AB3F0DAF8DE
:10D080009DED010AD5F8500AB3F044F9D5F8500ADD
:10D0900090ED030AB0EEC00A0FB1B1EE400AB3F052
:10D0A0002FF9002200230CA9D5F8500ACDE90C2352
:10D0B000CDE90E23CDE9102303AAB3F047F9F0EE32
:10D0C000087A9DED037AB4EEE77AF1EE10FA71DD9D
:10D0D0000CA89FED3B0B35F035F8022212A908A8E9
:10D0E0008DED120B8DED141B8DED162B17F02AFD17
:10D0F000314608A816F0EAFFE36808A91868B4F0FA
:10D100009FFA10B93148FCF739FE636904A906A8F3
:10D110001B6893EDB07B93EDAE6BD5F8503AB7EE4C
:10D12000C77BB7EEC66B8DED057A8DED046A93ED86
:10D13000087B93ED066BB7EEC77BB7EEC66B8DED44
:10D14000077A8DED066A33F083FB12A88DED120A83
:10D15000CDED130A33F040FC1D4B1B68022B20D091
:10D16000D5F8503A00219FED1B7AD3ED0C7A184880
:10D17000F4EEC77AF1EE10FABEBFD3ED027A9FED5E
:10D18000167A67EE877AB4EEE70AF1EE10FA0EDD52
:10D19000F1EE047AB4EEE70AF1EE10FA07DDFAF7E1
:10D1A00021FB04212046FFF753FC19B0F0BDFAF72C
:10D1B00005FBF6E72046FFF739FFF6E7AFF30080FF
:10D1C0000000000000005940E8A20030E8320030C2
:10D1D00094C70030000000340AD7233C344B70B5AC
:10D1E0002DED028BD3F8484A0646DFED328AD4EDA6
:10D1F000090AD3F8445AF4EEE80A9FED2F8A94ED19
:10D20000050A2846F1EE10FA20EE080AACBF60EEDF
:10D21000880AF0EE040AAFF04FFDD4ED090A94ED50
:10D22000050A2846F4EEE80A20EE080AF1EE10FAA4
:10D23000ACBF60EE880AF0EE040AAFF0A5FD284608
:10D24000AFF02CFF10B92846B1F038F894ED070A7A
:10D25000284694ED0B1A20EE080AD4ED060A21EEBA
:10D26000081A60EE880AB0EEC00AAFF025FF94ED10
:10D27000070A94ED0B1A284620EE080AD4ED060A98
:10D2800021EE081A60EE880AB0EEC00AAFF084FF03
:10D290002846AFF0F5FF10B92846B1F043FA002157
:10D2A0000648FAF78BFA0123BDEC028B337070BD90
:10D2B000E8A20030000000340AD7233C94C70030B5
:10D2C000074808B5D0F8D83A9B0704D50121A0F546
:10D2D000A040F5F733FB0348BDE808400CF0DAB98D
:10D2E000E8820030C8C8003030B589B00446FDF788
:10D2F000FFFE30B10021204609B0BDE83040FDF707
:10D300002DBF236A02211868B6F04CFFE368186845
:10D3100003681B6A984701461048FCF727FC6369BD
:10D320001868B1F067FBE3691D68636905AC1868AC
:10D33000B0F074F920460A498DED020ACDED030ADA
:10D340008DED041AFAF776FC079B02A92846009394
:10D3500094E80C00ADF0FAF909B030BDE8320030C5
:10D3600094C7003038B50446FDF7C2FE054628B123
:10D3700020460021BDE83840FDF7F0BE236A0221B7
:10D380001868B6F00FFF29462046BDE83840FEF782
:10D390000BBD00000021014807F0ECBAC4C2003008
